:100000000C94C8160C94F9160C94F9160C94F91665
:100010000C94F9160C94F9160C94F9160C94F91624
:100020000C94F9160C94F9160C94F9160C94F91614
:100030000C94F9160C94F9160C94F9160C94F91604
:100040000C94F9160C94C86D0C94F9160C94F916CE
:100050000C94F9160C94F9160C9469B90C94EEB73B
:100060000C94F9160C9427B60C94FEB50C94F91662
:100070000C94F9160C94F9160C94F9160C94F916C4
:100080000C94F9160C94F9160C94F9160C94F916B4
:100090000C94F9160C94F9160C94F9160C94F916A4
:1000A0000C94F9160C94F9160C94F9160C94F91694
:1000B0000C94F9160C94F9160C94F9160C94F91684
:1000C0000C94F9160C94F9160C94F9160C94D5B5F9
:1000D0000C94ACB50C94F9160C94F9160C94F91612
:1000E0000C94F91600B503B5F2B4F6B4FCB43AB505
:1000F00007B50BB511B515B519B51FB523B527B59E
:100100003AB52DB531B535B50AB70FB714B71EB727
:1001100028B7A1B732B73AB742B74CB756B760B7AE
:100120006FB779B7A1B783B78DB797B7084AD73BF1
:100130003BCE016E84BCBFFDC12F3D6C74319ABDB6
:1001400056833DDA3D00C77F11BED9E4BB4C3E91DA
:100150006BAAAABE000000803F05A84CCDB2D44EC9
:10016000B93836A9020C50B9918688083CA6AAAACB
:100170002ABE000000803F004E414E494E4954596E
:10018000494E46CDCCCC3D0AD7233C17B7D1387762
:10019000CC2B329595E6241FB14F0A000020410078
:1001A00000C84200401C4620BCBE4CCA1B0E5AAEC2
:1001B000C59D7447322F473320626164207061729D
:1001C000616D65746572730A00205A3A20002059E7
:1001D0003A200042656420583A20004D657368203B
:1001E000706F696E742063616E6E6F74206265203B
:1001F0007265736F6C7665640A004E6F206D6F7662
:10020000652E00456E642066696C65206C697374A8
:100210000A00426567696E2066696C65206C6973C7
:10022000740A005344207072696E74696E672062AC
:1002300079746520004E6F74205344207072696E8B
:1002400074696E670A0046696C652064656C657444
:1002500065643A0044656C6574696F6E2066616917
:100260006C65642C2046696C653A20006F70656E81
:10027000206661696C65642C2046696C653A2000D3
:100280005072696E742074696D653A200050726F07
:100290007465637465642050696E0A006F6E2E0A7F
:1002A000006F66662E0A0047323620446562756725
:1002B00020006D0046696C616D656E742075736514
:1002C000643A200053746174733A20002C204C6F00
:1002D0006E67657374206A6F623A2000546F7461B0
:1002E0006C2074696D653A200053746174733A2010
:1002F000002C204661696C65643A20002C20466918
:100300006E69736865643A20005072696E74733A5E
:10031000200053746174733A2000452569202573C9
:10032000005761686E616F204475706C6963617419
:100330006F7220693320506C757320726561647927
:100340002E004B494C4C45442E20004D313133207A
:1003500053006F6B0048656174696E6720646F6E4F
:10036000652E0020573A0045256920257300576106
:10037000686E616F204475706C696361746F722080
:10038000693320506C75732072656164792E007A30
:100390005F70726F62653A20007A5F6D696E3A2015
:1003A00000795F6D696E3A2000785F6D696E3A2062
:1003B000005265706F7274696E6720656E64737445
:1003C0006F70207374617475730A00536574746977
:1003D0006E672054726176656C20416363656C655D
:1003E000726174696F6E3A200053657474696E6748
:1003F000205265747261637420416363656C657239
:100400006174696F6E3A200053657474696E672079
:100410005072696E7420416363656C6572617469C2
:100420006F6E3A200053657474696E67205072696C
:100430006E7420616E642054726176656C20416335
:1004400063656C65726174696F6E3A2000205A00B2
:10045000205900580020204D61783A2000205A0091
:10046000205900580020204D696E3A20004F6E2020
:10047000004F666600536F667420656E6473746F18
:1004800070733A200000013D3E3C36FF40413F186A
:10049000FF434542171919FF0305FFFFFF3A3B3998
:1004A000FFFF034404FF37FFFFFFFFFFFF43290A5D
:1004B0000061626C656420286D696E2074656D70E2
:1004C0002000436F6C6420657874727564657320D6
:1004D00061726520004D3130362053300041757413
:1004E0006F205049442066696E6973686564002313
:1004F000646566696E65202044454641554C545FED
:100500004B64200023646566696E6520204445467F
:1005100041554C545F4B69200023646566696E65E4
:10052000202044454641554C545F4B7020005049B3
:1005300044204175746F74756E652066696E6973C9
:10054000686564212050757420746865206C61733F
:1005500074204B702C204B6920616E64204B64200A
:10056000636F6E7374616E74732066726F6D206258
:10057000656C6F7720696E746F20436F6E66696774
:1005800075726174696F6E2E680A0050494420418B
:1005900075746F74756E65206661696C6564212081
:1005A00074696D656F75740A00544845524D414C2D
:1005B0002052554E4157415900546865726D616C27
:1005C0002052756E617761790048656174696E6764
:1005D000206661696C65640048656174696E6720B6
:1005E0006661696C656400504944204175746F749C
:1005F000756E65206661696C6564212054656D7057
:100600006572617475726520746F6F2068696768C0
:100610000A00204B643A2000204B693A2000204B0E
:10062000703A20000A20436C61737369632050495B
:1006300044200A002054753A2000204B753A2000CF
:10064000206D61783A2000206D696E3A20002064A8
:100650003A200020626961733A20004F66660A0002
:100660004661646520486569676874200042656476
:10067000204C6576656C696E6720004661696C6523
:100680006420746F20656E61626C65204265642031
:100690004C6576656C696E670A004F6666736574B3
:1006A00073206170706C696564004572723A205401
:1006B0006F6F206661722100546F6F206661722037
:1006C00066726F6D207265666572656E6365207017
:1006D0006F696E740A003A2000207A5F6D696E3A85
:1006E00020202D3230207A5F6D61783A2020323020
:1006F0000A0050726F6265205A204F6666736574F7
:10070000004E6F2063617365206C696768740A002E
:100710004163746976652045787472756465723AD0
:100720002000556E6B6E6F776E20636F6D6D616E1E
:10073000643A202200496E76616C6964206B6579A9
:100740002076616C75652000496E76616C69642065
:100750006B65792076616C756520004530204338E3
:10076000205531004D3330332053004D3130362089
:100770005332353500496E76616C6964206B65795A
:100780002076616C75652000526563656976696ED7
:1007900067204672616D6520284D656173757265CD
:1007A000732900496E76616C6964206B65792076E7
:1007B000616C75652000473932204530004738327A
:1007C0000041646A7573743A206F6C64203D2000A8
:1007D0002C206578706563746564203D20002C20B2
:1007E0006D65617375726564203D20002C206E6517
:1007F00077203D2000526563656976696E67204603
:1008000072616D6520284D6561737572657329008D
:10081000473932204530004D383300496E76616CDF
:100820006964206B65792076616C756520004731BD
:10083000205A3330204632303030004731205A3091
:100840002046313030300047312058313030205987
:10085000313030204636303030004731205A313088
:10086000204632303030004C6576656C20737465FC
:10087000702035004731205A30204631303030006A
:100880004731205833302059313730204636303008
:1008900030004731205A3130204632303030004C61
:1008A0006576656C20737465702034004731205A7A
:1008B0003020463130303000473120583137302039
:1008C000593330204636303030004731205A3130ED
:1008D000204632303030004C6576656C207374658C
:1008E000702033004731205A3020463130303000FC
:1008F0004731205831373020593137302046363093
:100900003030004731205A3130204632303030000C
:100910004C6576656C207374657020320047312019
:100920005A302046313030300047312058333020A3
:10093000593330204636303030004731205A31307C
:10094000204632303030004C6576656C207374651B
:10095000702031004732380047393000496E7661E7
:100960006C6964206B65792076616C756520004D3B
:10097000353030004D353032004D35303000496E65
:1009800076616C6964206B65792076616C75652091
:10099000004D35303000526563656976696E6720B9
:1009A0004672616D652028416363656C6572617490
:1009B000696F6E2053657474696E677329004D35D5
:1009C000303000526563656976696E6720467261F2
:1009D0006D652028416363656C65726174696F6E33
:1009E0002053657474696E677329004D353030008B
:1009F000526563656976696E67204672616D652030
:100A00002846656564726174652053657474696E07
:100A1000677329004D35303000526563656976692A
:100A20006E67204672616D6520285374657073206F
:100A300053657474696E677329004D353030005208
:100A40006563656976696E67204672616D65202809
:100A50005049442053657474696E67732900526568
:100A600063656976696E67204672616D65202850FE
:100A700072696E742053657474696E6773290049D6
:100A80006E76616C6964206B65792076616C756542
:100A9000200047393000473120452D312046313282
:100AA0003000473931004739300047312045312087
:100AB0004631323000473931004739300047312064
:100AC0005A2D302E35204633303030004739310032
:100AD000473930004731205A302E352046333030E8
:100AE00030004739310047393000473120592D3522
:100AF0002046333030300047393100473930004725
:100B000031205935204633303030004739310047E5
:100B1000393000473120582D3520463330303000F1
:100B200047393100473930004731205835204633A6
:100B30003030300047393100496E76616C6964208D
:100B40006B65792076616C756520004D38340047FF
:100B5000323800473238205A300047323820593076
:100B600000473238205830004D31313700436F6F25
:100B70006C646F776E004D3134302053004D31304E
:100B8000342053004D353030005265636569766915
:100B90006E67204672616D652028507265736574BA
:100BA000732900496E76616C6964207072657365A3
:100BB000742023200050726568656174205374614D
:100BC00072740050726568656174207061676500B9
:100BD000496E76616C6964206B65792076616C750D
:100BE000652000473930004C6F61642F556E6C6F83
:100BF00061642053746F7000496E76616C69642083
:100C00006B65792076616C75652000526573756D32
:100C100065207072696E74696E6700526573756DD8
:100C200065205072696E7400506175736520707232
:100C3000696E74696E6700506175736520507269E2
:100C40006E740053746F70205072696E7400496E38
:100C500076616C6964206B65792076616C756520BE
:100C600000526573756D65207072696E74696E6788
:100C700000526573756D65205072696E7400506125
:100C8000757365207072696E74696E672E2E2E0002
:100C90005061757365205072696E740053746F7083
:100CA000205072696E7400496E76616C6964206BC5
:100CB00065792076616C75652000496E76616C6996
:100CC0006420616374696F6E20003E3E3E20002008
:100CD000776F7264732C20416374696F6E203D20BE
:100CE000002C204B657956616C7565203D200072A3
:100CF000656164696E6720696E636F6D696E6720F8
:100D00004672616D6500696E206D6F76655F746F08
:100D1000282920666565645F76616C756520666F5D
:100D2000722058593A002C2065793D0029202D3E2B
:100D3000202865783D002C2073793D0020436F6E9C
:100D40006E656374696E6720776974682076657272
:100D5000746963616C206C696E65202873783D004E
:100D60002C2065793D0029202D3E202865783D0006
:100D70002C2073793D0020436F6E6E656374696E3D
:100D800067207769746820686F72697A6F6E746122
:100D90006C206C696E65202873783D004C65617627
:100DA000696E6720473236002C2079693D0020208B
:100DB00020446F696E6720636972636C652061749B
:100DC0003A202878693D003F53706563696669651C
:100DD0006420582C5920636F6F7264696E6174656A
:100DE000206F7574206F6620626F756E64732E0AB3
:100DF000003F28522965706561742076616C7565C5
:100E0000206E6F7420706C61757369626C653B2035
:100E10006D757374206265206174206C65617374F4
:100E200020312E0A003F2852296570656174206DBB
:100E300075737420626520737065636966696564A3
:100E4000207768656E206E6F74207573696E6720F9
:100E5000616E204C43442E0A003F537065636966FF
:100E6000696564206E6F7A7A6C652074656D706553
:100E7000726174757265206E6F7420706C61757329
:100E800069626C652E0A003F537065636966696527
:100E9000642066696C616D656E742073697A652083
:100EA0006E6F7420706C61757369626C652E0A00D8
:100EB0003F537065636966696564207072696D652A
:100EC000206C656E677468206E6F7420706C61753D
:100ED0007369626C652E0A003F5072696D65206C03
:100EE000656E677468206D75737420626520737019
:100EF00065636966696564207768656E206E6F74E6
:100F0000207573696E6720616E204C43442E0A0081
:100F10003F537065636966696564206E6F7A7A6CA9
:100F2000652073697A65206E6F7420706C617573CB
:100F300069626C652E0A003F537065636966696576
:100F4000642052657472616374696F6E204D756CB4
:100F50007469706C696572206E6F7420706C617555
:100F60007369626C652E0A003F5265747261637426
:100F7000696F6E204D756C7469706C696572206D57
:100F80007573742062652073706563696669656452
:100F90002E0A003F537065636966696564206C6161
:100FA00079657220686569676874206E6F74207057
:100FB0006C61757369626C652E0A003F53706563DE
:100FC0006966696564206265642074656D70657228
:100FD0006174757265206E6F7420706C61757369D1
:100FE000626C652E0A0047323620636F6D6D616E4C
:100FF0006420737461727465642E2057616974692A
:101000006E6720666F722068656174657228732947
:101010002E0A002569730025696D20256973002556
:1010200069682025696D202569730025696420257C
:1010300069682025696D2025697300256979202557
:101040006964202569682025696D20256973004C35
:10105000696E65204E756D626572206973206E6FD2
:1010600074204C617374204C696E65204E756D62FE
:1010700065722B312C204C617374204C696E653A7B
:1010800020004B494C4C45442E200053544F5050A7
:1010900045442E20005072696E7465722073746F1F
:1010A000707065642064756520746F206572726F5E
:1010B00072732E2046697820746865206572726F9D
:1010C0007220616E6420757365204D393939207442
:1010D0006F20726573746172742E202854656D7070
:1010E00065726174757265206973207265736574C9
:1010F0002E205365742069742061667465722072B5
:10110000657374617274696E67290A004E6F2043BB
:101110006865636B73756D2077697468206C696EA0
:1011200065206E756D6265722C204C617374204C65
:10113000696E653A2000636865636B73756D206D39
:1011400069736D617463682C204C617374204C6901
:101150006E653A20004D313130004D33310053443B
:101160002072656164206572726F720A00446F6E4E
:1011700065207072696E74696E672066696C650AB5
:10118000007C3C3E5E2B3D3F2F5B5D3B2C2A225C6E
:101190000044617461207472756E636174656400EB
:1011A00044617461207472756E63617465640024B7
:1011B000F4D43050C38E20C2A24017828B7011121B
:1011C0007A910D816CD90AA861E108C75866076158
:1011D0005143061E4B5D05C145A7041A4111040980
:1011E0003D9803713931034036DB0265339102D4F7
:1011F000305402802E1D02632CEE01752AC501B009
:1012000028A001102781018F2564012B244B01E0C8
:10121000223401AC211F018D200D01801FFC0084B0
:101220001EED00971DDF00B81CD200E61BC6002093
:101230001BBC00641AB200B219A8000A19A0006A07
:10124000189900D117910040178B00B51684003112
:10125000167E00B31579003A157300C7146F005855
:10126000146A00EE1366008813630025135E00C73E
:10127000125B006C12570015125400C1115100701E
:10128000114F0021114B00D61049008D1047004628
:1012900010440002104200C00F4000800F3E004288
:1012A0000F3C00060F3B00CB0E3800930E37005C5E
:1012B0000E3500270E3400F30D3200C10D310090C1
:1012C0000D3000600D2E00320D2D00050D2C00D9C3
:1012D0000C2B00AE0C2900850C29005C0C27003576
:1012E0000C27000E0C2600E80B2400C40B2400A0E1
:1012F0000B23007D0B23005A0B2100390B21001812
:101300000B2000F80A1F00D90A1E00BB0A1E009D10
:101310000A1D00800A1D00630A1C00470A1B002CDE
:101320000A1B00110A1A00F7091A00DD091900C486
:10133000091900AB091900920917007B091800630D
:101340000917004C09160036091600200916000A74
:10135000091500F5081500E0081400CC081400B8C1
:10136000081400A4081400900813007D0812006BF4
:101370000813005808120046081200340811002310
:101380000811001208110001081100F0071000E018
:10139000071000D0071000C0071000B0070F00A111
:1013A00007100091070E0083070F0074070F0065F8
:1013B000070E0057070E0049070E003B070D002ED1
:1013C000070E0020070D0013070D0006070D00F99A
:1013D000060C00ED060D00E0060C00D4060C00C85B
:1013E000060C00BC060C00B0060C00A4060B00990D
:1013F000060C008D060B0082060B0077060B006CB6
:10140000060B0061060A0057060B004C060A004254
:10141000060A0038060A002E060A0024060A001AE8
:10142000060A001006090007060A00FD050900F477
:10143000050900EB050900E2050900D9050900D0FE
:10144000050900C7050900BE050900B5050800AD7E
:10145000050800A50509009C050800940508008CF6
:10146000050800840508007C050800740508006C68
:10147000050700650508005D050700560508004ED4
:10148000050700470507004005080038050700313B
:101490000507002A050700230507001C050600169E
:1014A0000507000F0507000805060002050700FBF9
:1014B000040600F5040700EE040600E8040600E256
:1014C000040700DB040600D5040600CF040600C9AB
:1014D000040600C3040600BD040600B7040600B1FC
:1014E000040500AC040600A6040600A00405009B49
:1014F00004060095040500900406008A0405008592
:10150000040500800406007A0405007504050070D7
:101510000405006B04050066040500610405005C19
:1015200004050057040500520405004D0405004859
:10153000040500430405003E0404003A0405003598
:10154000040500300404002C0405002704040023D3
:101550000405001E0404001A04040016040500110A
:101560000404000D04040009040500040404000040
:10157000040400FC030400F8030400F4030400F076
:10158000030400EC030400E8030400E4030400E0A7
:10159000030400DC030400D8030400D4030400D0D7
:1015A000030400CC030400C8030300C503030024A4
:1015B000F404D9201BC40C5C0E9804C4095F0265B6
:1015C000077101F405F900FB04B30048048700C16A
:1015D0000369005803550003034500BE023A008426
:1015E00002310053022A002902250004022000E4EF
:1015F000011C00C8011900AF0117009801140084F4
:10160000011300710110006101100051010E00432F
:10161000010D0036010B002B010B0020010B001502
:101620000109000C01090003010800FB000800F398
:10163000000800EB000700E4000600DE000600D80A
:10164000000600D2000600CC000500C7000500C25D
:10165000000500BD000400B9000400B5000400B19D
:10166000000400AD000400A9000400A5000300A2CE
:101670000003009F0004009B0003009800030095F6
:1016800000020093000300900003008D0002008B15
:10169000000300880002008600020084000300812D
:1016A0000002007F0002007D0002007B0002007942
:1016B0000002007700010076000200740002007250
:1016C000000100710002006F0002006D0001006C5B
:1016D0000002006A00010069000200670001006664
:1016E0000001006500010064000200620001006169
:1016F000000100600001005F0002005D0001005C6D
:101700000001005B0001005A00010059000100586F
:10171000000100570001005600010055000100546F
:10172000000100530000005300010052000100516D
:10173000000100500001004F0001004E0000004E6B
:101740000001004D0001004C0001004B0000004B67
:101750000001004A00010049000100480000004863
:10176000000100470001004600000046000100455E
:101770000000004500010044000100430000004358
:101780000001004200000042000100410000004151
:10179000000100400001003F0000003F0001003E4A
:1017A0000000003E0001003D0000003D0001003C43
:1017B0000000003C0000003C0001003B0000003B3A
:1017C0000001003A0000003A000100390000003931
:1017D0000001003800000038000000380001003728
:1017E000000000370001003600000036000000361F
:1017F0000001003500000035000000350001003414
:101800000000003400000034000100330000003309
:1018100000000033000100320000003200000032FE
:1018200000010031000000310000003100010030F3
:1018300000000030000000300001002F0000002FE9
:101840000000002F0000002F0001002E0000002EDD
:101850000000002E0001002D0000002D0000002DD2
:101860000000002D0001002C0000002C0000002CC6
:101870000000002C0001002B0000002B0000002BBA
:101880000000002B0001002A0000002A0000002AAE
:101890000000002A000100290000002900000029A2
:1018A0000000002900000029000100280000002895
:1018B0000000002800000028000000280001002788
:1018C000000000270000002700000027000000277C
:1018D000000100260000002600000026000000266F
:1018E0000000002600010025000000250000002562
:1018F0000000002500000025000000250001002454
:101900000000002400000024000000240000002447
:10191000000100230000002300000023000000233A
:10192000000000230000002300000023000100222B
:10193000000000220000002200000022000000221F
:101940000000002200010021000000210000002111
:101950000000002100000021000000210000002103
:1019600000010020000000200000002000000020F6
:1019700000000020000000200000002000000020E7
:101980000001001F0000001F0000001F0000001FDA
:101990000000001F0000001F0000001F0001001ECB
:1019A0000000001E0000001E0000001E0000004D90
:1019B000383420582059205A2045006265640A00B6
:1019C0002C2073797374656D2073746F7070656407
:1019D00021204865617465725F49443A200048657A
:1019E0006174696E67206661696C65640048656151
:1019F00074696E67206661696C656400486561742E
:101A0000696E67206661696C656400486561746928
:101A10006E67206661696C656400544845524D41AB
:101A20004C2052554E4157415900546865726D61C2
:101A30006C2052756E61776179004B494C4C45447E
:101A40002E2000202D20496E76616C696420657817
:101A5000747275646572206E756D62657220210AFC
:101A6000002020506C616E6E65724275666665720C
:101A700042797465733A20002046726565204D6591
:101A80006D6F72793A2000436F6D70696C65643ACE
:101A90002046656220313120323031380A00207C06
:101AA00020417574686F723A20284B6F6C64290A64
:101AB00000323031382D30322D30392031323A3049
:101AC0003000204C61737420557064617465643A11
:101AD0002000312E312E380A004D61726C696E0083
:101AE00020536F6674776172652052657365740A5E
:101AF00000205761746368646F6720526573657472
:101B00000A002042726F776E206F757420526573E1
:101B100065740A002045787465726E616C205265A8
:101B20007365740A00506F77657255700A0073749C
:101B30006172740A006572726F72207772697469DB
:101B40006E6720746F2066696C650A0020503A0049
:101B5000205A3A0020593A0020583A00656E6473C2
:101B6000746F7073206869743A2000446F6E65204A
:101B7000736176696E672066696C652E0A004D3266
:101B80003900202863616C63756C61746564292178
:101B90000A0020213D2000454550524F4D20435220
:101BA00043206D69736D61746368202D2028737400
:101BB0006F726564292000290A00206279746573B8
:101BC0003B2063726320002073746F72656420731E
:101BD000657474696E677320726574726965766581
:101BE00064202800204D61726C696E3D563437299F
:101BF0000A0028454550524F4D3D00454550524F33
:101C00004D2076657273696F6E206D69736D6174B6
:101C10006368200048617264636F64656420446592
:101C20006661756C742053657474696E6773204CBB
:101C30006F616465640A00E8030000E80300006463
:101C4000000000E80300000000E1430000E1430061
:101C500000A0400000C8410000A2420000A24200D3
:101C600040C8439A99BC4220204D383531205A0053
:101C70005A2D50726F6265204F6666736574202816
:101C80006D6D293A0A0020440020490020204D3380
:101C900030312050005049442073657474696E6778
:101CA000733A0A00205A0020204D3432302053006D
:101CB0004175746F20426564204C6576656C696E71
:101CC000673A0A00205A0020590020204D32303651
:101CD000205800486F6D65206F66667365743A0A18
:101CE00000204500205A00205900205800204200C2
:101CF00020540020204D323035205300416476615D
:101D00006E6365643A20533C6D696E5F6665656419
:101D1000726174653E20543C6D696E5F74726176C9
:101D2000656C5F66656564726174653E20423C6DFA
:101D3000696E5F7365676D656E745F74696D655F0D
:101D400075733E20583C6D61785F78795F6A657283
:101D50006B3E205A3C6D61785F7A5F6A65726B3EBC
:101D600020453C6D61785F655F6A65726B3E0A0075
:101D700020540020520020204D32303420500041A9
:101D80006363656C65726174696F6E2028756E6936
:101D900074732F7332293A20503C7072696E745FED
:101DA000616363656C3E20523C726574726163745A
:101DB0005F616363656C3E20543C74726176656C50
:101DC0005F616363656C3E0A00204500205A002075
:101DD000590020204D3230312058004D6178696D16
:101DE000756D20416363656C65726174696F6E2007
:101DF00028756E6974732F7332293A0A00204500E2
:101E0000205A0020590020204D3230332058004DF8
:101E10006178696D756D206665656472617465735E
:101E20002028756E6974732F73293A0A00204500C3
:101E3000205A0020590020204D3932205800537478
:101E40006570732070657220756E69743A0A00209F
:101E5000204D3230302044300A0020204D323030C6
:101E60002044002044697361626C65640A0046691D
:101E70006C616D656E742073657474696E67733A16
:101E8000002020473231202020203B20556E6974ED
:101E90007320696E206D6D0A0020746F6F206C6F67
:101EA0006E6720657874727573696F6E20707265E5
:101EB00076656E7465640A0020636F6C64206578D3
:101EC00074727573696F6E2070726576656E746575
:101ED000640A00496E76616C6964206261636B67B5
:101EE000726F756E64207461736B200047312045FA
:101EF00031204631303000473932204530004738F4
:101F0000320046696C616D656E7420657874727517
:101F10006465642000473120452D31204631323040
:101F200000556E6C6F61642046696C616D656E74FE
:101F30000047312045312046313230004C6F61641A
:101F40002046696C616D656E74004C6576656C69E0
:101F50006E6720486F6D65642C2073746172742005
:101F600070726F6365737300627573793A20706184
:101F70007573656420666F7220696E7075740A00EF
:101F8000627573793A2070617573656420666F724B
:101F900020757365720A00627573793A2070726FEA
:101FA00063657373696E670A004B494C4C45442E58
:101FB00020004B494C4C2063617573656420627945
:101FC00020746F6F206D75636820696E616374693A
:101FD00076652074696D65202D2063757272656E5B
:101FE0007420636F6D6D616E643A20005072696E8B
:101FF0007465722068616C7465642E206B696C6C0A
:1020000028292063616C6C6564210A0000000000CF
:1020100000000000000000000000484200004842AC
:1020200000008040000000005761726E696E673AE0
:1020300020486F6D696E672042756D702044697627
:1020400069736F72203C20310A000202040000A074
:10205000400000A04000000040000048430000484D
:102060004300003443FFFFFF20643A0020693A0038
:1020700020703A00536C6565702E2E2E0020706F14
:10208000736974696F6E206F7574206F662072615A
:102090006E67652E0A003F50726F6265200020282F
:1020A00044525952554E2900473239204175746FB8
:1020B00020426564204C6576656C696E6700284235
:1020C0002961636B00284629726F6E7400285229BB
:1020D0006967687400284C29656674003F28562992
:1020E0006572626F7365206C6576656C206973201C
:1020F000696D706C61757369626C652028302D3470
:10210000292E0A00426164205A2076616C75650AA6
:10211000004E6F2062696C696E656172206772693A
:10212000640A005374616E64617264204465766968
:102130006174696F6E3A20002052616E67653A20C3
:1021400000204D61783A2000204D696E3A20004D04
:1021500065616E3A200046696E6973686564210A9C
:10216000002072616E67653A2000206D61783A2028
:1021700000206D696E3A2000207369676D613A2016
:1021800000206D65616E3A20003A207A3A200020E6
:102190006F662000205A00205900205800476F69C0
:1021A0006E6720746F3A00436C6F636B7769736579
:1021B0000A00436F756E7465722D00204469726564
:1021C0006374696F6E3A2000202020616E676C6531
:1021D0003A20005374617274696E67207261646999
:1021E00075733A2000506F736974696F6E696E671A
:1021F000207468652070726F62652E2E2E0A003F73
:102200004E756D626572206F66206C65677320691C
:102210006E206D6F76656D656E74206E6F742070C4
:102220006C61757369626C652028302D3135292EFB
:102230000A00590058003F53616D706C6520736946
:102240007A65206E6F7420706C61757369626C655D
:102250002028342D3530292E0A004D3438205A2DAF
:1022600050726F6265205265706561746162696C5D
:1022700069747920546573740A003F285629657281
:10228000626F7365206C6576656C20697320696D7B
:10229000706C61757369626C652028302D34292E4D
:1022A0000A0043616E6E6F74206F70656E207375E7
:1022B0006264697220005354415455533A200065BA
:1022C0006E7175657565696E672022006563686F5C
:1022D0003A0053686F77207061676520005265612E
:1022E00064696E6720506963747572654944004380
:1022F000757272656E74207061676520696E6465C1
:1023000078203D20003E3E3E2000206279746573B7
:102310002C20636D64203D20003C3C3C200020626A
:10232000797465732E00496E76616C696420616D05
:102330006F756E74206F66206279746573207265A4
:10234000636569766564004461746120746F20621E
:102350006520726563656976656420697320746FB2
:102360006F2062696720666F72207468652046720C
:10237000616D652062756666657220736F20736B90
:10238000697020697400496E76616C6964206865C3
:1023900061646572207768656E2072656365697631
:1023A000696E672061204672616D65005472792004
:1023B000746F2072656164206120627974652061A8
:1023C000667465722074686520656E64206F66208F
:1023D000646174610054727920746F207265616465
:1023E000206120776F726420616674657220746862
:1023F0006520656E64206F662064617461004461CD
:102400007461206C656E67746820696E20726573F4
:10241000706F6E73652028002920646F6573206ECD
:102420006F7420636F72726573706F6E6420746F67
:1024300020726571756573742028002900526567E4
:10244000697374657220696E20726573706F6E7344
:10245000652028002920646F6573206E6F742063E7
:102460006F72726573706F6E6420746F2072657125
:10247000756573742028002900436F6D6D616E646B
:1024800020696E20726573706F6E73652028002955
:1024900020646F6573206E6F7420636F7272657352
:1024A000706F6E6420746F2072657175657374202F
:1024B0002800290044617461206C656E677468208F
:1024C000696E20726573706F6E73652028005265A7
:1024D00067697374657220696E20726573706F6EC0
:1024E00073652028002900436F6D6D616E6420695B
:1024F0006E20726573706F6E7365202800292064EA
:102500006F6573206E6F7420636F72726573706F86
:102510006E6420746F207265717565737420280075
:1025200029004572726F722077726974696E672034
:10253000746F20454550524F4D210A00290A002052
:1025400062797465733B2063726320005365747411
:10255000696E67732053746F726564202800700180
:102560002C0190012701B0012201C0011D01F001E1
:1025700018011002130130020E01600209019002DD
:102580000401C002FF000003FA004003F5008003CD
:10259000F000D003EB002004E6007004E100E0044A
:1025A000DC004005D700C005D2004006CD00D006B3
:1025B000C8008007C3003008BE00F008B900C00999
:1025C000B400B00AAF00B00BAA00D00CA500000EFA
:1025D000A000500F9B00C0109600501291000014F4
:1025E0008C00C0158700B0178200B0197D00D01B89
:1025F0007800001E730040206E0090226900F024D5
:10260000640040275F0090295A00E02B5500102EEF
:10261000500020304B0010324600E033410090352E
:102620003C001037370070383200A0392D00B03A26
:102630002800A03B2300603C1E00103D1900903D87
:102640001400103E0F00703E0A00C03E0500003F1F
:102650000000403FFBFF803FF6FFC03FF1FF4572A7
:10266000723A204D494E54454D5020424544004554
:1026700072723A204D494E54454D50004D494E54CA
:10268000454D5020747269676765726564004572D4
:10269000723A204D415854454D5020424544004522
:1026A00072723A204D415854454D50004D41585496
:1026B000454D502074726967676572656400202F0C
:1026C000002042403A0020403A000000210024004F
:1026D00027002A002D003000330001010000040112
:1026E00007010A0100002200250028002B002E000F
:1026F0003100340002010000050108010B01000057
:1027000020002300260029002C002F0032000001A9
:102710000000030106010901050505050705080874
:102720000808020202020A0A08080404040401015B
:102730000101010101010303030303030303040770
:1027400007070C0C0C0C0C0C0C0C02020202060607
:102750000606060606060B0B0B0B0B0B0B0B0102FA
:1027600010202008081020401020408002010201A3
:10277000080402010102040810204080804020105B
:1027800008040201800402018040201008040201B4
:10279000080402010102040810204080010204081C
:1027A0001020408000000A0B02090C0D0E080703E0
:1027B0000401000000000000000000000000000014
:1027C0000000000000000000000000000000000009
:1027D00012111000000000000000000000000000C6
:1027E0000000000000000000000053544154555305
:1027F0002050474D3A200053442063617264206F9B
:102800006B0A006F70656E526F6F74206661696C41
:1028100065640A00766F6C756D652E696E6974204B
:102820006661696C65640A00534420696E697420AE
:102830006661696C0A004D3234004D3233202573D5
:10284000006175746F25692E670057726974696E2F
:102850006720746F2066696C653A20006F70656E42
:10286000206661696C65642C2046696C653A2000BD
:102870006F70656E206661696C65642C2046696CBA
:10288000653A200046696C652073656C6563746504
:10289000640A002053697A653A200046696C652015
:1028A0006F70656E65643A20006F70656E206661BA
:1028B000696C65642C2046696C653A200020666965
:1028C0006C653A2000646F696E67006672657368B4
:1028D000004E6F772000454E4420535542524F55CD
:1028E00054494E450A002220706F73002220706107
:1028F00072656E743A2200535542524F5554494EF8
:10290000452043414C4C207461726765743A220043
:102910004B494C4C45442E2000747279696E6720F7
:10292000746F2063616C6C207375622D67636F64D4
:10293000652066696C6573207769746820746F6FB1
:10294000206D616E79206C6576656C732E204D412B
:1029500058206C6576656C2069733A004572726F19
:10296000723A00434F4D4D554E49434154494F4EE5
:102970000044525952554E004552524F525300494D
:102980004E464F004543484F0042656420646F6ED9
:10299000652E0020573A00426564204865617469DD
:1029A0006E672E0084297F297829712963296F6633
:1029B000660044454255473A00205A3A0020593AA9
:1029C0000020436F756E7420583A0020453A00206D
:1029D0005A3A0020593A00583A004361703A00458B
:1029E0004D455247454E43595F5041525345520061
:1029F000434153455F4C494748545F425249474819
:102A0000544E45535300544F47474C455F4C49473C
:102A100048545300534F4654574152455F504F5707
:102A20004552004255494C445F50455243454E542F
:102A3000004C4556454C494E475F44415441005A6D
:102A40005F50524F4245004155544F4C4556454CFE
:102A5000005052494E545F4A4F420050524F475225
:102A6000455353004155544F5245504F52545F54B3
:102A7000454D5000564F4C554D4554524943004525
:102A80004550524F4D0053455249414C5F584F4EAF
:102A90005F584F4646004649524D574152455F4E9A
:102AA000414D453A4D61726C696E20312E312E38A0
:102AB000202841445669332B2B41424C20322E3181
:102AC0002E302920534F555243455F434F44455FB5
:102AD00055524C3A68747470733A2F2F6769746852
:102AE00075622E636F6D2F784B6F6C64782F414445
:102AF00056693370702D4D61726C696E2050524F63
:102B0000544F434F4C5F56455253494F4E3A312E26
:102B100030204D414348494E455F545950453A573E
:102B200061686E616F204475706C696361746F7267
:102B300020693320506C75732045585452554445D4
:102B4000525F434F554E543A3120555549443A341B
:102B5000346232663564362D653765342D3437621C
:102B6000662D626538312D633261366234666337B3
:102B70003937350A002F2F20004D65736820706F9C
:102B8000696E742063616E6E6F7420626520726579
:102B9000736F6C7665640A004D34323120696E6360
:102BA0006F727265637420706172616D65746572B5
:102BB0002075736167650A00526563656976696EA1
:102BC00067204672616D65202854617267657420C4
:102BD00054656D706572617475726529004E6F2061
:102BE0004261636B207061676520646566696E652C
:102BF00064004C4344204669726D776172652072AF
:102C000061772076657273696F6E203D2000556E86
:102C10006B6E6F776E00526563656976696E6720CB
:102C20004672616D65202856657273696F6E290062
:102C300050726F62696E67206661696C65640A0034
:102C400050726F62696E67206661696C656400200E
:102C50005A3A200020593A200042656420583A2010
:102C60000053544154555320563A2000206669724F
:102C700073740A005A0059005800486F6D652000AF
:102C800020496E76616C696420657874727564653C
:102C900072200000000000000000000000000000A2
:102CA000004843000048430000344342696C696EA9
:102CB000656172204C6576656C696E672047726944
:102CC000643A0A00537562646976696465642077C2
:102CD000697468204341544D554C4C20524F4D204F
:102CE0004C6576656C696E6720477269643A0A00C4
:102CF000526573656E643A20006F6B0020746F6FCD
:102D0000206C6F6E6720657874727573696F6E20C2
:102D100070726576656E7465640A0020636F6C641A
:102D200020657874727573696F6E20707265766550
:102D30006E7465640A004D31313720004739310027
:102D40004E6F20466F7277617264207061676520F4
:102D5000646566696E65640041646A7573743A20DF
:102D60006F6C64203D20002C20657870656374656D
:102D700064203D20002C206D6561737572656420B0
:102D80003D20002C206E6577203D2000AFEE82EEC6
:102D900011241FBECFEFD1E2DEBFCDBF00E00CBFDC
:102DA00013E0A0E0B2E0E8E9F8E002E00BBF02C007
:102DB00007900D92AC39B107D9F729E1ACE9B3E03E
:102DC00001C01D92AE33B207E1F716E1C7ECD6E1C0
:102DD00000E006C021970109802FFE010F94C80270
:102DE000C63CD10780E00807A9F70E94F9E80D94D6
:102DF0003B040C9400002F923F924F925F926F928F
:102E00007F928F929F92AF92BF92CF92DF92EF927A
:102E1000FF920F931F93CF93DF93CDB7DEB7C859BF
:102E2000D1090FB6F894DEBF0FBECDBF81E090E0B0
:102E30009093830C8093820C8091F0148D3411F464
:102E40000C947C1F843511F40C94DC30873411F021
:102E50000C9428318091EE149091EF148C319105EF
:102E600009F405C6D4F4843091055CF482309105F0
:102E70009CF597FF02C00C9447310E94C2A50C94A8
:102E800047318430910509F4EEC54A9711F00C944E
:102E900047310E94E5510C9447318A32910509F47B
:102EA0004DC74CF48D31910509F454C64E9709F481
:102EB00055C60C9447318B35910509F4BFC68C3546
:102EC000910509F4C0C68A35910511F00C9447317B
:102ED0001092A1030C94473120910C02222311F48B
:102EE0000C94473111E0029709F010E00E94F7D4EA
:102EF00082E50E948650882309F45CC10E94245018
:102F00006B017C014090F10C5090F20C6090F30C3E
:102F10007090F40C2091F50C3091F60C4091F70C68
:102F20005091F80C23962CAF3DAF4EAF5FAF239777
:102F30008091461490914714A0914814B09149147F
:102F400027968CAF9DAFAEAFBFAF279720914A14A5
:102F500030914B1440914C1450914D1463962CAF0A
:102F60003DAF4EAF5FAF639720E030E0A901C701EE
:102F7000B6010E945FFB882309F455C5A3019201A5
:102F800027966CAD7DAD8EAD9FAD27970E945FFB00
:102F9000811111C023962CAD3DAD4EAD5FAD239791
:102FA00063966CAD7DAD8EAD9FAD63970E945FFB68
:102FB000882309F438C520E030E0A901C701B60133
:102FC0000E945FFB881F8827881F18130BC080E0B2
:102FD00090E0A0E8BFE36B968CAF9DAFAEAFBFAF04
:102FE0006B970AC020E030E040E85FEB6B962CAFB7
:102FF0003DAF4EAF5FAF6B97A301920127966CADCB
:103000007DAD8EAD9FAD27970E94D8FF2F966CAFF8
:103010007DAF8EAF9FAF2F9723962CAD3DAD4EADBC
:103020005FAD239763966CAD7DAD8EAD9FAD63971D
:103030000E94D8FF67966CAF7DAF8EAF9FAF67974A
:103040002F962CAD3DAD4EAD5FAD2F97CA01B901A6
:103050000E94C4FB4B015C0167962CAD3DAD4EADAB
:103060005FAD6797CA01B9010E94C4FB9B01AC0127
:10307000C501B4010E94D9FF0F9444022B966CAF96
:103080007DAF8EAF9FAF2B9720E030E040E05FE355
:103090000E94C4FB4B015C01A7019601C701B60168
:1030A0000E94C4FB6B017C01A5019401C501B40120
:1030B0000E94C4FB9B01AC01C701B6010E94D8FF6E
:1030C0000F9444029B01AC016B966CAD7DAD8EAD4F
:1030D0009FAD6B970E94C4FB4B015C0127962CAD02
:1030E0003DAD4EAD5FAD2797C301B2010E94D9FF40
:1030F00020E030E040E05FE30E94C4FB6B017C0114
:1031000067966CAD7DAD8EAD9FAD679790582B9651
:103110002CAD3DAD4EAD5FAD2B970F94B5009B012F
:10312000AC01C501B4010E94C4FB9B01AC01C70105
:10313000B6010E94D9FFA30192010E94D8FF6B0142
:103140007C0163962CAD3DAD4EAD5FAD639723968C
:103150006CAD7DAD8EAD9FAD23970E94D9FF20E071
:1031600030E040E05FE30E94C4FB2B013C012B9662
:103170002CAD3DAD4EAD5FAD2B972F966CAD7DADBB
:103180008EAD9FAD2F970F94B5009B01AC01C5018B
:10319000B4010E94C4FB9B01AC01C301B2010E94B7
:1031A000D9FF23962CAD3DAD4EAD5FAD23970E9468
:1031B000D8FF14C089E40E948650882329F00E9419
:1031C00024506B017C0103C0C12CD12C76018AE410
:1031D0000E9486508823F9F00E94245063966CAFB9
:1031E0007DAF8EAF9FAF639720E030E0A901C701AC
:1031F000B6010E945FFB81111EC020E030E0A901F2
:1032000063966CAD7DAD8EAD9FAD63970E945FFB05
:10321000811111C008C420E030E0A901C701B60146
:103220000E945FFB882309F4FEC363961CAE1DAEAB
:103230001EAE1FAE6397D701C601B05823968CAF60
:103240009DAFAEAFBFAF239763962CAD3DAD4EADF6
:103250005FAD6397505827962CAF3DAF4EAF5FAF31
:1032600027979C01AD01BC01CD010E94C4FB4B011D
:103270005C0127962CAD3DAD4EAD5FAD2797CA01E1
:10328000B9010E94C4FB9B01AC01C501B4010E94BD
:10329000D9FF0F944402AB966CAF7DAF8EAF9FAF5A
:1032A000AB978091F10C9091F20CA091F30CB0913E
:1032B000F40C2B968CAF9DAFAEAFBFAF2B97A70191
:1032C0009601BC01CD010E94D9FF6B966CAF7DAF1A
:1032D0008EAF9FAF6B972091F50C3091F60C40911B
:1032E000F70C5091F80C67962CAF3DAF4EAF5FAF27
:1032F000679763962CAD3DAD4EAD5FAD6397679616
:103300006CAD7DAD8EAD9FAD67970E94D9FF6F9676
:103310006CAF7DAF8EAF9FAF6F9780914614909149
:103320004714A0914814B0914914A3968CAF9DAF57
:10333000AEAFBFAFA3976B962CAD3DAD4EAD5FADBD
:103340006B97BC01CD010E94D8FF6B017C012091DD
:103350004A1430914B1440914C1450914D14A7963F
:103360002CAF3DAF4EAF5FAFA7976F962CAD3DAD85
:103370004EAD5FAD6F97A7966CAD7DAD8EAD9FAD39
:10338000A7970E94D8FF4B015C018091F90C9091A6
:10339000FA0CA091FB0CB091FC0CE3968CAF9DAFA6
:1033A000AEAFBFAFE3979C01AD0160914E14709139
:1033B0004F1480915014909151140E94D8FF2F9671
:1033C0006CAF7DAF8EAF9FAF2F972091521430918D
:1033D00053144091541450915514AF962CAF3DAFF7
:1033E0004EAF5FAFAF978091FD0C9091FE0CA09116
:1033F000FF0CB091000DE7968CAF9DAFAEAFBFAFA5
:10340000E797A701960123966CAD7DAD8EAD9FAD7C
:1034100023970E94C4FB2B013C01A5019401279630
:103420006CAD7DAD8EAD9FAD27970E94C4FB9B0117
:10343000AC01C301B2010E94D9FF2B013C01A501DF
:10344000940123966CAD7DAD8EAD9FAD23970E9408
:10345000C4FB4B015C01A701960127966CAD7DADC5
:103460008EAD9FAD27970E94C4FB9B01AC01C501A7
:10347000B4010E94D8FFA30192010F944C006B018C
:103480007C0120E030E0A9010E945FFB87FF0AC0B9
:103490002BED3FE049EC50E4C701B6010E94D9FF93
:1034A0006B017C01112351F02BED3FE049EC50E41E
:1034B000C701B6010E94D8FF6B017C0120E030E01B
:1034C000A901C701B6010E945FFB811128C0A39624
:1034D0002CAD3DAD4EAD5FADA3972B966CAD7DADE4
:1034E0008EAD9FAD2B970E945FFB811118C0A796F0
:1034F0002CAD3DAD4EAD5FADA79767966CAD7DAD84
:103500008EAD9FAD67970E945FFB811108C09BED58
:10351000C92E9FE0D92E99ECE92E90E4F92EAB96B6
:103520002CAD3DAD4EAD5FADAB97C701B6010E946E
:10353000C4FB9B01AC010E94C4FB4B015C012F96B4
:103540002CAD3DAD4EAD5FAD2F97CA01B9010E94C4
:10355000C4FB9B01AC01C501B4010E94D9FF0F94CB
:1035600044024B015C012FE632E143E85AE30E943A
:103570005FFB87FD54C2C501B4010F944E010F9447
:1035800022011B01672B19F422242394312CB10151
:1035900080E090E00E9463FB4B015C019B01AC0169
:1035A000C701B6010F94B5002B966CAF7DAF8EAFFF
:1035B0009FAF2B97A50194012F966CAD7DAD8EAD7D
:1035C0009FAD2F970F94B500AB966CAF7DAF8EAFCC
:1035D0009FAFAB97E7962CAD3DAD4EAD5FADE79796
:1035E000AF966CAD7DAD8EAD9FADAF970E94D8FF0D
:1035F000A50194010F94B500AF966CAF7DAF8EAF6F
:103600009FAFAF972B962CAD3DAD4EAD5FAD2B97D9
:10361000CA01B9010E94C4FB20E030E040E05FE352
:103620000E94C4FB9B01AC0160E070E080E89FE376
:103630000E94D8FFA3966CAF7DAF8EAF9FAFA397CC
:10364000E3962CAD3DAD4EAD5FADE39729873A874C
:103650004B875C87E7968CAD9DADAEADBFADE79770
:103660008D879E87AF87B88B6091010270910202AF
:10367000072E000C880B990B0E9465FB20913C02E1
:1036800030913D0240913E0250913F020E94C4FBA6
:103690002AE037ED43E25CE30E94C4FB6BAF7CAFF2
:1036A0008DAF9EAF0E94E2B79B01AC0128533F4F04
:1036B0004F4F5F4FA7962CAF3DAF4EAF5FAFA79771
:1036C0004FAC21965FAC219722966FAC2297239640
:1036D0007FAC239741E050E065965FAF4EAF6597B2
:1036E00059E12C965FAF2C976596AEADBFAD65974F
:1036F000A215B30509F458C10E94D86B0E94E2B725
:10370000DC01CB01A7962CAD3DAD4EAD5FADA797CB
:10371000821B930BA40BB50BB7FD10C00E94E2B740
:103720009B01AC0128533F4F4F4F5F4FA7962CAFE3
:103730003DAF4EAF5FAFA7970E9457962C963FAD17
:103740002C9731502C963FAF2C97332309F44BC064
:10375000A3962CAD3DAD4EAD5FADA39727966CAD56
:103760007DAD8EAD9FAD27970E94C4FB6B017C01A0
:103770002B962CAD3DAD4EAD5FAD2B97B201C30185
:103780000E94C4FBA70196010E94D9FF7B018C0116
:10379000A3962CAD3DAD4EAD5FADA397B201C30175
:1037A0000E94C4FB4B015C012B962CAD3DAD4EAD90
:1037B0005FAD2B9727966CAD7DAD8EAD9FAD2797F6
:1037C0000E94C4FB9B01AC01C501B4010E94D8FF5B
:1037D0002B013C01C701D80127968CAF9DAFAEAF3E
:1037E000BFAF279761C065964EAD5FAD6597BA01D3
:1037F00080E090E00E9463FB2B962CAD3DAD4EAD7A
:103800005FAD2B970E94C4FB4B015C010F94B2008B
:103810006B017C01C501B4010F943A024B015C01BC
:10382000A701960123966CAD7DAD8EAD9FAD23971C
:103830000E94C4FB2B013C01A501940163966CAD71
:103840007DAD8EAD9FAD63970E94C4FB9B01AC0123
:10385000C301B2010E94D9FF2B013C01A5019401D3
:1038600023966CAD7DAD8EAD9FAD23970E94C4FBBA
:103870004B015C01A701960163966CAD7DAD8EADE9
:103880009FAD63970E94C4FB9B01AC01C501B401CD
:103890000E94D8FF27966CAF7DAF8EAF9FAF279762
:1038A00059E12C965FAF2C979201A3016B966CADFA
:1038B0007DAD8EAD9FAD6B970E94D9FF69837A83F2
:1038C0008B839C8327962CAD3DAD4EAD5FAD279786
:1038D0006F966CAD7DAD8EAD9FAD6F970E94D9FF99
:1038E0006D837E838F839887AB962CAD3DAD4EADB7
:1038F0005FADAB9769857A858B859C850E94D9FFE2
:1039000069877A878B879C87AF962CAD3DAD4EAD8E
:103910005FADAF976D857E858F8598890E94D9FFB1
:103920006D877E878F87988B80914A02882321F04C
:10393000CE0101960E94A694E090F91889819A819F
:10394000AB81BC8188A399A3AAA3BBA38D819E81CF
:10395000AF81B8858CA39DA3AEA3BFA389859A85AB
:10396000AB85BC8588A799A7AAA7BBA7CE018096DF
:103970000E94E14F8E01055C1F4F9E01235F3F4F68
:10398000AE01485D5F4FBE016C5D7F4FCE018096FA
:103990000E94059065968EAD9FAD659701966596E0
:1039A0009FAF8EAF6597A0CEE090F9188091461436
:1039B00090914714A0914814B091491488A399A3F9
:1039C000AAA3BBA380914A1490914B14A0914C14CC
:1039D000B0914D148CA39DA3AEA3BFA380914E14B0
:1039E00090914F14A0915014B091511488A799A7A9
:1039F000AAA7BBA7CE0180960E94E14F8E01055C6D
:103A00001F4F22E534E1AE01485D5F4FBE016C5DA2
:103A10007F4FCE0180960E9405900E94DB510E944C
:103A2000E94F0C944731ECE5F9E284918F010F5F87
:103A30001F4F882339F0082E000C990B0E94CBA54C
:103A4000F801F3CFE3EBF1E084918F010F5F1F4F9B
:103A5000882311F40C944731082E000C990B0E9416
:103A6000CBA5F801F1CF0E9474A50C9447310E94B8
:103A7000BA6D80E00E941DD80E94BBD811E010935F
:103A8000720E88E50E945750E82E89E50E94575033
:103A9000082F8AE50E945750F82EE11004C001114A
:103AA00004C0182705C0011102C010E001C0182F82
:103AB0000E949250111104C0E11002C00023C1F114
:103AC00080E090E0A0EAB0E480934E1490934F140D
:103AD000A0935014B09351149C01AD016091F90C66
:103AE0007091FA0C8091FB0C9091FC0C0E945FFB92
:103AF00087FF0BC019821A821B821C82BE016F5F76
:103B00007F4F8EE494E10E94C0D9111105C0E110ED
:103B100003C0011107C00CC080E090E00E943895FE
:103B20001123B9F381E090E00E943895111102C091
:103B3000FF2021F082E090E00E9438950E94BB4E69
:103B40008091710E8093720E0E94A1D80E94F6C2DD
:103B50000C9447310E94D9A00C944731C090F10CCD
:103B6000D090F20CE090F30CF090F40C88E50E94F9
:103B70008650811109C020E030E048E152E4C701DD
:103B8000B6010E94D8FF02C00E94245068A379A306
:103B90008AA39BA3C090F50CD090F60CE090F70C94
:103BA000F090F80C89E50E948650811109C020E050
:103BB00030E048EC51E4C701B6010E94D8FF02C0D2
:103BC0000E9424506B017C0169837A838B839C83E0
:103BD00088A099A0AAA0BBA02FE632E143E85AEB47
:103BE000C501B4010F94FF0187FF02C00C94473157
:103BF00022E430E042E253E4C501B4010E945FFBDD
:103C0000181614F40C9447312FE632E143E85AEBCE
:103C1000C701B6010F94FF0187FF02C00C94473122
:103C200022E430E04FE253E4C701B6010E945FFB9B
:103C3000181614F40C9447310C944E3181E08093A3
:103C4000A1030C9447310E94BA6D19E5212E12E0B0
:103C5000312E03E9C02E0CE0D02EE12CF12C00E037
:103C600010E01FAEF10181911F010E948650882350
:103C700009F450C00E9424504B015C01033011052F
:103C800059F0F701E65DFB4E20813181428153817D
:103C90000E94D8FF4B015C01F701EF50F34F2081E8
:103CA000318142815381C501B4010E94D8FF2B01AB
:103CB0003C012DEB37E346E855EB0F94FF0187FD00
:103CC0000AC02DEB37E346E855E3C301B2010E9479
:103CD0005FFB1816FCF40330110559F48092FD0CBB
:103CE0009092FE0CA092FF0CB092000DF1E0FFAF9D
:103CF00011C0A3019201D6016D917D918D919C918E
:103D00000E94D9FFF6016083718382839383C80187
:103D10000E9453DA0F5F1F4FF4E0CF0ED11C24E056
:103D2000E20EF11C0430110509F09CCF3FAD3111BA
:103D30000E94D0A50E94F6C20C94473180910C02DB
:103D4000882311F40C94473189E40E948650182F7F
:103D5000882321F00E94F44FE62E01C0E12C8AE472
:103D60000E948650082F882331F00E94F44FF62ECF
:103D7000111104C00BC0F12C1123D9F045E04E15F0
:103D800010F00C94FD34EBEDF1E004C055E05F154C
:103D9000D0F30FC084918F010F5F1F4F882311F460
:103DA0000C944731082E000C990B0E94CBA5F8010A
:103DB000F1CF0E9492501123F1F020914E0C3091DE
:103DC0004F0C4E2D4203B001439F700D1124809182
:103DD0004A0C90914B0C680F791F072E000C880B32
:103DE000990B0E9465FB609346147093471480936F
:103DF0004814909349140023F1F02091500C309115
:103E0000510C5F2D5203B001539F700D112420916E
:103E10004C0C30914D0C620F731F072E000C880B59
:103E2000990B0E9465FB60934A1470934B14809326
:103E30004C1490934D1480E50E948650882319F00D
:103E40000E94155003C080E50E945750882381F1DD
:103E50001123B1F020E030E048E152E460914614D3
:103E60007091471480914814909149140E94D9FF91
:103E700060934614709347148093481490934914A8
:103E80000023B1F020E030E048EC51E460914A14A6
:103E900070914B1480914C1490914D140E94D9FF55
:103EA00060934A1470934B1480934C1490934D1468
:103EB00086E40E9486508823D9F00E9424506B012A
:103EC0007C0120E030E0A9010F94FF01181684F472
:103ED00020E030E040E752E4C701B6010F94B5009E
:103EE00060933C0270933D0280933E0290933F02A8
:103EF0000E94F6DA0C9447318091EE149091EF1401
:103F00008237910509F42AC70CF0E8C08C3491057A
:103F100009F48FC40CF085C08A31910509F440C2C0
:103F20000CF03FC08531910509F40FC224F58231B0
:103F3000910509F40BC78431910509F4BBC1419780
:103F400011F00C9447318AEF91E00E9425C18E98C0
:103F50009FB7F894809108018D7F809308019FBFDF
:103F60009FB7F894809108018F7E809308019FBFCE
:103F70008B980C9447318731910509F4F0C10CF40A
:103F8000E8C18831910509F400C2499711F00C94F9
:103F9000473110922B0F80E09FE00E945A6D0C94E5
:103FA00047318032910509F469C324F58C319105BC
:103FB00009F44CC20CF402C28E31910509F450C2CE
:103FC0004F9711F00C94473180E09FE00E942D6DD7
:103FD00068A379A38AA39BA3BE016F5F7F4FCE0125
:103FE00080960E94124FCE0101960E94ECA7ECEC45
:103FF000F2E290C38033910509F4ECC32CF48A9764
:1040000009F4A2C30C9447318133910509F4E6C346
:104010008B34910511F00C9447310E9464E20C94AA
:1040200047318836910509F440C584F582359105FC
:1040300009F483C6C4F48E34910509F404C40CF465
:10404000FEC38135910511F00C9447310E94D8BA16
:104050000E94BA6D0E94DDDA1092011410920014D1
:1040600000E010E053C68435910509F46FC60CF4E6
:1040700068C68535910509F46DC68C35910511F03A
:104080000C9447310E9404C40C9447318D3691053D
:1040900009F412C69CF48A36910509F42FC60CF473
:1040A000C3C58B36910509F42DC68C36910511F0E8
:1040B0000C944731109200020C9447318F369105D1
:1040C00009F45CC50CF447C58037910509F45AC55D
:1040D0008137910509F45AC50C944731823E910508
:1040E00011F40C941E2A0CF065C08E3B910509F466
:1040F00001C624F58737910509F442C67CF485375B
:10410000910509F431C60CF037C68337910511F0DB
:104110000C9447310E94ACC20C9447318937910509
:1041200009F4BEC60CF4B5C68C38910509F45EC519
:104130008B39910509F499C50C9447318D3C910553
:1041400009F4AEC7ACF4893C910509F4F7C634F420
:10415000883C910509F4AAC60C9447318B3C910523
:1041600009F40FC78C3C910509F42AC70C94473118
:10417000833D910511F40C94DA2884F48E3C91056A
:1041800011F00C94473149E5C42E42E0D42E5BE097
:10419000E52E5AE0F52E00E010E0F9C78C3D9105C0
:1041A00011F40C94CA298D3D910511F40C94D72972
:1041B0000C944731843AA1E09A0711F40C94922EA2
:1041C000CCF58336E1E09E0711F40C94AA309CF400
:1041D0008E3221E0920711F40C946E2A8F3231E076
:1041E000930711F40C94C82A8D32914011F00C946D
:1041F00047310C94482A813951E0950711F40C9409
:104200008A2E4CF48039914011F00C9447310E9471
:10421000BA6D0C9447318239E1E09E0711F40C9499
:104220008E2E8A39914011F00C9447310E9430C291
:104230000C944731863F21E0920711F40C943730FB
:10424000FCF48C3A41E0940711F40C94742F4CF474
:10425000853A914011F00C9447310E9481C10C9431
:104260004731843FB1E09B0711F40C943430853F13
:10427000914011F00C9447310E94E87B0C94473137
:104280008335F3E09F0711F40C9446303CF4873FEC
:10429000914011F40C943A300C944731803A43E049
:1042A000940709F42AC2873E934011F40C94C93054
:1042B0000C944731E2E1F2E084918F010F5F1F4FD0
:1042C000882339F0082E000C990B0E94CBA5F80129
:1042D000F3CF1092B1111092B01140E050E0BA014A
:1042E0008CE59FE00E94EE608BE1ECE5FFE0DE01F3
:1042F000159601900D928A95E1F780915A0F909151
:104300005B0F9C838B8387EA92E09A83898340E0EA
:1043100050E0BE016F5F7F4F8AE993E00E94AEA834
:10432000CE0101960E941896E3E0F2E084918F019D
:104330000F5F1F4F882311F40C944731082E000C97
:10434000990B0E94CBA5F801F1CF0E94C6BF0C9437
:10435000473110922B0F10922C0F0C944731E091A3
:10436000EC14F091ED148081882329F0803209F457
:1043700010823196F8CF40E061E08091EC1490918A
:10438000ED140E945BBC0C94473180912C0F882364
:1043900019F081E080932B0F0E9464E20C94473166
:1043A00080912C0F882311F40C94473183E50E94EF
:1043B000865081110C94A6310C94473180912C0FBA
:1043C000882399F1E3E2F2E084918F010F5F1F4FA0
:1043D000882339F0082E000C990B0E94CBA5F80118
:1043E000F3CF4091A7115091A8116091A91170913C
:1043F000AA112AE08EEA9DE00E9479768FE290E091
:104400000E94CBA54091A3115091A4116091A511D8
:104410007091A6112AE08EEA9DE00E9479768AE0EA
:1044200090E00E94CBA50C944731E5E3F2E0849143
:104430008F010F5F1F4F882311F40C944731082E12
:10444000000C990B0E94CBA5F801F1CF40E060E091
:104450008091EC149091ED140E945BBC0C94473158
:1044600080912C0F882311F40C94473186EF90E152
:104470000E94BC6086EF90E10E94D16610922A0FE4
:104480001092290FE090EC14F090ED1480912C0F15
:10449000882311F40C9447310E94D4AA1D821886F7
:1044A0001C821B8287EA92E09A83898388E59FE0D9
:1044B0009093780F8093770FD7018C918F3209F00A
:1044C00066C06FE270E0C7010F94F8038C010F5FC4
:1044D0001F4FFE0131964F010115110509F45DC012
:1044E0006FE270E0C8010F94F8036C01009709F4C3
:1044F00055C00817190708F051C05C01A01AB10A8D
:10450000A501B801CE0180960F942104E0E2F0E00D
:10451000EC0FFD1FEA0DFB1D1082BE01605E7F4F98
:104520008EEA9DE00E94C9768AE090E00E94CBA5C9
:104530006091770F7091780F6115710511F06C5FC4
:104540007F4F21E0AE01405E5F4FCE0105960E9495
:10455000D966811114C0BE01605E7F4F8CE692E087
:104560000E94268E8EE290E00E94CBA58AE090E029
:104570000E94CBA5C4010E9418960C9447319092DA
:10458000780F8092770F86010F5F1F4FA5CF89E7C5
:104590009FE09093780F8093770F87016091770F5A
:1045A0007091780F6115710511F06C5F7F4F18A243
:1045B0001BA222E0A801CE0180960E94D96681113B
:1045C00002C0F12C14C0CE0180960E941CA8882342
:1045D000C1F361E0CE0180960E942E92009789F38C
:1045E00025EEDC012C931BA20E94CD5EF82ECE019D
:1045F00080960E94D24FFF2011F1E6E4F2E0849110
:104600007F01BFEFEB1AFB0A882339F0082E000C5C
:10461000990B0E94CBA5F701F2CFB8018EEA9DE07D
:104620000E94C9768AE090E00E94CBA51092A71163
:104630001092A8111092A9111092AA1119C0E4E5C4
:10464000F2E084917F012FEFE21AF20A882339F019
:10465000082E000C990B0E94CBA5F701F2CFB801F0
:104660008EEA9DE00E94C9768EE290E00E94CBA582
:10467000CE0101960E9418960C94473180912B0F21
:1046800081110E94BA6D80912C0F882311F40C9433
:10469000473180E50E948650882319F00E9415500A
:1046A00003C080E50E945750182F482F61E0809189
:1046B000EC149091ED140E945BBC83E50E9486503F
:1046C000882381F00E94F44FAB01BC014093A711F5
:1046D0005093A8116093A9117093AA1186EF90E1ED
:1046E0000E94EE6080912C0F882319F081E0809366
:1046F0002B0F11110C9447314FCE8091EC149091F7
:10470000ED1421E020932A0F40E060E00E945BBCA2
:104710000C94473184918F010F5F1F4F882339F02C
:10472000082E000C990B0E94CBA5F801F3CFBE0117
:104730006F5F7F4F80E892E00E94268E8AE090E0D3
:104740000E94CBA50C94473183E50E9486508823B4
:1047500011F40C9447310E940450E82E80E50E9429
:104760008650882341F00E94F44F8B0177FF02C0EE
:104770000C94473102C00DE010E0902FE5E8F4E022
:1047800088E28E0F2491921729F031968E13FACF7A
:104790000C94B731ECE5F9E284918F010F5F1F4F64
:1047A000882339F0082E000C990B0E94CBA5F80144
:1047B000F3CFEDE8F2E084918F010F5F1F4F882364
:1047C00011F40C944731082E000C990B0E94CBA5D4
:1047D000F801F1CF0E94389B0C944731F0909C0374
:1047E00081E0F826F0929C03E7EAF2E084918F01E1
:1047F0000F5F1F4F882339F0082E000C990B0E9481
:10480000CBA5F801F3CFF11003C0E1EAF2E002C05A
:10481000ECE9F2E084918F010F5F1F4F882311F4C0
:104820000C944731082E000C990B0E94CBA5F8017F
:10483000F1CF80E09FE00E945A6D0C9447310E94B6
:104840000EA60C94473183E50E948650882359F0C8
:104850000E94F44F6E34710531F480E09FE00E94B5
:10486000588E0C94473118A219A21AA21BA2E2E199
:10487000F3E084918F010F5F1F4F882339F0082EDA
:10488000000C990B0E94CBA5F801F3CFE9E0F3E00F
:1048900084918F010F5F1F4F882339F0082E000C81
:1048A000990B0E94CBA5F801F3CF40910E0F5091C8
:1048B0000F0F60E070E02AE08EEA9DE00E947976BA
:1048C000ECEFF2E084918F010F5F1F4F882339F0E6
:1048D000082E000C990B0E94CBA5F801F3CF409154
:1048E000100F5091110F60E070E02AE08EEA9DE019
:1048F0000E947976E1EFF2E084918F010F5F1F4F04
:10490000882339F0082E000C990B0E94CBA5F801E2
:10491000F3CF40910E0F50910F0F8091100F909197
:10492000110F481B590B8091000F9091010F0197B7
:1049300021E030E0029710F020E030E0421B530B02
:1049400060E070E02AE08EEA9DE00E9479768AE0DD
:1049500090E00E94CBA5E9EEF2E084918F010F5F19
:104960001F4F882339F0082E000C990B0E94CBA50D
:10497000F801F3CF8091120F9091130FA091140FB3
:10498000B091150F88A399A3AAA3BBA3BE016F5F23
:104990007F4FCE0180960E94124FECEDF2E08491A1
:1049A0008F010F5F1F4F882339F0082E000C990BE1
:1049B0000E94CBA5F801F3CFBE016F5F7F4F8EEA57
:1049C0009DE00E94C9768091160F9091170FA091DB
:1049D000180FB091190F88A399A3AAA3BBA3BE0176
:1049E0006F5F7F4FCE0180960E94124FECECF2E099
:1049F00084918F010F5F1F4F882339F0082E000C20
:104A0000990B0E94CBA5F801F3CFBE016F5F7F4FDA
:104A10008EEA9DE00E94C9768AE090E00E94CBA5D4
:104A2000E4ECF2E084918F010F5F1F4F882339F08F
:104A3000082E000C990B0E94CBA5F801F3CFE4EBF4
:104A4000F2E084918F010F5F1F4F882339F0082E09
:104A5000000C990B0E94CBA5F801F3CF20E030E0C9
:104A60004AE754E460911A0F70911B0F80911C0F5C
:104A700090911D0F0F94B50042E050E00E94A7C72F
:104A8000E2EBF2E084918F010F5F1F4F882339F032
:104A9000082E000C990B0E94CBA5F801F3CF8AE0F9
:104AA00090E00E94CBA50C94473188E690E00E94EC
:104AB00094DA81110C9447318091680C83FF02C015
:104AC0000C94473183E50E948650882309F43FC047
:104AD0000E9424500F941D017093FF136093FE13E6
:104AE00080E00E9471690E94245020E030E04AEA90
:104AF00052E40E945FFB181634F00E940EA681E279
:104B000093E00E9425C10E9424502091021430910C
:104B1000031440910414509105140F94FF011816CA
:104B2000B4F482EE92E09F938F938091D51190E040
:104B300001969F938F938AE193E09F938F931F92A7
:104B40000E943BF10FB6F894DEBF0FBECDBF0E94AE
:104B5000CFED0C9447318EE40E948650882311F4E7
:104B60000C9447310E94F44F60930C1470930D1411
:104B700080930E1490930F140C9447310E941AC521
:104B80000C94473182E493E00E94209683E50E94D2
:104B90008650882369F00E9404508D3320F480935E
:104BA00023020C9447318CE3809323020C94473109
:104BB000ECECF2E284918F010F5F1F4F882339F0F4
:104BC000082E000C990B0E94CBA5F801F3CF409161
:104BD000230250E060E070E08BE493E00E94958D4A
:104BE0008AE090E00E94CBA50C9447318091680C3C
:104BF00083FF02C00C94473183E50E9486508823CE
:104C000011F40C9447310E9424500F941D01673910
:104C1000710514F066E970E07093FD136093FC1366
:104C20000E9426690C94473189E690E00E9494DA4C
:104C3000811115C0E2E5F3E084918F010F5F1F4FF2
:104C4000882339F0082E000C990B0E94CBA5F8019F
:104C5000F3CF0E94E0B88AE090E00E94CBA51092CA
:104C6000830C1092820C0C942C3583E50E948650A4
:104C7000882311F40C9447310E940450182F8D336F
:104C800008F01CE31093880C0E94E2B76B017C01D2
:104C9000212F30E0A8EEB3E00E94C9FFC60ED71E58
:104CA000E81EF91EC092840CD092850CE092860C0E
:104CB000F092870C0C9447318DE690E00E9494DAD4
:104CC00081110C9447318091680C83FF02C00C94D1
:104CD000473183E50E94865060968FAF60978111BF
:104CE0000C94CD3182E50E94865081110C94CD3117
:104CF0000C9447310E949FC50C9447310E9449C7CC
:104D00000C9447310E943AC70C94473162E370E03B
:104D100080E090E00E94AAB70E94D86B0F5F1F4FFF
:104D20000331110599F762E370E080E090E00E94A2
:104D3000AAB70E94D86B0C9447311092A0030C9430
:104D4000473181E08093A0030C9447310E94BAC49C
:104D50000C9447310E94A2C40C9447310E94BA6D52
:104D60000E94F6C20C9447318091EC149091ED149E
:104D70000E94ECA70C9447310E9466C20C94473104
:104D8000E1EBF3E084918F010F5F1F4F882339F02F
:104D9000082E000C990B0E94CBA5F801F3CFE9EA8D
:104DA000F3E084918F010F5F1F4F882339F0082EA5
:104DB000000C990B0E94CBA5F801F3CF789B03C0A0
:104DC00061ED72E002C067EC72E08EEA9DE00E9445
:104DD000C9768AE090E00E94CBA5E1EAF3E08491F5
:104DE0008F010F5F1F4F882339F0082E000C990B9D
:104DF0000E94CBA5F801F3CF029B03C061ED72E0E6
:104E000002C067EC72E08EEA9DE00E94C9768AE0FB
:104E100090E00E94CBA5E9E9F3E084918F010F5F58
:104E20001F4F882339F0082E000C990B0E94CBA548
:104E3000F801F3CF019B03C061ED72E002C067ECA3
:104E400072E08EEA9DE00E94C9768AE090E00E94BE
:104E5000CBA5EFE8F3E084918F010F5F1F4F88230C
:104E600039F0082E000C990B0E94CBA5F801F3CF66
:104E7000039903C061ED72E002C067EC72E08EEA54
:104E80009DE00E94C9768AE090E00E94CBA50C9438
:104E9000473181E08093720E8093710E0C944731FC
:104EA0001092720E1092710E0C94473188EC90E0C3
:104EB0000E9494DA81110C94473184E40E94575087
:104EC0008823C1F10E94245011E020E030E0A901C4
:104ED0000E945FFB811101C010E01093560C11235A
:104EE00049F10E942450E091D511A4E0EA9FF0011D
:104EF0001124E55AF34F608371838283938320E00A
:104F000030E0A90160915B0C70915C0C80915D0CAC
:104F100090915E0C0E945FFB81110CC080E090E0DC
:104F2000A0EEBFE380935B0C90935C0CA0935D0CB0
:104F3000B0935E0C0E94C9910C944731EEEBEE2EBB
:104F4000E3E0FE2E09E512E0F4E0DF2ED00EF801DA
:104F500081918F010E945750882351F00E94245064
:104F60000F942201D7016D937D938D939C9313979A
:104F7000B4E0EB0EF11CD012EACF0E946D8E0C94BF
:104F8000473166EDE62E63E0F62E09E512E074E0A7
:104F9000D72ED00EF80181918F010E94575088239F
:104FA00041F00E942450D7016D937D938D939C9383
:104FB0001397B4E0EB0EF11CD012ECCF0C944731F8
:104FC00083E50E9457508823E1F00E942450AB01F2
:104FD000BC014093BA035093BB036093BC0370932E
:104FE000BD034093B2035093B3036093B403709333
:104FF000B50385E294E00E94E18D8AE090E00E9492
:10500000CBA580E50E9457508823A1F00E94245030
:10501000AB01BC014093BA035093BB036093BC0344
:105020007093BD0388E094E00E94E18D8AE090E0F7
:105030000E94CBA582E50E9457508823A1F00E94D0
:105040002450AB01BC014093B6035093B703609367
:10505000B8037093B90389EE93E00E94E18D8AE072
:1050600090E00E94CBA584E50E945750882311F45C
:105070000C9447310E942450AB01BC014093B20311
:105080005093B3036093B4037093B5038BEC93E038
:105090000E94E18D8AE090E00E94CBA50C944731FC
:1050A00083E50E945750882351F00E94245060935A
:1050B000D2037093D3038093D4039093D50384E5F4
:1050C0000E945750882351F00E9424506093CE03D1
:1050D0007093CF038093D0039093D10382E40E9416
:1050E0005750882351F00E94024F6093600C7093D8
:1050F000610C8093620C9093630C88E50E9457507A
:10510000882351F00E9424506093A2037093A3035C
:105110008093A4039093A50389E50E9457508823A8
:1051200051F00E9424506093A6037093A7038093CC
:10513000A8039093A9038AE50E945750882351F051
:105140000E9424506093AA037093AB038093AC0336
:105150009093AD0385E40E945750882311F40C947A
:1051600047310E9424506093AE037093AF03809345
:10517000B0039093B1030C9447310F5F1F4FB4E01D
:10518000EB0EF11C0330110511F40C949A1EF6017C
:1051900081916F010E945750882379F30E94245017
:1051A000D7016D937D938D939C931397C8010E94B3
:1051B00053DAE3CFECECF2E284918F010F5F1F4FE3
:1051C000882339F0082E000C990B0E94CBA5F8011A
:1051D000F3CF83E50E945750882321F00E94155099
:1051E00080934A02E5E7F4E084918F010F5F1F4F3F
:1051F000882339F0082E000C990B0E94CBA5F801EA
:10520000F3CF80914A02811103C0E1E7F4E002C0CC
:10521000EDE6F4E084918F010F5F1F4F882339F092
:10522000082E000C990B0E94CBA5F801F3CFE5E600
:10523000F4E084918F010F5F1F4F882339F0082E0F
:10524000000C990B0E94CBA5F801F3CF20912A14F2
:1052500030912B1440912C1450912D1460919F0C7F
:105260007091A00C8091A10C9091A20C0E94D9FF8A
:10527000AB01BC0183E694E00E94E18D20912E14E5
:1052800030912F1440913014509131146091A30C3F
:105290007091A40C8091A50C9091A60C0E94D9FF4E
:1052A000AB01BC0180E694E00E94E18D20913214B4
:1052B0003091331440913414509135146091A70CFF
:1052C0007091A80C8091A90C9091AA0C0E94D9FF12
:1052D000AB01BC018DE594E00E94E18DE5E5F4E0D1
:1052E00084918F010F5F1F4F882339F0082E000C27
:1052F000990B0E94CBA5F801F3CF20912A1430918D
:105300002B1440912C1450912D146091280270910F
:10531000290280912A0290912B020E94D9FFAB01B1
:10532000BC0183E594E00E94E18D20912E14309120
:105330002F14409130145091311460912C027091CF
:105340002D0280912E0290912F020E94D9FFAB0175
:10535000BC0180E594E00E94E18D209132143091EF
:10536000331440913414509135146091300270918F
:10537000310280913202909133020E94D9FFAB0139
:10538000BC018DE494E00E94E18D8AE090E00E94EF
:10539000CBA57DC783E50E948650882309F477C793
:1053A0000E94F44F709302026093010270C78DED6A
:1053B00090E00E9494DA81116AC783E50E948650CA
:1053C000882309F464C70091D51110E00E94F44FBE
:1053D000000F111FF801ED5EFD4F71836083809116
:1053E000D51190E08C01000F111F000F111FF80163
:1053F000EC59F34F7F01880F991FFC01ED5EFD4FC3
:1054000060817181072E000C880B990B0E9465FB4F
:105410002AE037ED43E25CE30E94C4FBF801E95A5D
:10542000F34F20813181428153810E94C4FBD70117
:105430006D937D938D939C93139729C780E50E946C
:105440005750882309F423C70E94F44F6B017C0155
:1054500083E50E948650882321F00E94F44F8B013F
:1054600002C00FEF1FEFC8010196039708F00FC7A6
:10547000D7FC0DC79C2DE5E8F4E088E28E0F24915F
:10548000921709F404C731968E13F9CF0C940435A2
:1054900085E40E948650811103C00E94FFEDF7C68B
:1054A0000E9404508823C9F3ECE5F9E284918F014E
:1054B0000F5F1F4F882339F0082E000C990B0E94B4
:1054C000CBA5F801F3CF6DEE72E08EEA9DE00E946D
:1054D000C9768AE090E00E94CBA5D9C683E50E94F8
:1054E0005750182F882371F00E9424500F941D01EB
:1054F000709316026093150221E0672B09F020E0FB
:1055000020935F0C80E50E945750882359F020912A
:10551000150230911602232B11F00E941550809332
:105520005F0CB5C61111B3C6ECECF2E284918F01A9
:105530000F5F1F4F882339F0082E000C990B0E9433
:10554000CBA5F801F3CF80915F0C811103C066ED0C
:1055500072E002C063ED72E082EC94E00E94268E5D
:10556000609115027091160281EB94E00E94028E08
:10557000EDEAF4E084918F010F5F1F4F882309F457
:1055800086C6082E000C990B0E94CBA5F801F2CF1D
:1055900085E40E948650882321F00E94F44F7B010D
:1055A00002C0E12CF12C83E40E948650882341F054
:1055B0000E94F44FC058DF4F6883C058D04006C0E7
:1055C00025E0C058DF4F2883C058D04085E50E94B1
:1055D0008650882319F00E94155003C085E50E946B
:1055E0005750C457DF4F8883CC58D040F7FC07C0D2
:1055F000812C912CB6E1AB2EB3E4BB2E06C0812CDE
:10560000912CACE8AA2EA2E4BA2E83E50E94865023
:10561000882321F00E9424504B015C01E114F10425
:1056200011F41092D5110E94E2B72B013C01EE203B
:1056300059F06EEF72E08EEA9DE00E94C9768AE032
:1056400090E00E94CBA523C6C501B4010F941D01B3
:10565000072E000C880B990B0E9465FB60966FAFBC
:10566000609728967FAF28972C968FAF2C976496DB
:105670009FAF6497D301C201805D9A48AF4FBF4F7F
:10568000CB56DF4F88839983AA83BB83C559D0400B
:1056900067E273E08EEA9DE00E94C9768AE090E0BE
:1056A0000E94CBA50E94D8BA8FE78093D31181E0E6
:1056B00080930002CC57DF4F488259826A827B82F6
:1056C000C458D040C357DF4F488259826A827B82D8
:1056D000CD58D040CD57DF4F1882C358D040CF5659
:1056E000DF4F188219821A821B82C159D0406C96F2
:1056F0001FAE6C9790E4A0969FAFA097ACE1A496E4
:10570000AFAFA497B6E4E096BFAFE097E4961FAEC4
:10571000E497A8961FAEA897AC961FAEAC97E896F4
:105720001FAEE897C458DF4F188219821A821B8275
:10573000CC57D040EC961CAE1DAE1EAE1FAEEC9703
:10574000C12CD12C7601FFE78F2E912CA12CB12CEE
:105750002FE730E040E050E027962CAF3DAF4EAF52
:105760005FAF2797C857DF4F188219821A821B82B2
:10577000C858D04031E0CE57DF4F3883C258D040B0
:1057800069961FAE1EAE699710E0212C312C00E007
:10579000C058DF4F4881C058D040042E000C550B34
:1057A000C058DF4F59834883C058D04080910002D1
:1057B000882309F413C10E94E2B723966CAF7DAF32
:1057C0008EAF9FAF23978091D111882309F4E2C057
:1057D0000E945B6A1091021420900314309004140C
:1057E00000910514212F322D432D502FE4966FADDB
:1057F000E497A8967FADA897AC968FADAC97E89646
:105800009FADE8970E945FFB87FF0CC0E4961FAF37
:10581000E497A8962FAEA897AC963FAEAC97E896C3
:105820000FAFE897212F322D432D502F6C966FAD7F
:105830006C97A0967FADA097A4968FADA497E096A5
:105840009FADE0970F94FF01181664F46C961FAF9C
:105850006C97A0962FAEA097A4963FAEA497E09623
:105860000FAFE097CE57DF4F5881C258D0406096B7
:105870002FAD609728963FAD28972C964FAD2C976B
:10588000552309F462C064965FAD6497612F722D51
:10589000832D902F0F94FF0118160CF07BC02396D8
:1058A0004CAD5DAD6EAD7FAD2397441955096609CA
:1058B0007709DB01CA0188589341A109B109B7FDF5
:1058C00069C027968CAD9DADAEADBFAD2797881949
:1058D0009909AA09BB09B595A795979587958093CE
:1058E000D311C857DF4F488359836A837B83C858D5
:1058F000D04060968FAD6097E4968FAFE49728967E
:105900009FAD2897A8969FAFA8972C96AFAD2C97E0
:10591000AC96AFAFAC976496BFAD6497E896BFAF57
:10592000E89723962CAD3DAD4EAD5FAD2397CC5798
:10593000DF4F288339834A835B83C458D040CE57D6
:10594000DF4F1882C258D04025C064965FAD64977F
:10595000612F722D832D902F0E945FFB87FF1AC04D
:1059600023968CAD9DADAEADBFAD2397CC57DF4F29
:10597000288139814A815B81C458D040821B930BB6
:10598000A40BB50BAC01BD01485853416109710925
:1059900077FF9CC620E030E040EA51E460966FADAE
:1059A000609728967FAD28972C968FAD2C9764969C
:1059B0009FAD64970E94D9FF9B01AC01612F722DAE
:1059C000832D902F0F94FF01181694F4E7EEF5E065
:1059D00084918F010F5F1F4F811103C00E94D8BABD
:1059E00056C4082E000C990B0E94CBA5F801F0CFED
:1059F00023968CAD9DADAEADBFAD2397C357DF4FA2
:105A0000288139814A815B81CD58D040821B930B1C
:105A1000A40BB50BB7FDBAC00E94E0B80E94E8CF56
:105A20008AE090E00E94CBA523968CAD9DADAEADF3
:105A3000BFAD23978053984FAF4FBF4FC357DF4F32
:105A400088839983AA83BB83CD58D040CD57DF4F3D
:105A50009881C358D040911176C0CF56DF4F28812E
:105A600039814A815B81C159D040612F722D832DCC
:105A7000902F0F94FF0118160CF04CC020E030E07E
:105A800040EE50E460966FAD609728967FAD289702
:105A90002C968FAD2C9764969FAD64970E94D8FF8B
:105AA0009B01AC01A1E0CD57DF4FA883C358D04084
:105AB000612F722D832D902F0F94FF0118162CF05B
:105AC000CD57DF4F1882C358D04020E030E040E48B
:105AD00050E4612F722D832D902F0E94D9FFCF5655
:105AE000DF4F688379838A839B83C159D040239693
:105AF0002CAD3DAD4EAD5FAD2397205D3A484F4F85
:105B00005F4FCB56DF4F288339834A835B83C55968
:105B1000D0403CC023968CAD9DADAEADBFAD2397BC
:105B2000CB56DF4F288139814A815B81C559D040EE
:105B3000821B930BA40BB50BB7FD28C049EC55E0B5
:105B400068ED75E020C020E030E040EA51E4609666
:105B50006FAD609728967FAD28972C968FAD2C97C8
:105B600064969FAD64970E94D8FF9B01AC01612FA2
:105B7000722D832D902F0E945FFB87FF07C049EA9B
:105B800055E069EB75E080E00E947E6A23968CAD5B
:105B90009DADAEADBFAD2397880F991FAA1FBB1F48
:105BA000CC57DF4F288139814A815B81C458D0406E
:105BB000821B930BA40BB50B84199509A609B70991
:105BC00081389F44A241B10580F0EBE8F5E0849173
:105BD0008F010F5F1F4F882309F400CF082E000CA0
:105BE000990B0E94CBA5F801F2CF69964EAD5FAD3F
:105BF0006997C058DF4F88819981C058D040841779
:105C000095070CF0D3CDEEE2F5E084918F010F5FA4
:105C10001F4F882339F0082E000C990B0E94CBA54A
:105C2000F801F3CFB701A60189E195E00E94E18D6B
:105C30008AE090E00E94CBA5EC964CAD5DAD6EADD8
:105C40007FADEC9784E095E00E94E18D8AE090E0E2
:105C50000E94CBA5C458DF4F488159816A817B815E
:105C6000CC57D0408FEE94E00E94E18D8AE090E026
:105C70000E94CBA5C457DF4F9881CC58D0409923C0
:105C800091F1C0922A19D0922B19E0922C19F0921E
:105C90002D192CEA35EC47E25EE3EC966CAD7DAD58
:105CA0008EAD9FADEC970E94C4FB60932E1970934C
:105CB0002F1980933019909331192CEA35EC47E273
:105CC0005EE3C458DF4F688179818A819B81CC571C
:105CD000D0400F94B50060933219709333198093BC
:105CE0003419909335196DED74E0CE0101960E9440
:105CF0003976CE0101960E94347685ED94E090933A
:105D0000FB138093FA130E94BA4B60E080E00E947C
:105D100069F4BDC281E00E94C7D9B9C280E00E9487
:105D2000C7D9B5C28091F10C9091F20CA091F30CFF
:105D3000B091F40C89839A83AB83BC838091F50C7A
:105D40009091F60CA091F70CB091F80C8D839E8386
:105D5000AF83B8878091F90C9091FA0CA091FB0C5D
:105D6000B091FC0C89879A87AB87BC8786E50E9437
:105D70005750882351F080914E0C90914F0C892BF5
:105D800021F00E9435F20E941DF28AE50E945750D0
:105D9000882321F00E9424500E94D1D283E50E94E2
:105DA0005750882331F00E941550182F0E941DD89B
:105DB00001C010E0F0901814111103C0ECECF2E2F5
:105DC00020C0F110FBCFECE5F9E284918F010F5F69
:105DD0001F4F882339F0082E000C990B0E94CBA589
:105DE000F801F3CFEBE7F6E084918F010F5F1F4FCF
:105DF000882321F3082E000C990B0E94CBA5F801F3
:105E0000F3CF84918F010F5F1F4F882339F0082E45
:105E1000000C990B0E94CBA5F801F3CFF11003C041
:105E20006EED72E002C06AED72E08DE696E00E94CF
:105E3000268E8AE090E00E94CBA5ECECF2E2849101
:105E40008F010F5F1F4F882339F0082E000C990B2C
:105E50000E94CBA5F801F3CFE0E6F6E084918F0134
:105E60000F5F1F4F882339F0082E000C990B0E94FA
:105E7000CBA5F801F3CFC0901914D0901A14E0907C
:105E80001B14F0901C1420E030E0A901C701B601FA
:105E90000F94FF0118165CF442E050E0C701B60110
:105EA0000E94A7C78AE090E00E94CBA50FC0EBE557
:105EB000F6E084918F010F5F1F4F882339F0082E81
:105EC000000C990B0E94CBA5F801F3CF4CE050E0F9
:105ED00061EF7CE0CE0101960F94C403892B09F495
:105EE000D6C10E94F6C2D3C10E9454CE8111CFC147
:105EF0009CE0892E90E2992EA1EFBCE02196BFAFE5
:105F0000AEAF2197FE0131965F0105E610E21F0159
:105F1000F3E0F00F2496FFAF2497F401659175919B
:105F2000859194912196AEADBFAD2197CD90DD9036
:105F3000ED90FD902196BFAFAEAF2197A7019601DE
:105F40000E94D8FF2B013C0120E030E040EA51ECF8
:105F50000F94FF0187FD10C020E030E040EA51E4DB
:105F6000C301B2010E945FFB181634F0F1014082B8
:105F70005182628273820EC0F80184911816B4F7C0
:105F8000F7FAF094F7F8F094D101CD92DD92ED920A
:105F9000FC921397D101CD90DD90ED90FD901D0105
:105FA00020E030E040EA51ECC701B6010F94FF0158
:105FB00087FF03C0ECE5F9E20BC020E030E040EAE7
:105FC00051E4C701B6010E945FFB181614F5F2CF29
:105FD00084918F010F5F1F4F882339F0082E000C2A
:105FE000990B0E94CBA5F801F3CFE8EBF6E0849182
:105FF0008F010F5F1F4F882339F0082E000C990B7B
:106000000E94CBA5F801F3CF8AEA96E00E9425C151
:106010003EC1B4E08B0E911C0F5F1F4F2496EFAD75
:106020002497E0137ACF8BE0E82E8AE0F82E00E088
:1060300010E0F50181919191A191B1915F01F7017A
:1060400081939193A193B1937F01C8010E9453DA88
:106050000F5F1F4F0330110561F70E94F6C28AE9F6
:1060600096E00E9425C113C10E9450AB10C10E944E
:10607000BF7A0DC183E50E945750882321F00E940A
:10608000155091E089270E94CB7601C1ECECF2E239
:1060900084918F010F5F1F4F882339F0082E000C69
:1060A000990B0E94CBA5F801F3CFE2EFF6E08491C3
:1060B0008F010F5F1F4F882339F0082E000C990BBA
:1060C0000E94CBA5F801F3CF8AE50E9457508823A0
:1060D00081F10E9424506B017C0120E030E040EA15
:1060E00051EC0F94FF0187FF03C0E9EDF6E013C008
:1060F00020E030E040EA51E4C701B6010E945FFBB6
:1061000018169CF3C0923614D0923714E0923814CB
:10611000F09239140EC084918F010F5F1F4F8823B6
:1061200009F4B5C0082E000C990B0E94CBA5F8010C
:10613000F2CF409136145091371460913814709119
:10614000391486ED96E00E94E18D8AE090E00E948D
:10615000CBA59DC0ECE5F9E284918F010F5F1F4F45
:10616000882339F0082E000C990B0E94CBA5F8016A
:10617000F3CFE1E0F7E084918F010F5F1F4F882399
:1061800009F485C0082E000C990B0E94CBA5F801DC
:10619000F2CF81E080930C0283E50E948650882331
:1061A00019F00E94155003C083E50E9457508111D9
:1061B0006EC00E94C7E06BC0F090EE14FF2059F152
:1061C000ECECF2E284918F010F5F1F4F882339F0CE
:1061D000082E000C990B0E94CBA5F801F3CF84E5A3
:1061E00090E00E94CBA54F2D50E060E070E02AE0E7
:1061F0008EEA9DE00E94797680E290E00E94CBA535
:106200006DEE72E08EEA9DE00E94C9768AE090E031
:106210000E94CBA53CC01092F918ECECF2E28491FC
:106220008F010F5F1F4F882339F0082E000C990B48
:106230000E94CBA5F801F3CF6091F91870E080E1DE
:1062400097E00E94028E8AE090E00E94CBA51FC0DA
:10625000ECECF2E284918F010F5F1F4F882339F03D
:10626000082E000C990B0E94CBA5F801F3CF60918A
:10627000890C70918A0C82E297E00E94268E82E25D
:1062800090E00E94CBA58AE090E00E94CBA51092FE
:10629000830C1092820C0E94A4E0DEC380E00E9476
:1062A0001DD80E94BBD885E40E948650882319F02F
:1062B0000E94155003C085E40E94575021E0482FEA
:1062C000BE016F5F7F4FCE0180960E946CD06B0144
:1062D0007C019B01AC010F948502811132C02CEA34
:1062E00035EC47E257E368A179A18AA19BA10E94FE
:1062F000D9FFAB01BC0183ED91E00E94C08D2CEA77
:1063000035EC47E257E369817A818B819C810E9459
:10631000D9FFAB01BC018EEC91E00E94C08D2CEA4C
:1063200035EC47E257E3C701B6010E94D9FFAB0144
:10633000BC0189EC91E00E94C08D8AE090E00E944F
:10634000CBA50E94A1D80E94F6C2A1CF0E94F44F13
:10635000AB01BC014093A7115093A8116093A91100
:106360007093AA1186EF90E10E94EE6090CF61E0F9
:10637000802F0E94A7B66E2D802F0E9478B6F12C38
:10638000B701802F0E94E3B60530110509F07FCFD9
:10639000F0920114E09200147ACF0E9424500F94DE
:1063A0001D017093FF136093FE1380E00E947169DA
:1063B0000E94245020E030E04AEA52E40E945FFB51
:1063C00018163CF00E940EA68EE693E00E9425C1AE
:1063D00002C00E9464E26091FE137091FF13072EC9
:1063E000000C880B990B0E9465FB209102143091E0
:1063F000031440910414509105140F94FF011816D2
:10640000B4F482EE92E09F938F938091D51190E047
:1064100001969F938F9387E693E09F938F931F92AC
:106420000E943BF10FB6F894DEBF0FBECDBF0E94B5
:10643000CFED81E08093000227961CAE1DAE1EAE0C
:106440001FAE27972B961CAE1DAE1EAE1FAE2B9710
:106450001FAE2C961FAE2C979CE364969FAF64975B
:10646000ACE16896AFAF6897B6E46C96BFAF6C9737
:10647000C12CD12CA0E8EA2EBFEBFB2E812C912C55
:1064800054016091FE137091FF13072E000C880BCE
:10649000990B0E9465FB162F072F782E692E262F49
:1064A000372F482F592FB601C7010E945FFB882361
:1064B00019F1209102143091031440910414509169
:1064C0000514612F702F872D962D0E945FFB881F6A
:1064D0008827881F8FAF6096EFAD6097EE2381F01D
:1064E000882371F080910002882309F4D0CE85E5DD
:1064F00093E00E9425C1CBCE1C2D0D2D7E2C6F2C40
:106500000E94E2B76B017C01DC01CB012B962CAD24
:106510003DAD4EAD5FAD2B97821B930BA40BB50B1E
:10652000B7FD44C0D701C60188519C4FAF4FBF4F44
:106530002B968CAF9DAFAEAFBFAF2B970E94E0B84C
:10654000E3E6F3E084912F019FEF491A590A88236B
:1065500039F0082E000C990B0E94CBA5F201F2CF66
:1065600081149104A104B104C9F0D501C401805F74
:10657000984DAF4FBF4FBC01CD016C197D098E09FD
:106580009F0928EE33E040E050E00E947BFFBA0113
:10659000A9018EEA9DE00E948BA604C08FE390E0E3
:1065A0000E94CBA58AE090E00E94CBA50E9457965E
:1065B0000E94E94F2090021430900314409004147C
:1065C000509005149101A201612F702F872D962DF7
:1065D0000E94D8FF9F7781149104A104B10449F46B
:1065E00020E030E040E85FE30E945FFB87FF0BC0E4
:1065F00008C020E030E040E450E40F94FF0118169A
:1066000014F446015701AFADAA2309F443C02796FD
:106610002CAD3DAD4EAD5FAD279721153105410540
:10662000510541F0D701C601821B930BA40BB50B9A
:10663000B7FD30C09101A2012C966FAD2C976496E6
:106640007FAD649768968FAD68976C969FAD6C9799
:106650000E94D8FF20E030E040EC5FE30E945FFB47
:1066600087FD40CFD701C601805A9541AF4FBF4F3C
:1066700027968CAF9DAFAEAFBFAF27972C962FAEAE
:106680002C9764963FAE649768964FAE68976C9669
:106690005FAE6C9780910002882309F423CF8114A8
:1066A0009104A104B10429F4C12ED02EE72CF62CBC
:1066B000E8CE90E1C91A97E2D90AE108F108C818B2
:1066C000D908EA08FB08F7FE0DCFEECF69964EAD6C
:1066D0005FAD6997452B09F451C1C857DF4F48801A
:1066E00059806A807B80C858D040480E591E6A1E67
:1066F0007B1EC857DF4F288139814A815B81C8588A
:10670000D040281B390B4A0B5B0BCA01B901A5010C
:1067100094010E946CFFA30192010E949DFF2796A5
:106720008CAC9DACAEACBFAC2797820E931EA41E62
:10673000B51E34E183169104A104B1041CF14CEEA2
:1067400084169104A104B1043CF450E88516910428
:10675000A104B10434F426C05BEE852E912CA12C4B
:10676000B12C27968CAE9DAEAEAEBFAE27978EEF06
:1067700090E0A0E0B0E088199909AA09BB094C0192
:106780005D0116C024E130E040E050E027962CAFD8
:106790003DAF4EAF5FAF279744E1842E912CA12CE3
:1067A000B12C06C027968CAE9DAEAEAEBFAE27977D
:1067B00027964CAD5DAD6EAD7FAD279783E596E036
:1067C0000E94A5EDB501A4018EE496E00E94A5ED1E
:1067D0006C964FAD6C97A0965FADA097A4966FADE9
:1067E000A497E0967FADE09787E496E00E94E18D64
:1067F000E4964FADE497A8965FADA897AC966FADC1
:10680000AC97E8967FADE89780E496E00E94E18D32
:1068100069964EAD5FAD6997433051050CF4AEC03B
:10682000C501B4010E9465FB20E030E040E850E47F
:106830000E94C4FB6B017C016C962FAD6C97A096F7
:106840003FADA097A4964FADA497E0965FADE097BB
:10685000E4966FADE497A8967FADA897AC968FAD00
:10686000AC97E8969FADE8970E94D8FF2BED3FE0EC
:1068700049E450E40E94C4FB20E030E040E05FE3E4
:106880000E94C4FB9B01AC01C701B6010F94B50087
:106890006B017C01C301B2010E9465FB2FE632E16E
:1068A00043E85AE30E94C4FB2B013C01B701A60157
:1068B0008AE396E00E94E18DB301A20184E396E0B1
:1068C0000E94E18D2AE939E949E15FE3C701B60198
:1068D0000E94C4FB6B017C019B01AC010E94D9FFAB
:1068E000A30192010F94B500EC966CAF7DAF8EAF13
:1068F0009FAFEC97A3019201C701B6010E94C4FBB0
:1069000020E030E040E05EE30E94C4FBC458DF4F6B
:10691000688379838A839B83CC57D040E4E2F6E096
:1069200084913F015FEF651A750A882339F0082EBC
:10693000000C990B0E94CBA5F301F2CFB701A60181
:106940008EE196E00E94E18DEC964CAD5DAD6EADB2
:106950007FADEC9788E196E00E94E18DC458DF4F4F
:10696000488159816A817B81CC57D04082E196E091
:106970000E94E18D8AE090E00E94CBA527968CAD25
:106980009DADAEADBFAD2797880D991DAA1DBB1D4E
:10699000B595A795979587958093D31169968EADF8
:1069A0009FAD6997019669969FAF8EAF6997609684
:1069B0009FAD60976C969FAF6C972896AFAD289768
:1069C000A096AFAFA0972C96BFAD2C97A496BFAF63
:1069D000A4976496EFAD6497E096EFAFE0972396A7
:1069E0004CAC5DAC6EAC7FAC2397F1E0CE57DF4F83
:1069F000F883C258D0400C94CA2C01110C94C61EC6
:106A00000E9492500C94DD1E0E94BA6DBC2C60E076
:106A10008C2D0E94A7B60F3FBFEF1B0759F48C2D9A
:106A20000E9450B631E020E0892B09F030E0032FBE
:106A3000122F05C00130110561F000E010E08B2D30
:106A40000E9450B68017910709F421CC0E945796F6
:106A5000F6CF01E010E0F3CFC856DF4F0FB6F89441
:106A6000DEBF0FBECDBFDF91CF911F910F91FF9081
:106A7000EF90DF90CF90BF90AF909F908F907F90DE
:106A80006F905F904F903F902F9008954F925F923C
:106A90006F927F928F929F92AF92BF92CF92DF922E
:106AA000EF92FF920F931F93CF93DF93CDB7DEB793
:106AB000CD52D3400FB6F894DEBF0FBECDBFC0504D
:106AC000DD4F1882C050D34081E19DE00E940CB49C
:106AD000039714F40C94014BCE018F5F9D4F0E94DD
:106AE000B5B181110CC06FEE7CE0CE0101960E9421
:106AF0003976CE0101960E9434760C94014BCF5D1D
:106B0000DC4F1882C152D340C15EDC4F198218821B
:106B1000CF51D3401982BE016F5F7F4FCE018F5F8F
:106B20009D4F0E9434B11A821982BE016F5F7F4F60
:106B3000CE018F5F9D4F0E946BB109811A81BE010A
:106B40006F5D7C4FCE018F5F9D4F0E9434B1BE01BF
:106B5000615E7C4F0E946BB1C15EDC4FE880F980C2
:106B6000CF51D34061EE7CE0CE0101960E94397690
:106B70006FEC7CE0CE018F5F9E4F0E9439766AEC0D
:106B80007CE0CE018F5F9C4F0E943976CE018F5FF3
:106B90009C4F0E943476CE018F5F9E4F0E943476C8
:106BA000CE0101960E943476033124E0120709F4E5
:106BB000DDC308F07FC0003342E0140709F4D1C4FC
:106BC00008F057C0003182E0180709F476C430F5A8
:106BD0000115A2E01A0709F454C40130124011F063
:106BE0000C94F74A0E94B34B80E29BE09093FB1316
:106BF0008093FA130E94BA4B83E19BE09093FB13BE
:106C00008093FA130E94BA4B8FE09BE09093FB13A2
:106C10008093FA130E94BA4B0C94014B0032E2E0CD
:106C20001E0709F466C40132F2E01F0709F47DC4AF
:106C30000131124011F00C94F74A0E94B34B87EFD8
:106C40009AE09093FB138093FA130E94BA4B8AEE5A
:106C50009AE09093FB138093FA130E94BA4B86EE4E
:106C60009AE09093FB138093FA130E94BA4B0C9412
:106C7000014B013034E0130709F4FFC058F401332D
:106C800052E0150709F49BC40115144009F460C0D3
:106C90000C94F74A003194E0190709F4FBC1023162
:106CA000A4E01A0709F442C20230144011F00C9417
:106CB000F74A6FC10333E4E01E0711F40C94414519
:106CC00000F5013224E0120709F4CFC458F404316E
:106CD00044E0140709F460C30032144009F49DC471
:106CE0000C94F74A013384E0180711F40C94FD3E2C
:106CF00010F00C9404450033144009F43EC50C9484
:106D0000F74A0234B4E01B0711F40C94CA4768F444
:106D10000034F4E01F0711F40C946E450134144064
:106D200011F40C9462460C94F74A003534E01307D2
:106D300011F40C945949013544E0140711F40C94F2
:106D4000D34A0334144011F00C94F74A0C94D648FB
:106D500083E0E816F10409F472C030F4A1E0EA1609
:106D6000F10481F188F065C0E5E0EE16F10409F464
:106D700072C008F46AC009E9E016F10409F071C0B4
:106D80000E94CCCB0C94014B0E941FF580912C0FDC
:106D9000882351F080912B0F882331F061E08AE243
:106DA0000E9454A70C94014B8091000F9091010F09
:106DB000019711F086E501C08CE261E00E9454A7C2
:106DC0000C94014B80912C0F882361F080912B0F44
:106DD000882341F061E08AE20E9454A70E941FF5D7
:106DE0000C94014B8091000F9091010F019741F499
:106DF00061E08CE20E9454A70E941FF50C94014BA5
:106E00000E94C6BF80912C0F811108C061E086E509
:106E10000E9454A70E941FF50C94014B0E94C1E2EE
:106E200001970E941CE361E088E20E9454A70C9441
:106E3000014B61E088E10E9454A70C94014B61E092
:106E40008AE10E9454A70C94014B61E08CE10E94FE
:106E500054A70C94014B61E08EE30E9454A70C945C
:106E6000014B67EA7CE0CE0101960E943976CE01A3
:106E700001960E9434760C94014B11E0E116F10466
:106E8000C9F170F032E0E316F10409F453C049E9A6
:106E9000E416F10409F071C00E94CCCB0C94014BB4
:106EA0006CE97CE0CE0101960E943976CE01019614
:106EB0000E9434766AE973E08CEB91E10E940A76D5
:106EC0006AE973E082EC91E10E940A768FEF9FEF0E
:106ED0009093C9118093C8110E94D4AA0E94B34B09
:106EE0000E9430C20E940EA60E94D8BA0E94CCCB4B
:106EF0000C94014B60E97CE0CE0101960E9439764A
:106F0000CE0101960E9434766EE77CE0CE010196B8
:106F10000E943976CE0101960E94AAE3CE01019625
:106F20000E94347610922B0F80E09FE00E945A6DF1
:106F30000C94014B61E77CE0CE0101960E9439760A
:106F4000CE0101960E94347661E67CE0CE01019686
:106F50000E943976CE0101960E94AAE3CE010196E5
:106F60000E94347680912C0F882319F081E0809361
:106F70002B0F0E9464E20C94014B6EE47CE0CE0186
:106F800001960E943976CE0101960E9434760C94C7
:106F9000014B51E0E516F104B9F170F092E0E91609
:106FA000F10409F44FC0A9E9EA16F10409F066C03A
:106FB0000E94CCCB0C94014B63E47CE0CE010196A3
:106FC0000E943976CE0101960E9434766AE973E018
:106FD0008CEB91E10E940A766AE973E082EC91E120
:106FE0000E940A768FEF9FEF9093C9118093C8118A
:106FF0000E94B34B0E9430C20E940EA60E94D8BAD3
:107000000E94CCCB0C94014B67E37CE0CE0101964F
:107010000E943976CE0101960E94347668E27CE0C7
:10702000CE0101960E943976CE0101960E94AAE314
:10703000CE0101960E94347680E09FE00E945A6D56
:107040000C94014B6BE17CE0CE0101960E943976F5
:10705000CE0101960E9434766BE07CE0CE01019671
:107060000E943976CE0101960E94AAE3CE010196D4
:107070000E9434760E9464E20C94014B68EF7BE03E
:10708000CE0101960E943976CE0101960E94347697
:107090000C94014BB1E0EB16F10491F148F1F2E0F0
:1070A000EF16F10491F109E9E016F10499F567EEA4
:1070B0007BE0CE0101960E943976CE0101960E94B6
:1070C000347610927D0E0E94B34B83EE9BE090933A
:1070D000FB138093FA130E94BA4B1092FF13109285
:1070E000FE1380E00E9471690E94CCCB0C94014B8E
:1070F0000E9450CC61E08EE10E9454A70C94014B99
:1071000081E00E947FE30C94014B80E00E947FE3CA
:107110000C94014B60ED7BE0CE0101960E94397624
:10712000CE0101960E9434760C94014BE114F104D7
:1071300049F019E9E116F10409F048C00E94CCCBEE
:107140000C94014B63EC7BE0CE0101960E943976F2
:10715000CE0101960E94347660E775E0CE0101967B
:107160000E9415B103E71EE0D8015D968D919C91B8
:107170005E97CF5FDC4F99838883C150D3405B9685
:107180008D919C915C97CF5FDE4F99838883C1502E
:10719000D140BE016F5F7E4FCE0101960E945B5DC4
:1071A000BE016F5F7C4F0E945B5D0C5F1F4FBEE0B6
:1071B0000F371B07C9F661E0CE0101960E948AB322
:1071C00061E084E20E9454A70C94014B65EB7BE0E4
:1071D000CE0101960E943976CE0101960E94347646
:1071E000E1E0EE1AF108F3E0EF16F10460F063EA73
:1071F0007BE0CE0101960E943976CE0101960E9475
:1072000034760C94014B46E060E775E0CE018F5F69
:107210009E4F0E94E9B061E0CE018F5F9E4F0E94B9
:107220008AB3C050DF4F1882C050D140BE016F5F9B
:107230007E4FCE0101960E9475B281110EC069E8A1
:107240007BE0CE018F5F9C4F0E943976CE018F5F2D
:107250009C4F0E9434760C94014BC35FDC4F198223
:107260001882CD50D340C95FDC4F19821882C750B5
:10727000D34003E71EE0BE01635F7C4FCE01019661
:107280000E946BB1BE01695F7C4F0E946BB1C35F0E
:10729000DC4F88819981CD50D340D8015C969C9376
:1072A0008E935B97C95FDC4F88819981C750D3402B
:1072B0005E969C938E935D970C5F1F4FBEE00F37D9
:1072C0001B07C9F684E89BE09093FB138093FA13A5
:1072D0000E94BA4B6AE973E0CE018F5F9C4F0E9417
:1072E00041766DE77BE0CE018F5F9C4F0E94C575B4
:1072F000C701880F991F880F991F8C010D58114FD6
:10730000F801638D748DCE018F5F9C4F0E9467756D
:10731000CF5FDC4F88819981C150D3400E94C1A7C3
:1073200066E77BE0CE018F5F9C4F0E94C575D80158
:107330005D966D917C915E97CE018F5F9C4F0E9410
:107340006775CF5FDC4F88819981C150D3400E941F
:10735000C1A761E086E50E9454A70E941FF5CE01F7
:107360008F5F9C4F0E9434760C94014B6DE67BE05E
:10737000CE0101960E943976CE0101960E943476A4
:1073800088E69BE09093FB138093FA130E94BA4B1C
:107390000E94D8BA0C94014BB1E0EB16FB06C9F180
:1073A000B8F4F9E9EF16F10409F45BC0E11401E067
:1073B000F00609F44CC0EF2809F057C00E94BA6DDE
:1073C0000E94DDDA61E086E20E9454A70C94014B32
:1073D00013E0E11611E0F10681F128F1E11432E049
:1073E000F30609F042C08BE49BE09093FB1380937B
:1073F000FA130E94BA4B1092EB031092EA03109218
:10740000E9031092E8031092E7031092E6030C944C
:10741000014B81E69BE09093FB138093FA130E944B
:10742000BA4B0C94014B8AE59BE09093FB1380933D
:10743000FA130E94BA4B0C94014B83E59BE09093A6
:10744000FB138093FA130E94BA4B0C94014B8FE408
:107450009BE09093FB138093FA130E94BA4B0C9419
:10746000014B0E94CCCB0C94014B68E37BE0CE0136
:1074700001960E943976CE0101960E9434760C94D2
:10748000014B0E94B34B84E39BE09093FB138093EA
:10749000FA130E94BA4B88E29BE09093FB1380930F
:1074A000FA130E94BA4B84E29BE09093FB13809303
:1074B000FA130E94BA4B0C94014B0E94B34B8BE021
:1074C0009BE09093FB138093FA130E94BA4B8FEFCB
:1074D0009AE09093FB138093FA130E94BA4B8BEFC0
:1074E0009AE09093FB138093FA130E94BA4B0C948A
:1074F000014B0E94B34B82EE9AE09093FB13809372
:10750000FA130E94BA4B84ED9AE09093FB13809398
:10751000FA130E94BA4B80ED9AE09093FB1380938C
:10752000FA130E94BA4B0C94014B0E94B34B8CECA3
:107530009AE09093FB138093FA130E94BA4B8DEB61
:107540009AE09093FB138093FA130E94BA4B89EB55
:107550009AE09093FB138093FA130E94BA4B0C9419
:10756000014B20E030E044E353E460910214709159
:10757000031480910414909105140E945FFB87FF0F
:1075800002C00C94014B0E94B34B85EB9AE09093A0
:10759000FB138093FA130E94BA4B8AEA9AE0909305
:1075A000FB138093FA130E94BA4B86EA9AE09093F9
:1075B000FB138093FA130E94BA4B0C94014B20E00A
:1075C00030E044E353E4609102147091031480911D
:1075D0000414909105140E945FFB87FF02C00C9475
:1075E000014B0E94B34B82EA9AE09093FB13809385
:1075F000FA130E94BA4B86E99AE09093FB138093AA
:10760000FA130E94BA4B82E99AE09093FB1380939D
:10761000FA130E94BA4B0C94014B80912C0F8823D3
:1076200011F40C94014B0E94C1E2AC01069710F4D6
:107630000C94014B8091730E9091740EE114F1043F
:1076400021F0EA94EF2849F00CC09C012B5F3F4FDA
:107650002417350730F4C90104C08530910508F0BE
:1076600005970E941CE30C94014B80912C0F8823FA
:1076700011F40C94014B8091730E9091740E8E1541
:107680009F0510F40C94014B60E070E08E199F0987
:107690000E9480AA6BE37FE0CE0101960E944176B2
:1076A0004AE150E0BE016F5F7F4FCE018F5F9E4F7A
:1076B0000E940F5ECE0101960E943476CB5FDE4FB2
:1076C00088819981C550D140892B09F44FC06BE363
:1076D0007FE0CE0101960E944176BE016F5F7F4F31
:1076E0008CEB91E10E941F766AE973E082EC91E1F4
:1076F0000E940A768FEF9FEF9093C9118093C81173
:10770000CE0101960E9434766EE471E0CE010196BE
:107710000E9415B1BE016F5F7E4FCE0101960E949F
:10772000275D61E0CE0101960E948AB340E061E0EE
:107730008EE29FE00E945BBC80912C0F882319F0A1
:1077400081E080932B0F0E9464E20E94BA6D0E9438
:10775000DDDA61E08AE20E9454A70E941FF5CE01A3
:107760008F5F9E4F0E9434760C94014BCE018F5F49
:107770009E4F0E9434760C94014B52E0E516F104C2
:1077800009F437C170F4E114F10409F4D7C0EA94A4
:10779000EF2809F026C361E081E00E9469F40C94AF
:1077A000014BA4E0EA16F10409F41BC208F426C157
:1077B000E5E0EE16F10409F014C38091A203909164
:1077C000A303A091A403B091A5038093EA0E909324
:1077D000EB0EA093EC0EB093ED0E8091A60390916A
:1077E000A703A091A803B091A9038093EE0E9093F4
:1077F000EF0EA093F00EB093F10E8091AA0390913A
:10780000AB03A091AC03B091AD038093F20E9093C3
:10781000F30EA093F40EB093F50E8091AE03909109
:10782000AF03A091B003B091B1038093F60E909393
:10783000F70EA093F80EB093F90E0E944BCC60E5C2
:1078400073E0CE0101960E9415B120E030E040E2E5
:1078500051E46091F60E7091F70E8091F80E9091C0
:10786000F90E0E94C4FB0F942201C35FDC4F7983A1
:107870006883CD50D34020E030E040E251E4609195
:10788000F20E7091F30E8091F40E9091F50E0E941D
:10789000C4FB0F942201C95FDC4F79836883C75012
:1078A000D34020E030E040E251E46091EE0E709170
:1078B000EF0E8091F00E9091F10E0E94C4FB0F9498
:1078C0002201CF5FDC4F79836883C150D34020E031
:1078D00030E040E251E46091EA0E7091EB0E80914D
:1078E000EC0E9091ED0E0E94C4FB0F942201CF5F2D
:1078F000DE4F79836883C150D140BE016F5F7E4FF8
:10790000CE0101960E945B5DBE016F5F7C4F0E94BD
:107910005B5DBE01695F7C4F0E945B5DBE01635F82
:107920007C4F0E945B5D61E0CE0101960E948AB3AC
:1079300061E08EE40E9454A70C94014B60E273E076
:10794000CE0101960E9415B12091001430910114CE
:1079500044E6429FC001439F900D11246FEF70E0F9
:107960000F94B502C35FDC4F79836883CD50D34059
:107970008091FC139091FD13C95FDC4F998388833C
:10798000C750D3408091FE139091FF13CF5FDC4F1F
:1079900099838883C150D340809101029091020263
:1079A000CF5FDE4F99838883C150D140BE016F5FA6
:1079B0007E4FCE0101960E945B5DBE016F5F7C4FE2
:1079C0000E945B5DBE01695F7C4F0E945B5DBE01F2
:1079D000635F7C4F0E945B5D61E0CE0101960E9477
:1079E0008AB30E944BCC61E080E50E9454A70C94BE
:1079F000014B81E00E9464F00C94014B8091D6030E
:107A00009091D703A091D803B091D9038093B60E7B
:107A10009093B70EA093B80EB093B90E8091DA038D
:107A20009091DB03A091DC03B091DD038093BA0E4B
:107A30009093BB0EA093BC0EB093BD0E8091DE035D
:107A40009091DF03A091E003B091E1038093BE0E1B
:107A50009093BF0EA093C00EB093C10E8091E2032D
:107A60009091E303A091E403B091E5038093C20EEB
:107A70009093C30EA093C40EB093C50E8091D20311
:107A80009091D303A091D403B091D5038093C60EF7
:107A90009093C70EA093C80EB093C90E8091CE03E9
:107AA0009091CF03A091D003B091D1038093CA0EDF
:107AB0009093CB0EA093CC0EB093CD0E0E944BCCE6
:107AC00060E373E0CE0101960E9415B16091CA0E89
:107AD0007091CB0E8091CC0E9091CD0E0F9422011F
:107AE000C75EDC4F79836883C951D3406091C60E6D
:107AF0007091C70E8091C80E9091C90E0F9422010B
:107B0000CD5EDC4F79836883C351D3406091C20E50
:107B10007091C30E8091C40E9091C50E0F942201F6
:107B2000C35FDC4F79836883CD50D3406091BE0E34
:107B30007091BF0E8091C00E9091C10E0F942201E2
:107B4000C95FDC4F79836883C750D3406091BA0E18
:107B50007091BB0E8091BC0E9091BD0E0F942201CE
:107B6000CF5FDC4F79836883C150D3406091B60EFC
:107B70007091B70E8091B80E9091B90E0F942201BA
:107B8000CF5FDE4F79836883C150D140BE016F5F04
:107B90007E4FCE0101960E945B5DBE016F5F7C4F00
:107BA0000E945B5DBE01695F7C4F0E945B5DBE0110
:107BB000635F7C4F0E945B5DBE016D5E7C4F0E94E7
:107BC0005B5DBE01675E7C4F0E945B5D61E0CE0144
:107BD00001960E948AB361E08AE40E9454A70C9443
:107BE000014B8091BE039091BF03A091C003B0915F
:107BF000C1038093CE0E9093CF0EA093D00EB0937E
:107C0000D10E8091C2039091C303A091C403B0919F
:107C1000C5038093D20E9093D30EA093D40EB0934D
:107C2000D50E8091C6039091C703A091C803B0916F
:107C3000C9038093D60E9093D70EA093D80EB0931D
:107C4000D90E8091CA039091CB03A091CC03B0913F
:107C5000CD038093DA0E9093DB0EA093DC0EB093ED
:107C6000DD0E8091BA039091BB03A091BC03B0914B
:107C7000BD038093DE0E9093DF0EA093E00EB093D1
:107C8000E10E8091B6039091B703A091B803B09133
:107C9000B9038093E20E9093E30EA093E40EB093A9
:107CA000E50E8091B2039091B303A091B403B0911B
:107CB000B5038093E60E9093E70EA093E80EB09381
:107CC000E90E0E944BCC60E473E0CE0101960E9465
:107CD00015B16091E60E7091E70E8091E80E9091DB
:107CE000E90E0F942201C55EDC4F79836883CB5186
:107CF000D3406091E20E7091E30E8091E40E90917A
:107D0000E50E0F942201C75EDC4F79836883C95169
:107D1000D3406091DE0E7091DF0E8091E00E909165
:107D2000E10E0F942201CD5EDC4F79836883C3514D
:107D3000D3408091DA0E9091DB0EC35FDC4F9983C4
:107D40008883CD50D3408091D60E9091D70EC95FD5
:107D5000DC4F99838883C750D3408091D20E909195
:107D6000D30ECF5FDC4F99838883C150D34080917D
:107D7000CE0E9091CF0ECF5FDE4F99838883C15096
:107D8000D140BE016F5F7E4FCE0101960E945B5DC8
:107D9000BE016F5F7C4F0E945B5DBE01695F7C4FDF
:107DA0000E945B5DBE01635F7C4F0E945B5DBE0114
:107DB0006D5E7C4F0E945B5DBE01675E7C4F0E94E2
:107DC0005B5DBE01655E7C4F0E945B5D61E0CE0144
:107DD00001960E948AB361E08CE40E9454A70C943F
:107DE000014B6FE77AE0CE0101960E943976CE0111
:107DF00001960E9434760C94014BF2E0EF16F104E8
:107E000009F45BC140F4E114F10491F0EA94EF2825
:107E100009F4A6C0EEC524E0E216F10409F48DC30E
:107E200008F435C245E0E416F10409F405C5E1C5DE
:107E300044E060E273E0CE018F5F9E4F0E94E9B0A4
:107E400061E0CE018F5F9E4F0E948AB3C050DF4F2A
:107E50001882C050D140BE016F5F7E4FCE010196A7
:107E60000E9475B281110EC06EE57AE0CE018F5F7F
:107E70009C4F0E943976CE018F5F9C4F0E943476D2
:107E80000C94014BCD5EDC4F19821882C351D34054
:107E9000C35FDC4F19821882CD50D340C95FDC4FDD
:107EA00019821882C750D340CF5FDC4F19821882E5
:107EB000C150D340BE016D5E7C4FCE0101960E9441
:107EC0006BB1BE01635F7C4F0E946BB1BE01695F05
:107ED0007C4F0E946BB1BE016F5F7C4F0E946BB103
:107EE000CD5EDC4F88819981C351D34090930202CB
:107EF00080930102C35FDC4F88819981CD50D340CC
:107F00009093FF138093FE1380E00E947169C95F14
:107F1000DC4F88819981C750D3408739910514F08F
:107F200086E990E09093FD138093FC130E942669EC
:107F3000CF5FDC4F28813981C150D3404FEF429F42
:107F4000C001439F900D112464E670E00F94B502C8
:107F500070930114609300140E9421F40C94014B5F
:107F600043E060E173E0CE018F5F9E4F0E94E9B075
:107F700061E0CE018F5F9E4F0E948AB3C050DF4FF9
:107F80001882C050D140BE016F5F7E4FCE01019676
:107F90000E9475B281110EC06FE37AE0CE018F5F4F
:107FA0009C4F0E943976CE018F5F9C4F0E943476A1
:107FB0000C94014BC35FDC4F19821882CD50D34023
:107FC000C95FDC4F19821882C750D340CF5FDC4FA6
:107FD00019821882C150D340BE01635F7C4FCE012D
:107FE00001960E946BB1BE01695F7C4F0E946BB12C
:107FF000BE016F5F7C4F0E946BB1C35FDC4F688135
:108000007981CD50D34080E090E00E9463FB20E076
:1080100030E048EC52E40F94B50060932A19709355
:108020002B1980932C1990932D19C95FDC4F68810F
:108030007981C750D34080E090E00E9463FB20E04C
:1080400030E048EC52E40F94B5002CEA35EC47E2FE
:108050005EE30E94C4FB60932E1970932F198093E6
:10806000301990933119CF5FDC4F68817981C1500D
:10807000D34080E090E00E9463FB20E030E048ECD9
:1080800052E40F94B5002CEA35EC47E25EE30F941E
:10809000B50060933219709333198093341990931B
:1080A00035198AE39AE09093FB138093FA130E94A8
:1080B000BA4B0E9421F40C94014B44E060E073E061
:1080C000CE018F5F9E4F0E94E9B061E0CE018F5FCD
:1080D0009E4F0E948AB3C050DF4F1882C050D140DB
:1080E000BE016F5F7E4FCE0101960E9475B2811175
:1080F0000EC069E17AE0CE018F5F9C4F0E94397615
:10810000CE018F5F9C4F0E9434760C94014BCD5E64
:10811000DC4F19821882C351D340C35FDC4F1982F0
:108120001882CD50D340C95FDC4F19821882C750E6
:10813000D340CF5FDC4F19821882C150D340BE01BB
:108140006D5E7C4FCE0101960E946BB1BE01635FF4
:108150007C4F0E946BB1BE01695F7C4F0E946BB186
:10816000BE016F5F7C4F0E946BB1CD5EDC4F6881BA
:108170007981C351D34080E090E00E9463FB20E00E
:1081800030E040E251E40F94B5002B013C016093D4
:10819000A60E7093A70E8093A80E9093A90EC35FAE
:1081A000DC4F68817981CD50D34080E090E00E941F
:1081B00063FB20E030E040E251E40F94B5004B0156
:1081C0005C016093AA0E7093AB0E8093AC0E9093FB
:1081D000AD0EC95FDC4F68817981C750D34080E024
:1081E00090E00E9463FB20E030E040E251E40F9415
:1081F000B5006B017C016093AE0E7093AF0E80935F
:10820000B00E9093B10ECF5FDC4F68817981C15081
:10821000D34080E090E00E9463FB20E030E040E249
:1082200051E40F94B5006093B20E7093B30E809337
:10823000B40E9093B50E4092010D5092020D6092D3
:10824000030D7092040D8092050D9092060DA09280
:10825000070DB092080DC092090DD0920A0DE09260
:108260000B0DF0920C0D60930D0D70930E0D80931D
:108270000F0D9093100D84E19AE09093FB1380937F
:10828000FA130E94BA4B0E9421F40C94014B46E071
:1082900060E373E0CE018F5F9E4F0E94E9B061E022
:1082A000CE018F5F9E4F0E948AB3C050DF4F18826D
:1082B000C050D140BE016F5F7E4FCE0101960E943B
:1082C00075B281110EC060EF79E0CE018F5F9C4FD7
:1082D0000E943976CE018F5F9C4F0E9434760C94B9
:1082E000014BC55EDC4F19821882CB51D340C75E6B
:1082F000DC4F19821882C951D340CD5EDC4F198200
:108300001882C351D340C35FDC4F19821882CD500D
:10831000D340C95FDC4F19821882C750D340CF5F6A
:10832000DC4F19821882C150D340BE01655E7C4F7C
:10833000CE0101960E946BB1BE01675E7C4F0E9428
:108340006BB1BE016D5E7C4F0E946BB1BE01635F7D
:108350007C4F0E946BB1BE01695F7C4F0E946BB184
:10836000BE016F5F7C4F0E946BB1C55EDC4F6881C0
:108370007981CB51D34080E090E00E9463FB9B0168
:10838000AC016093B60E7093B70E8093B80E9093C5
:10839000B90EC75EDC4F68817981C951D34080E056
:1083A00090E0C65DDC4F2883CA52D340C55DDC4FE8
:1083B0003883CB52D340C45DDC4F4883CC52D3408A
:1083C000C35DDC4F5883CD52D3400E9463FB2B0129
:1083D0003C016093BA0E7093BB0E8093BC0E9093D9
:1083E000BD0ECD5EDC4F68817981C351D34080E002
:1083F00090E00E9463FB4B015C016093BE0E7093A2
:10840000BF0E8093C00E9093C10EC35FDC4F688196
:108410007981CD50D34080E090E00E9463FB6B01F6
:108420007C016093C20E7093C30E8093C40E909330
:10843000C50EC95FDC4F68817981C750D34080E0A9
:1084400090E00E9463FBCE5DDC4F688379838A8372
:108450009B83C252D3406093C60E7093C70E809325
:10846000C80E9093C90ECF5FDC4F68817981C150EF
:10847000D34080E090E00E9463FB6093CA0E70934B
:10848000CB0E8093CC0E9093CD0EC65DDC4F288131
:10849000CA52D340C55DDC4F3881CB52D340C45D56
:1084A000DC4F4881CC52D340C35DDC4F5881CD5264
:1084B000D3402093D6033093D7034093D8035093EF
:1084C000D9034092DA035092DB036092DC0370928E
:1084D000DD038092DE039092DF03A092E003B0926E
:1084E000E103C092E203D092E303E092E403F0924E
:1084F000E503CE5DDC4FE880F9800A811B81C25222
:10850000D340E092D203F092D3030093D4031093AC
:10851000D5036093CE037093CF038093D0039093E1
:10852000D1038BEE99E09093FB138093FA130E9492
:10853000BA4B0E9421F40C94014B47E060E473E0D5
:10854000CE018F5F9E4F0E94E9B061E0CE018F5F48
:108550009E4F0E948AB3C050DF4F1882C050D14056
:10856000BE016F5F7E4FCE0101960E9475B28111F0
:108570000EC063EC79E0CE018F5F9C4F0E9439768C
:10858000CE018F5F9C4F0E9434760C94014BC35EEA
:10859000DC4F19821882CD51D340C55EDC4F198261
:1085A0001882CB51D340C75EDC4F19821882C95163
:1085B000D340CD5EDC4F19821882C351D340C35FD4
:1085C000DC4F19821882CD50D340C95FDC4F19822D
:1085D0001882C750D340CF5FDC4F19821882C15038
:1085E000D340BE01635E7C4FCE0101960E946BB109
:1085F000BE01655E7C4F0E946BB1BE01675E7C4F21
:108600000E946BB1BE016D5E7C4F0E946BB1BE01DA
:10861000635F7C4F0E946BB1BE01695F7C4F0E941B
:108620006BB1BE016F5F7C4F0E946BB1C35EDC4FCC
:1086300088809980CD51D340A12CB12C8092CE0E50
:108640009092CF0EA092D00EB092D10EC55EDC4FAC
:10865000C880D980CB51D340E12CF12CC092D20EEE
:10866000D092D30EE092D40EF092D50EC75EDC4FBE
:1086700088819981C951D3409C0140E050E0CE5D92
:10868000DC4F288339834A835B83C252D3402093D3
:10869000D60E3093D70E4093D80E5093D90ECD5EA0
:1086A000DC4F88819981C351D3409C0140E050E068
:1086B000CA5DDC4F288339834A835B83C652D3402B
:1086C0002093DA0E3093DB0E4093DC0E5093DD0ED8
:1086D000C35FDC4F68817981CD50D34080E090E06A
:1086E0000E9463FB9B01AC016093DE0E7093DF0E72
:1086F0008093E00E9093E10EC95FDC4F6881798131
:10870000C750D34080E090E0C65DDC4F2883CA525A
:10871000D340C55DDC4F3883CB52D340C45DDC4FC2
:108720004883CC52D340C35DDC4F5883CD52D340F5
:108730000E9463FB2B013C016093E20E7093E30EF9
:108740008093E40E9093E50ECF5FDC4F68817981D2
:10875000C150D34080E090E00E9463FB6093E60E3E
:108760007093E70E8093E80E9093E90E8092BE031B
:108770009092BF03A092C003B092C103C092C20303
:10878000D092C303E092C403F092C503CE5DDC4FE8
:10879000E880F9800A811B81C252D340E092C6036F
:1087A000F092C7030093C8031093C903CA5DDC4F5E
:1087B000E880F9800A811B81C652D340E092CA0347
:1087C000F092CB030093CC031093CD03C65DDC4F36
:1087D0002881CA52D340C55DDC4F3881CB52D3408B
:1087E000C45DDC4F4881CC52D340C35DDC4F58811F
:1087F000CD52D3402093BA033093BB034093BC03C4
:108800005093BD034092B6035092B7036092B803F1
:108810007092B9036093B2037093B3038093B4036F
:108820009093B5038EEB99E09093FB138093FA132A
:10883000A1D70E9421F4E5C644E060E573E0CE01D3
:108840008F5F9E4F0E94E9B061E0CE018F5F9E4F27
:108850000E948AB3C050DF4F1882C050D140BE0181
:108860006F5F7E4FCE0101960E9475B281110DC0DF
:1088700066E979E0CE018F5F9C4F0E943976CE0188
:108880008F5F9C4F0E943476BCC6CD5EDC4F198250
:108890001882C351D340C35FDC4F19821882CD5078
:1088A000D340C95FDC4F19821882C750D340CF5FD5
:1088B000DC4F19821882C150D340BE016D5E7C4FDF
:1088C000CE0101960E946BB1BE01635F7C4F0E9496
:1088D0006BB1BE01695F7C4F0E946BB1BE016F5FDF
:1088E0007C4F0E946BB1CD5EDC4F88819981C35172
:1088F000D3400AE010E0B8010F94A10280E090E0BC
:108900000E9463FB2B013C016093EA0E7093EB0E17
:108910008093EC0E9093ED0EC35FDC4F88819981BC
:10892000CD50D340B8010F94A10280E090E00E94A6
:1089300063FB4B015C016093EE0E7093EF0E80932E
:10894000F00E9093F10EC95FDC4F88819981C7507A
:10895000D340B8010F94A10280E090E00E9463FB35
:108960006B017C016093F20E7093F30E8093F40E12
:108970009093F50ECF5FDC4F88819981C150D34031
:10898000B8010F94A10280E090E00E9463FB609325
:10899000F60E7093F70E8093F80E9093F90E4092B6
:1089A000A2035092A3036092A4037092A503809245
:1089B000A6039092A703A092A803B092A903C09225
:1089C000AA03D092AB03E092AC03F092AD036093A4
:1089D000AE037093AF038093B0039093B10381E92A
:1089E00099E09093FB138093FA13C4D60E9421F46C
:1089F00008C66EE779E0CE0101960E943976CE0175
:108A000001960E943476FDC5EA94EF28B9F580916D
:108A10009A0E90919B0EA0919C0EB0919D0E80930A
:108A20002A1990932B19A0932C19B0932D1980918A
:108A30009E0E90919F0EA091A00EB091A10E8093DA
:108A40002E1990932F19A0933019B093311980915A
:108A5000A20E9091A30EA091A40EB091A50E8093AA
:108A6000321990933319A0933419B093351989E7CB
:108A700099E09093FB138093FA137CD60E94CCCBA1
:108A8000C0C511E0E116F10469F038F039E9E316E8
:108A9000F104C9F40E94CCCBB4C561E082E40E9429
:108AA00054A7AFC584E799E09093FB138093FA1322
:108AB00061D68FE699E09093FB138093FA135AD610
:108AC0000E94CCCB9EC56CE579E0CE0101960E9458
:108AD0003976CE0101960E94347693C543E0E416C0
:108AE000F10409F484C068F581E0E816F10409F4A2
:108AF0003EC008F05CC061E08EE20E9454A7109274
:108B0000EB031092EA031092E9031092E80310922B
:108B1000E7031092E60388E599E09093FB138093B6
:108B2000FA1328D684E599E09093FB138093FA1307
:108B300021D681E080937D0E84EF91E00E9446CAA9
:108B400060C5A5E0EA16F10409F491C008F46FC00D
:108B5000E9E9EE16F10409F0AAC08EE298E09093DC
:108B6000FB138093FA1306D60E94CCCB4AC567E468
:108B700079E0CE0101960E943976CE0101960E94DD
:108B800034768AE399E09093FB138093FA13F2D53D
:108B900089E299E09093FB138093FA13EBD58DE172
:108BA00099E09093FB138093FA13E4D52AC560E112
:108BB00079E0CE0101960E943976CE0101960E949D
:108BC000347683E099E09093FB138093FA13D2D527
:108BD00080EF98E09093FB138093FA13CBD584EE4B
:108BE00098E09093FB138093FA13C4D50AC567ED00
:108BF00078E0CE0101960E943976CE0101960E945E
:108C000034768AEC98E09093FB138093FA13B2D5F4
:108C100088EB98E09093FB138093FA13ABD58CEA22
:108C200098E09093FB138093FA13A4D5EAC46FE9FC
:108C300078E0CE0101960E943976CE0101960E941D
:108C4000347682E998E09093FB138093FA1392D5DF
:108C500080E898E09093FB138093FA138BD584E718
:108C600098E09093FB138093FA1384D5CAC467E607
:108C700078E0CE0101960E943976CE0101960E94DD
:108C800034768AE598E09093FB138093FA1372D5BB
:108C900087E498E09093FB138093FA136BD58BE3F2
:108CA00098E09093FB138093FA1364D5AAC46BE108
:108CB00078E0CE0101960E943976CE0101960E949D
:108CC00034769FC4F1E0EF16F10409F44EC050F180
:108CD00012E0E116F10409F46EC029E9E216F1048C
:108CE00009F04DC110927D0E1092FF131092FE13E9
:108CF00080E00E9471691092FD131092FC130E9493
:108D000026698DEB97E09093FB138093FA1332D58D
:108D100086EB97E09093FB138093FA132BD50E9478
:108D2000CCCB6FC40E9450CC61E275E0CE010196BD
:108D30000E9415B188EC90E0CF5FDE4F9983888365
:108D4000C150D140BE016F5F7E4FCE0101960E949F
:108D50005B5D61E0CE0101960E948AB30E944BCC1C
:108D600061E082E30E9454A74CC40E94F8CB0097B4
:108D700009F447C49093FF138093FE1380E00E9490
:108D8000716984E080937D0E84EF91E00E9446CA71
:108D900087E198E09093FB138093FA13EBD480E182
:108DA00098E09093FB138093FA13E4D460E084E39B
:108DB0000E9454A726C441E061E275E0CE018F5FB6
:108DC0009E4F0E94E9B061E0CE018F5F9E4F0E94EE
:108DD0008AB3C050DF4F1882C050D140BE016F5FD0
:108DE0007E4FCE0101960E9475B281110DC065EFD4
:108DF00077E0CE018F5F9C4F0E943976CE018F5F66
:108E00009C4F0E943476FDC3C75EDC4F19821882E6
:108E1000C951D340BE01675E7C4FCE0101960E94CE
:108E20006BB1C75EDC4F88819981C951D3406AE03C
:108E300070E00F94A1028B01C75EDC4F79836883D9
:108E4000C951D3408091010D9091020DA091030D65
:108E5000B091040D8093A60E9093A70EA093A80E38
:108E6000B093A90E8091050D9091060DA091070D6C
:108E7000B091080D8093AA0E9093AB0EA093AC0E08
:108E8000B093AD0E8091090D90910A0DA0910B0D3C
:108E9000B0910C0D8093AE0E9093AF0EA093B00ED8
:108EA000B093B10EC090FC0ED090FD0EE090FE0E7F
:108EB000F090FF0E20910D0D30910E0D40910F0D91
:108EC0005091100DC701B6010E94C4FB4B015C011B
:108ED00020E030E040EA51E4C701B6010E94D9FF2A
:108EE0006B017C01B80180E090E00E9463FB9B0174
:108EF000AC01C701B6010E94D8FF9B01AC01C501BE
:108F0000B4010F94B5006093B20E7093B30E8093CA
:108F1000B40E9093B50E6CEE77E0CE018D5E9C4F53
:108F20000E9439766EED77E0CE01835F9C4F0E9400
:108F3000397660ED77E0CE01895F9C4F0E943976EB
:108F400061EC77E0CE018F5F9C4F0E943976CE01B5
:108F50008F5F9C4F0E943476CE01895F9C4F0E94A8
:108F60003476CE01835F9C4F0E943476CE018D5EB5
:108F70009C4F0E94347680E00E9464F042C363EA12
:108F800077E0CE0101960E943976CE0101960E94CB
:108F9000347637C332E0E316F10409F43FC049E9FF
:108FA000E416F10409F4F4C0EF2809F0F4C061E21A
:108FB00075E0CE0101960E9415B188EC90E0C95F82
:108FC000DC4F99838883C750D340CF5FDC4F9983B0
:108FD0008883C150D340CF5FDE4F99838883C150CF
:108FE000D140BE016F5F7E4FCE0101960E945B5D56
:108FF000BE016F5F7C4F0E945B5DBE01695F7C4F6D
:109000000E945B5D61E0CE0101960E948AB30E94DE
:109010004BCC61E088E30E9454A7F3C243E061E2D5
:1090200075E0CE018F5F9E4F0E94E9B061E0CE01F6
:109030008F5F9E4F0E948AB3C050DF4F1882C0508E
:10904000D140BE016F5F7E4FCE0101960E9475B286
:1090500081110DC068E877E0CE018F5F9C4F0E94C0
:109060003976CE018F5F9C4F0E943476CAC2C35FAF
:10907000DC4F19821882CD50D340C95FDC4F198272
:109080001882C750D340CF5FDC4F19821882C1507D
:10909000D340BE01635F7C4FCE0101960E946BB14D
:1090A000BE01695F7C4F0E946BB1BE016F5F7C4F58
:1090B0000E946BB1C35FDC4F68817981CD50D34092
:1090C00080E090E00E9463FB9B01AC016091010D88
:1090D0007091020D8091030D9091040D0E94CFF3C9
:1090E0006093A60E7093A70E8093A80E9093A90E7E
:1090F000C95FDC4F68817981C750D34080E090E040
:109100000E9463FB9B01AC016091050D7091060DFF
:109110008091070D9091080D0E94CFF36093AA0EE5
:109120007093AB0E8093AC0E9093AD0ECF5FDC4F7F
:1091300068817981C150D34080E090E00E9463FB58
:109140009B01AC016091090D70910A0D80910B0D8E
:1091500090910C0D0E94CFF36093AE0E7093AF0E02
:109160008093B00E9093B10E80910D0D90910E0DE5
:10917000A0910F0DB091100D8093B20E9093B30E8D
:10918000A093B40EB093B50E80E00E9464F039C293
:109190000E94CCCB36C265E777E0CE0101960E94F3
:1091A0003976CE0101960E9434762BC251E0E51645
:1091B000F10409F442C040F099E9E916F10409F01C
:1091C0006DC00E94CCCB1DC280912A1990912B19A1
:1091D000A0912C19B0912D1980939A0E90939B0E0B
:1091E000A0939C0EB0939D0E80912E1990912F19F3
:1091F000A0913019B091311980939E0E90939F0EDB
:10920000A093A00EB093A10E8091321990913319C2
:10921000A0913419B09135198093A20E9093A30EAA
:10922000A093A40EB093A50E0E9450CC0E944BCCEC
:1092300061E08AE30E9454A7E4C10E94F8CB8C014C
:10924000892B09F4DEC18BE697E09093FB138093A2
:10925000FA1390D26AE973E0CE0101960E9441763A
:1092600064E677E0CE0101960E9475EDB801CE016B
:1092700001960E9467756BE577E0CE0101960E942A
:1092800075ED89819A810E94C1A761E08CE30E94FB
:1092900054A7CE0101960E943476B3C168E477E00A
:1092A000CE0101960E943976CE0101960E94347655
:1092B000A8C1E114F10441F0A9E9EA16F10409F0AA
:1092C00067C10E94CCCB9DC100910E0F10910F0F72
:1092D000A090100FB090110F2091120F3091130F2A
:1092E0004091140F5091150FCE5DDC4F28833983C8
:1092F0004A835B83C252D3404090160F5090170FA1
:109300006090180F7090190FC0901A0FD0901B0F1B
:10931000E0901C0FF0901D0F60E475E0CE01019607
:109320000E9415B1CF5FDC4FB982A882C150D340F3
:10933000CF5FDE4F19830883C150D140BE016F5FFC
:109340007E4FCE0101960E945B5DBE016F5F7C4F38
:109350000E945B5D61E0CE0101960E948AB38AE5BE
:10936000A82EA98295EAB92EBA8201E00B8314E0F7
:10937000C050DF4F1883C050D14082E495E0CF5FEA
:10938000DE4F99838883C150D140BE016F5F7E4F0D
:10939000CE0101960E945B5DCE5DDC4F2881398154
:1093A0004A815B81C252D340C35FDC4F288339833B
:1093B0004A835B83CD50D3406AE973E0CE018F5F6F
:1093C0009C4F0E944176BE016F5F7E4FCE01835F4E
:1093D0009C4F28D540E150E0BE016F5F7E4FCE012B
:1093E0008F5F9C4F0E94CB5DBE016F5F7C4FCE01B3
:1093F00001960E94275DCE018F5F9C4F0E943476BC
:1094000061E0CE0101960E948AB3A982BA820B83E1
:10941000C050DF4F1883C050D1408DE495E0CF5F3E
:10942000DE4F99838883C150D140BE016F5F7E4F6C
:10943000CE0101960E945B5DC95FDC4F4882598274
:109440006A827B82C750D3406AE973E0CE018F5FA6
:109450009C4F0E944176BE016F5F7E4FCE01895FB7
:109460009C4FE0D440E150E0BE016F5F7E4FCE01E3
:109470008F5F9C4F0E94CB5DBE016F5F7C4FCE0122
:1094800001960E94275DCE018F5F9C4F0E9434762B
:1094900061E0CE0101960E948AB36AE973E0CE01D1
:1094A0008F5F9C4F0E9441766BEE72E0CE018F5F22
:1094B0009E4F0E94417620E030E04AE754E4C70125
:1094C000B6010F94B5000F942201CE018F5F9C4F1F
:1094D0000E946775BE016F5F7E4FCE018F5F9C4F0C
:1094E0000E94967520E030E048EC52E4C701B601D6
:1094F0000F94B5000F942201CB016AE070E00F9445
:10950000A102BC01CE018F5F9C4F0E946775CE0106
:109510008F5F9E4F0E943476A982BA820B83C0501F
:10952000DF4F1883C050D14088E595E0CF5FDE4F14
:1095300099838883C150D140BE016F5F7E4FCE01B9
:1095400001960E945B5D40E150E0BE016F5F7C4F81
:10955000CE018F5F9E4F0E940F5EBE016F5F7E4FF8
:10956000CE0101960E94275DCE018F5F9E4F0E9423
:10957000347661E0CE0101960E948AB3CE018F5FFE
:109580009C4F0E94347661E084E40E9454A739C065
:1095900065E377E0CE0101960E943976CE0101960F
:1095A0000E9434762EC031E0E316F10439F049E927
:1095B000E416F10441F40E94CCCB23C060E086E4C1
:1095C0000E9454A71EC0F092FB0EE092FA0E0E9479
:1095D0005CCA8091FA0E9091FB0E8031924011F09E
:1095E00084E501C086E461E00E9454A70AC06AEBEA
:1095F0007CE0CE0101960E943976CE0101960E9450
:109600003476C35DDC4F0FB6F894DEBF0FBECDBF1E
:10961000DF91CF911F910F91FF90EF90DF90CF904E
:10962000BF90AF909F908F907F906F905F904F9082
:1096300008959091C804E92FF0E0E95EF54F80832A
:109640009F5F943018F49093C80402C01092C8042D
:109650008091B80B8F5F8093B80B0895089580E0D8
:1096600090E00895CF92DF92EF92FF92CF93DF9335
:109670006B017C01EA012FE632E143E85AEB0F94DB
:10968000FF0187FD23C022E430E048E453E4C70132
:10969000B6010E945FFB1816CCF0C880D980EA8022
:1096A000FB802FE632E143E85AEBC701B6010F9485
:1096B000FF0187FD0BC0C1E022E430E048E453E441
:1096C000C701B6010E945FFB18160CF4C0E08C2F96
:1096D000DF91CF91FF90EF90DF90CF900895CF92E0
:1096E000DF92EF92FF92C0903C02D0903D02E0905A
:1096F0003E02F0903F02FC0180819181A281B38102
:1097000080933C0290933D02A0933E02B0933F02AF
:109710000E94F6DAC0923C02D0923D02E0923E02F4
:10972000F0923F02FF90EF90DF90CF900895CF939B
:10973000FC0180818B33A1F08091B80B843080F4E0
:10974000C62FBF018091C80420E6829FC00111246A
:10975000895C954F0F940C048C2F6BDF81E001C066
:1097600080E0CF9108958091C8048093B70B109248
:10977000B80B0895DF92EF92FF920F931F93CF9350
:10978000DF93CDB7DEB76E970FB6F894DEBF0FBE8E
:10979000CDBF6091FA137091FB136115710549F10A
:1097A0004DE150E0CE0101967C010E94ACFA1E8E84
:1097B000F7018F010E191F09D190DD2019F09AE0F1
:1097C000D912F7CFF701E00FF11F1082C7010E94F5
:1097D000C1A7882371F0DD20A9F00F5F1F4F809192
:1097E000FA139091FB13080F191F1093FB130093AA
:1097F000FA1381E02091FA133091FB13232B29F403
:1098000080E003C000E010E0F0CF6E960FB6F89451
:10981000DEBF0FBECDBFDF91CF911F910F91FF90A3
:10982000EF90DF9008954F925F926F927F929F9298
:10983000AF92BF92CF92DF92EF92FF920F931F935E
:10984000CF93DF931F92CDB7DEB794DF811182C231
:109850008091B80B843038F48EEA9DE00E94EAB320
:10986000AC0197FF54C180912B0F882309F472C279
:109870008091B80B811102C01092CA04EE24E394C7
:109880004091A7115091A8116091A9117091AA114E
:109890008091A3119091A411A091A511B091A6114E
:1098A000481759076A077B0708F4E12C00E010E02D
:1098B000BB24B39480E6A82E9AE5C92E91E1D92E57
:1098C0002DE8922E8091B80B843008F043C2E1104D
:1098D00041C28091CA0481113DC28091FE109091D5
:1098E000FF10A0910011B09101118093A7119093E6
:1098F000A811A093A911B093AA1141E050E0BE01B4
:109900006F5F7F4F86EF90E10E941463019719F417
:10991000898190E002C08FEF9FEFF82EEE24E39450
:109920004090A7115090A8116090A9117090AA11B1
:109930004091A3115091A4116091A5117091A611AD
:109940004416550666067706C8F4E12C8F3FFFEFF4
:109950009F0709F484C02AE0821709F4ABC08DE0A8
:10996000F81609F4A7C093E2F91619F0EAE3FE121B
:10997000B4C08091C9048111B0C091C00E94BA6D79
:1099800086EF90E10E94D16680911111882359F1F0
:10999000815080931111989EC001112441E061E033
:1099A0008A5E9E4E0E945BBCE091111124E0E29F12
:1099B000F0011124EE5EFE4E40815181628173817F
:1099C0004093A7115093A8116093A9117093AA1105
:1099D00086EF90E10E94EE6080912C0F8823D9F0F1
:1099E000B0922B0F18C010922B0F81E090E0909353
:1099F0009F0980939E090E940EA680E09FE00E942E
:109A00002D6D6D3371058105910528F0D092FB1302
:109A1000C092FA13AFDE80912B0F811144C0EDE6A6
:109A2000F1E184913F019FEF691A790A882339F0A7
:109A3000082E000C990B0E94CBA5F301F2CF1092D7
:109A4000AF1180912C0F882319F00E94AEBE27C061
:109A50000E94C6BF80912C0F8111F7CF20C0ECE58A
:109A6000F9E284913F012FEF621A720A882339F0DC
:109A7000082E000C990B0E94CBA5F301F2CFEEE566
:109A8000F1E184913F019FEF691A790A882339F047
:109A9000082E000C990B0E94CBA5F301F2CFE3E254
:109AA000FE1208C005C023E2F2124FC100E010E030
:109AB000B092CA041092C9040115110509F402CF2D
:109AC0008091C804A89E000D111D1124F801E95CC5
:109AD000F54F108280E0ADDD3AC10F35110508F079
:109AE000F1CEFBE3FF1202C0B092C9048091C90419
:109AF0008111E8CE8091C804F801A89EE00DF11D07
:109B00001124E95CF54FF0820F5F1F4FDBCE982FD9
:109B100020910A1430910B148A3019F09D3009F00D
:109B2000E0C01092C7042115310509F491CEF90166
:109B3000E959FB4F108210920B1410920A1427E679
:109B400034E08901F90180812F5F3F4F8032C9F3F2
:109B500078018E3409F07BC00115110509F477C036
:109B600065E571E1C8010E94BBFADD24D394892B1D
:109B700011F4D12C09C06EE470E0C80104960F9472
:109B8000F803009709F08C014AE050E060E070E0D3
:109B9000C80101960E9420F86093630470936404E6
:109BA000809365049093660400910C1410910D1439
:109BB00020910E1430910F140F5F1F4F2F4F3F4F06
:109BC000601771078207930729F0D11003C08FE453
:109BD00090E127C06AE270E0C7010F9430049C0155
:109BE000009711F1982F9E1910E0992339F09150A8
:109BF000F701E90FF11D80811827F7CF4AE050E007
:109C000060E070E0C90101960E9420F8012F10E089
:109C100020E030E0601771078207930741F086E388
:109C200091E10E946CC71FCE8CE091E1FACF809148
:109C3000630490916404A0916504B09166048093DC
:109C40000C1490930D14A0930E14B0930F148091E4
:109C50000C02811124C067E470E0C7010F94F8037F
:109C60000097E9F04AE050E060E070E001960E9461
:109C700020F86430710598F4E5E9F0E184918F01F2
:109C80000F5F1F4F882339F0082E000C990B0E949C
:109C9000CBA5F801F3CF8BE890E10E9425C16AE3E0
:109CA00073E0C7010F940304892B11F41092000292
:109CB0006FE373E0C7010F940304892B21F482E85A
:109CC00090E10E94209664E473E0C7010F940304BE
:109CD000892B11F40E9430C261E087E694E027DD11
:109CE000B7CD2F3531050CF0B3CD9C35D1F48EEACC
:109CF0009DE00E94EAB397FDABCD2091C7042111EE
:109D0000A7CD20910A1430910B14A9014F5F5F4F2A
:109D100050930B1440930A14F901E959FB4F8083C7
:109D200097CD9B3319F481E08093C7048091C704D9
:109D300081118ECDC901019690930B1480930A1462
:109D4000F901E959FB4F408383CD1092C90400E02B
:109D500010E0B8CD0F90DF91CF911F910F91FF9040
:109D6000EF90DF90CF90BF90AF909F907F906F90DB
:109D70005F904F9008950F931F93CF93DF93CDB7CC
:109D8000DEB72C970FB6F894DEBF0FBECDBFE1EF64
:109D9000FCE080859185A285B385448155816681EB
:109DA0007781008111812281338109831A832B837A
:109DB0003C834D835E836F83788789879A87AB87DF
:109DC000BC87AE01475F5F4FBE016B5F7F4FCE0127
:109DD00001960E9462912DEF3CE0AE01475F5F4F1C
:109DE000BE016B5F7F4FCE0101960E94D78E2C96ED
:109DF0000FB6F894DEBF0FBECDBFDF91CF911F919C
:109E00000F9108958091610490916204009731F060
:109E10004AE050E060E070E00C9448F960E070E0E7
:109E2000CB0108954F925F926F927F92AF92BF9253
:109E3000CF92DF92EF92FF92CF93DF93EB01FC0181
:109E400060817181828193812CE3C22ED12CE12C1F
:109E5000F12CA70196010E947BFFB62EA72ECA0106
:109E6000B901A70196010E947BFF6B017C01CA0129
:109E7000B90128E130E040E050E00E947BFF2B0177
:109E80003C01C9016DE671E00F94A10261157105F5
:109E9000D9F0AF92BF92DF92CF925F924F929F9391
:109EA0008F937F936F938BE390E19F938F93DF93D7
:109EB000CF930E94F8FA8DB79EB70E960FB6F8941E
:109EC0009EBF0FBE8DBF61C00097C9F0AF92BF9219
:109ED000DF92CF925F924F929F938F938BE290E1AC
:109EE0009F938F93DF93CF930E94F8FAEDB7FEB75D
:109EF0003C960FB6F894FEBF0FBEEDBF46C04114AE
:109F0000510461047104B9F0AF92BF92DF92CF9215
:109F10005F924F928FE190E19F938F93DF93CF9366
:109F20000E94F8FA8DB79EB70A960FB6F8949EBFB6
:109F30000FBE8DBF2AC0C114D104E104F104A9F001
:109F4000AF92BF92DF92CF9287E190E19F938F9380
:109F5000DF93CF930E94F8FAEDB7FEB738960FB6AD
:109F6000F894FEBF0FBEEDBF10C0AF92BF9283E169
:109F700090E19F938F93DF93CF930E94F8FA0F9015
:109F80000F900F900F900F900F90DF91CF91FF9057
:109F9000EF90DF90CF90BF90AF907F906F905F90E9
:109FA0004F900895FC01238121110C94D1660895EE
:109FB00020916F0E9091700E81E0291301C080E016
:109FC0000895AC01485F5F4FBC016C5F7F4F0C94FC
:109FD00062910E94E2B760938B0C70938C0C80931B
:109FE0008D0C90938E0C0895809161049091620481
:109FF000009731F04AE050E060E070E00C9420F807
:10A0000060E070E0CB010895EFDF97FD0AC0ECDF60
:10A010006F3F71058105910509F02CF4E5DF862F6E
:10A02000089580E008958FEF0895809161049091E4
:10A030006204892B31F0E8DF91E0811103C090E0E8
:10A0400001C091E0892F08950F931F93CF938091C2
:10A050006104909162040097F1F0FC018F01C191BD
:10A060002C2F2F7D89F0C53411F0C536B9F7F801D2
:10A07000108260E070E00E94B9F6F801C083562FAC
:10A08000472F382F292F0BC060E070E0CF911F9130
:10A090000F910C94B9F650E040E030E020E0652FDD
:10A0A000742F832F922FCF911F910F910895815478
:10A0B0008A3150F5482F50E0FA0193E0F595E79585
:10A0C0009A95E1F7E851FB4E208130E08770B901A5
:10A0D00002C0759567958A95E2F760FF15C0FA0191
:10A0E000E253FB4E2081222339F08091890C90911C
:10A0F0008A0C820F911D02C080E090E09093620470
:10A100008093610481E0089580E00895D0DF882382
:10A1100041F081E02091610430916204232B09F425
:10A1200080E0089580E1E1EFFCE0A6E4B4E1019075
:10A130000D928A95E1F708952F923F924F925F9288
:10A140006F927F928F929F92AF92BF92CF92DF9247
:10A15000EF92FF920F931F93CF93DF9300D01F9244
:10A160001F92CDB7DEB77C018B016A011901809087
:10A17000F10C9090F20CA090F30CB090F40CA501AF
:10A180009401FC0160817181828193810E945FFB57
:10A19000F1E0FD83811112C02091F50C3091F60C95
:10A1A0004091F70C5091F80CF80160817181828127
:10A1B00093810E945FFB811101C01D82F6014080E6
:10A1C000518062807380209103023091040240919B
:10A1D000050250910602C301B2010E945FFB882371
:10A1E00009F455C0409203025092040260920502A5
:10A1F0007092060220E030E040E450E46091DE031B
:10A200007091DF038091E0039091E1030F94B5001A
:10A2100069837A838B839C8380924614909247143F
:10A22000A0924814B09249148091F50C9091F60CCC
:10A23000A091F70CB091F80C80934A1490934B14B2
:10A24000A0934C14B0934D14F60180819181A281AA
:10A25000B38180934E1490934F14A0935014B093F5
:10A2600051148091FD0C9091FE0CA091FF0CB091C7
:10A27000000D8093521490935314A0935414B093F0
:10A280005514CE0101962BDA0E94BA6D4BDFFD8189
:10A29000FF2311F14090D6035090D7036090D8036C
:10A2A0007090D9038090DA039090DB03A090DC03D8
:10A2B000B090DD03A5019401C301B2010E945FFBD0
:10A2C00020E030E040E251E487FF03C0C301B20167
:10A2D0000FC0C501B4010CC020E030E040EC5FE3EA
:10A2E0006091E2037091E3038091E4039091E503B0
:10A2F0000F94B50069837A838B839C8320919C03A0
:10A30000222351F0AB01BC0186E09DE00E94E18D6B
:10A310008AE090E00E94CBA5F70180819181A28123
:10A32000B3818093461490934714A0934814B0933C
:10A330004914F80180819181A281B38180934A14EC
:10A3400090934B14A0934C14B0934D14F1012081C1
:10A3500031814281538160915214709153148091E4
:10A360005414909155140E94D9FF60935214709325
:10A3700053148093541490935514CE010196AFD981
:10A380000E94BA6DCFDE0F900F900F900F900F903C
:10A39000DF91CF911F910F91FF90EF90DF90CF90C1
:10A3A000BF90AF909F908F907F906F905F904F90F5
:10A3B0003F902F90089580E1E6E4F4E1A1EFBCE046
:10A3C00001900D928A95E1F708952F923F924F9256
:10A3D0005F926F927F928F929F92AF92BF92CF9235
:10A3E000DF92EF92FF920F931F93CF93DF93CDB73E
:10A3F000DEB7C25AD1090FB6F894DEBF0FBECDBF8B
:10A40000E6EEFFE084918F010F5F1F4F882339F044
:10A41000082E000C990B0E94CBA5F801F3CF0E94E7
:10A4200054CE81110C940D5D80E090E0A0E8BFE374
:10A4300080933E1490933F14A0934014B093411422
:10A440008093421490934314A0934414B093451402
:10A450008DEC9CECACE4BEE380933A1490933B14F7
:10A46000A0933C14B0933D1480E090E0A0E2B1E4EE
:10A4700080935D0490935E04A0935F04B0936004A6
:10A480008CE390E090935C0480935B048DEC90E00F
:10A4900090935A0480935904109258048FE436DE46
:10A4A000882311F0D1DD04C06AE979E989E99EE3E6
:10A4B000CD57DF4F688379838A839B83C358D0400D
:10A4C00083E424DE882311F0B0DD02C083E4EFDDF5
:10A4D000C156DF4F8883CF59D0408BE417DE8823E5
:10A4E00011F0A3DD02C08BE4E2DDC056DF4F8883AC
:10A4F000C05AD04082E40ADE8823E9F0A5DD0F943B
:10A500001D0170935C0460935B046F5071096E379A
:10A51000710588F0EBEBFFE084918F010F5F1F4F17
:10A52000882311F40C940D5D082E000C990B0E94E9
:10A53000CBA5F801F1CF8CE4E9DD882379F184DD46
:10A540006B017C0160933A1470933B1480933C142C
:10A5500090933D1420E030E0A9010F94FF0187FFA4
:10A5600003C0E3E9FFE00BC020E030E040E050E44E
:10A57000C701B6010E945FFB181684F4F2CF8491E4
:10A580008F010F5F1F4F882311F40C940D5D082E6F
:10A59000000C990B0E94CBA5F801F1CF81E587DD76
:10A5A000882309F447C08091610490916204892B4B
:10A5B00081F14ADD6B017C01609342147093431476
:10A5C00080934414909345142DEC3CEC4CE45DE3F3
:10A5D0000F94FF0187FF03C0E7E3FFE00BC020E01B
:10A5E00030E040E751E4C701B6010E945FFB181656
:10A5F0000CF5F2CF84918F010F5F1F4F882311F468
:10A600000C940D5D082E000C990B0E94CBA5F8014F
:10A61000F1CFE8E6FFE084918F010F5F1F4F8823A1
:10A6200011F40C940D5D082E000C990B0E94CBA523
:10A63000F801F1CF83E56ADD882341F105DD4B01A7
:10A640005C012DEC3CEC4CEC5DE30F94FF0187FFCB
:10A6500003C0E0E1FFE00BC020E030E040E85FE352
:10A66000C501B4010E945FFB18169CF316C08491CB
:10A670008F010F5F1F4F882311F40C940D5D082E7E
:10A68000000C990B0E94CBA5F801F1CFBDEC8B2EED
:10A69000BCEC9B2EA92CBEE3BB2E80E508DD8823F5
:10A6A00009F44BC08091610490916204892B89F474
:10A6B000E8EDFEE084918F010F5F1F4F882311F4B6
:10A6C0000C940D5D082E000C990B0E94CBA5F8018F
:10A6D000F1CF809158048F5F80935804B5DC6B01F3
:10A6E0007C0160935D0470935E0480935F0490939B
:10A6F000600420E030E0A9010F94FF0187FF03C050
:10A70000E0EBFEE00BC020E030E048EC51E4C70194
:10A71000B6010E945FFB181684F4F2CF84918F017A
:10A720000F5F1F4F882311F40C940D5D082E000C51
:10A73000990B0E94CBA5F801F1CF86E4E7DC8823D2
:10A7400041F182DC6B017C0120E030E040E85FE316
:10A750000F94FF0187FF03C0E7E8FEE00BC020E095
:10A7600030E040E850E4C701B6010E945FFB1816D4
:10A77000B4F4F2CF84918F010F5F1F4F882311F43F
:10A780000C940D5D082E000C990B0E94CBA5F801CE
:10A79000F1CFC12CD12CA0EEEA2EAFE3FA2EA70107
:10A7A0009601C701B6010E94C4FB9B01AC0160E0A9
:10A7B00070E084E490E40F94B50020913E14309151
:10A7C0003F1440914014509141140E94C4FB2B014E
:10A7D0003C01A5019401C501B4010E94C4FB9B0189
:10A7E000AC01C701B6010E94C4FB2CEE31E548EB79
:10A7F0005DE30F94B5009B01AC01C301B2010E945F
:10A80000C4FB60933E1470933F1480934014909364
:10A81000411488E47BDC8823E9F016DC0F941D01E9
:10A8200070935A0460935904655A7109643771052D
:10A8300088F0E9E5FEE084918F010F5F1F4F8823C8
:10A8400011F40C940D5D082E000C990B0E94CBA501
:10A85000F801F1CF85E52BDC8823E9F00E94E2B70F
:10A86000611571058105910511F00E94B0F6809186
:10A87000610490916204892B11F0E6DB04C060E072
:10A8800070E088E492E460935404709355048093DC
:10A8900056049093570482E50ADC811111C0E5E269
:10A8A000FEE084918F010F5F1F4F882311F40C94F9
:10A8B0000D5D082E000C990B0E94CBA5F801F1CF7D
:10A8C0008091610490916204892BD9F08DDBC3568D
:10A8D000DF4F79836883CD59D04016161706CCF028
:10A8E000E1EFFDE084918F010F5F1F4F882311F48A
:10A8F0000C940D5D082E000C990B0E94CBA5F8015D
:10A90000F1CF85E290E0C356DF4F99838883CD591C
:10A91000D04088E5FBDB882361F096DB20912A1488
:10A9200030912B1440912C1450912D140E94D8FF7B
:10A9300008C06091F10C7091F20C8091F30C909131
:10A94000F40C6093500470935104809352049093DC
:10A95000530489E5DBDB882361F076DB20912E143C
:10A9600030912F1440913014509131140E94D8FF2F
:10A9700008C06091F50C7091F60C8091F70C9091E5
:10A98000F80C60934C0470934D0480934E049093A4
:10A990004F04609150047091510480915204909141
:10A9A00053044CE454E00E94324B811111C0E7EC97
:10A9B000FDE084918F010F5F1F4F882311F40C94E9
:10A9C0000D5D082E000C990B0E94CBA5F801F1CF6C
:10A9D00084E46DDB91E089270E941DD820E030E0FF
:10A9E00040EA50E46091F90C7091FA0C8091FB0CF4
:10A9F0009091FC0C0E945FFB87FF16C01DAA1EAA47
:10AA00001FAA18AE80E090E0A0EAB0E489839A83A0
:10AA1000AB83BC83BE016B5C7F4FCE0101960E946D
:10AA2000C0D90E94BA6DC7DC0E94E2B76B017C01FD
:10AA3000A8E8CA0EA3E1DA1EE11CF11C80915B04B8
:10AA400090915C048739910514F086E990E0909329
:10AA5000FD138093FC130E94266960915B04709142
:10AA60005C04072E000C880B990B0E9465FB9B0170
:10AA7000AC016091061470910714809108149091B4
:10AA800009140E94D8FF4B015C0120E030E0A901CD
:10AA90000F94FF0118163CF520E030E040E450E44C
:10AAA000C501B4010F94FF0118163CF50E94E2B7EE
:10AAB000DC01CB018C199D09AE09BF09B7FD10C09F
:10AAC0000E94E2B76B017C01B8E8CB0EB3E1DB1E5C
:10AAD000E11CF11C0E94E0B88AE090E00E94CBA546
:10AAE0000E945796BACF20E030E040E450ECC50118
:10AAF000B4010E945FFB87FDD9CF809159049091EA
:10AB00005A049093FF138093FE1380E00E947169B2
:10AB10006091590470915A04072E000C880B990B10
:10AB20000E9465FB9B01AC016091021470910314BB
:10AB300080910414909105140E94D8FF4B015C0190
:10AB400020E030E0A9010F94FF0118163CF520E049
:10AB500030E040E450E4C501B4010F94FF01181641
:10AB60003CF50E94E2B7DC01CB018C199D09AE09CE
:10AB7000BF09B7FD10C00E94E2B76B017C01E8E895
:10AB8000CE0EE3E1DE1EE11CF11C0E94E0B88AE07B
:10AB900090E00E94CBA50E945796BACF20E030E00B
:10ABA00040E450ECC501B4010E945FFB87FDD9CFA2
:10ABB0001092FD0C1092FE0C1092FF0C1092000DE2
:10ABC0000E94D0A5809158048823B1F1ABDA20917E
:10ABD0005D0430915E0440915F0450916004609187
:10ABE00052147091531480915414909155140E94F2
:10ABF000D9FF60935214709353148093541490931C
:10AC0000551420E030E040E751E46091E203709198
:10AC1000E3038091E4039091E5030F94B500698309
:10AC20007A838B839C83CE0101960E946F4B0E9496
:10AC3000BA6D78DA0E947FCC80E2ECE2F4E0DF01CA
:10AC4000282F1D922A95E9F7ECE0F4E0DF01282F88
:10AC50001D922A95E9F7ECEEF3E0DF011D928A954B
:10AC6000E9F760DA80913A1490913B14A0913C147A
:10AC7000B0913D1480934E1490934F14A0935014B0
:10AC8000B093511419821A821B821C829E012F5F7D
:10AC90003F4F4EE454E16AE474E186E494E14CDA17
:10ACA0009E012D573F4F4EE454E16AE474E186E47F
:10ACB00094E142DA8E010F5F1F4F6E01B5E3CB0EB8
:10ACC000D11CE12CF12CB7010F2C000C880B990B37
:10ACD0000E9465FB20E030E040EF51E40E94C4FB9D
:10ACE0004B015C0120E030E044EB53E40F94FF01A2
:10ACF00018164CF420E030E044EB53E4C501B401F5
:10AD00000E94D8FFEDCF20E030E0A901C501B401D9
:10AD10000E945FFB87FF0BC020E030E044EB53E470
:10AD2000C501B4010E94D9FF4B015C01ECCF2BEDB2
:10AD30003FE049E450E4C501B4010E94C4FB20E0B7
:10AD400030E044E353E40F94B5004B015C010F94F1
:10AD5000B20020E030E040EA50E40E94C4FBF80179
:10AD600061937193819391938F01C501B4010F9405
:10AD70003A0220E030E040EA50E40E94C4FBD601F1
:10AD80006D937D938D939D936D01BFEFEB1AFB0A3D
:10AD9000EDE0EE16F10409F096CFC156DF4FF881D1
:10ADA000CF59D040FF2329F065EF7CE081EF9CE094
:10ADB00004C06CE474E080E594E00E947BE7AA960E
:10ADC0002FAFAA97AB963FAFAB97AC964FAFAC9770
:10ADD000AD965FAFAD97AE966FAFAE97AF967FAFC4
:10ADE000AF97C456DF4F2883CC59D040CD56DF4FA4
:10ADF0003883C359D040C456DF4F2881CC59D04046
:10AE000027FD9EC4CD56DF4F3881C359D04037FD52
:10AE100097C4E22E220FFF0880914E0C90914F0CA8
:10AE2000E89EB001E99E700DF89E700D112480918E
:10AE30004A0C90914B0C680F791F072E000C880B61
:10AE4000990B0E9465FBCC56DF4F688379838A8318
:10AE50009B83C459D040CD56DF4F8881C359D04021
:10AE6000082F880F110B8091500C9091510C089F66
:10AE7000B001099F700D189F700D112480914C0C2A
:10AE800090914D0C680F791F072E000C880B990BC1
:10AE90000E9465FBC856DF4F688379838A839B8352
:10AEA000C859D040C158DF4F688379838A839B8318
:10AEB000CF57D040AE0141585F4FCC56DF4F68812D
:10AEC00079818A819B81C459D0400E94324B88236A
:10AED00009F436C480919C03882391F0B7018EEA6F
:10AEE0009DE00E94028EB80188EA9DE00E94028ED9
:10AEF00089E290E00E94CBA58AE090E00E94CBA579
:10AF0000C456DF4F9881CC59D04091110DC0CD5619
:10AF1000DF4FA881C359D040AA2399F1A530C1F5CC
:10AF2000412C512C32013AC0C456DF4FB881CC5964
:10AF3000D040B53081F4CD56DF4FE881C359D040C1
:10AF4000EE2399F1412C512CF7E86F2EF3E47F2E7C
:10AF5000E53089F50FC0CD56DF4FF881C359D04099
:10AF6000FF2381F1412C512CE4EB6E2EE3E47E2E85
:10AF7000F53071F5C12CD12C74E3E72E73E4F72E74
:10AF800053C1412C512C64EB662E62E4762E20C016
:10AF9000412C512C54EB652E52E4752EC12CD12C32
:10AFA00044EBE42E42ECF42E3FC1412C512C34E30F
:10AFB000632E33E4732EC12CD12C24EBE22E22E439
:10AFC000F22E32C1412C512C94E3692E93E4792E58
:10AFD000C12CD12C760128C120E030E040EF51E4B3
:10AFE000C701B6010F94B5000F941D018B0177FFC7
:10AFF0002CC1045F1F4F5801AA0CBB1CAA0CBB1C20
:10B0000021E030E02C0F3D1FA20EB31ED5012D9183
:10B010003D914D915C91CC56DF4F688179818A8159
:10B020009B81C459D0400E94D9FFC957DF4F688324
:10B0300079838A839B83C758D040F50124A935A919
:10B0400046A957A9C856DF4F688179818A819B81BB
:10B05000C859D0400E94D9FFC557DF4F6883798314
:10B060008A839B83CB58D0400F5F1F4F000F111F67
:10B07000000F111F21E030E02C0F3D1F020F131FA6
:10B08000D8012D913D914D915C91CC56DF4F688157
:10B0900079818A819B81C459D0400E94D9FFC157D0
:10B0A000DF4F688379838A839B83CF58D040F80130
:10B0B00024A935A946A957A9C856DF4F68817981C7
:10B0C0008A819B81C859D0400E94D9FF4B015C0105
:10B0D00020E030E040E85FE3C957DF4F68817981C5
:10B0E0008A819B81C758D0400E945FFB87FFB5C013
:10B0F00080E090E0A0E8BFE3C957DF4F88839983E1
:10B10000AA83BB83C758D040C957DF4F8881998134
:10B11000AA81BB81C758D040EF968CAF9DAFAEAF30
:10B12000BFAFEF9720E030E040E85FE3C557DF4F67
:10B13000688179818A819B81CB58D0400E945FFBD6
:10B1400087FFA1C080E090E0A0E8BFE3C557DF4FD4
:10B1500088839983AA83BB83CB58D040C557DF4FE0
:10B1600088819981AA81BB81CB58D040EB968CAF66
:10B170009DAFAEAFBFAFEB9720E030E040E85FE3BC
:10B18000C157DF4F688179818A819B81CF58D04038
:10B190000E945FFB87FF8DC080E090E0A0E8BFE3E6
:10B1A000C157DF4F88839983AA83BB83CF58D04090
:10B1B000C157DF4F88819981AA81BB81CF58D04088
:10B1C000E7968CAF9DAFAEAFBFAFE79720E030E022
:10B1D00040E85FE3C501B4010E945FFB87FF7FC0C9
:10B1E000812C912CA0E8AA2EAFE3BA2EE3968CAE68
:10B1F0009DAEAEAEBFAEE3979E0121593F4FAE016B
:10B200004D585F4FBE0169587F4FCE0185589F4F03
:10B210000E94ABCC20E030E040EF51E4C701B60122
:10B220000E94D9FF6B017C012DEC3CEC4CEC5DE302
:10B23000C301B2010E94D8FF9B01AC01C701B60156
:10B240000E945FFB87FDC8CE5CC06C3071050CF4BA
:10B25000D2CE8B010C501109CECE20E030E047E475
:10B2600053E4C957DF4F688179818A819B81C75830
:10B27000D0400F94FF0118160CF046CF80E090E00C
:10B28000A7E4B3E439CF20E030E047E453E4C55706
:10B29000DF4F688179818A819B81CB58D0400F94A0
:10B2A000FF0118160CF05ACF80E090E0A7E4B3E459
:10B2B0004DCF20E030E047E453E4C157DF4F6881D1
:10B2C00079818A819B81CF58D0400F94FF01181655
:10B2D0000CF06ECF80E090E0A7E4B3E461CF20E013
:10B2E00030E047E453E4C501B4010F94FF011816A0
:10B2F0000CF07CCF812C912CF7E4AF2EF3E4BF2E21
:10B3000075CFA1E0B0E0C957DF4FB983A883C75814
:10B31000D040C957DF4FA881B981C758D040119795
:10B32000C856DF4FB983A883C859D04001E010E068
:10B33000C856DF4F0880C859D04002C0000F111F07
:10B340000A94E2F7E1E0F0E0C957DF4F0880C75800
:10B35000D04002C0EE0FFF1F0A94E2F7CF55DF4F37
:10B36000F983E883C15AD0402CEE33E0CC56DF4F4E
:10B3700039832883C459D0408CE294E0C157DF4F11
:10B3800099838883CF58D040ACE0B4E0C557DF4FF5
:10B39000B983A883CB58D040212C312CC157DF4F23
:10B3A00068807980CF58D040F301808191819C01E1
:10B3B00020233123232B09F4BFC0CF55DF4F288131
:10B3C0003981C15AD04082239323892B09F4B4C018
:10B3D000C557DF4FA881B981CB58D0408D919C9142
:10B3E00080239123892B09F0A7C0C0904A0CD090EC
:10B3F0004B0CE0904E0CF0904F0CC856DF4F8881FC
:10B400009981C859D0408E9DB0018F9D700D9E9D31
:10B41000700D11246C0D7D1D6E5F7F4F072E000C8B
:10B42000880B990B0E9465FB4B015C01C957DF4FEC
:10B43000A881B981C758D040AE9DB001AF9D700DB5
:10B44000BE9D700D11246C0D7D1D62507109072E7B
:10B45000000C880B990B0E9465FB6B017C0120E0BE
:10B4600030E040E85FE3C501B4010E945FFB87FF65
:10B4700086C1812C912CE0E8AE2EEFE3BE2EEF9634
:10B480008CAE9DAEAEAEBFAEEF978091500C90915A
:10B49000510C289EB001299E700D389E700D11240C
:10B4A00080914C0C90914D0C680F791F1616170661
:10B4B0000CF077C1683C710514F067EC70E0072E62
:10B4C000000C880B990B0E9465FBE3966CAF7DAF77
:10B4D0008EAF9FAFE397EB966CAF7DAF8EAF9FAF14
:10B4E000EB9720E030E040E85FE3C701B6010E943F
:10B4F0005FFB87FF5BC1C12CD12C60E8E62E6FE3B8
:10B50000F62EE796CCAEDDAEEEAEFFAEE797AE011F
:10B5100049585F4FC501B4010E94324B811158C197
:10B52000C557DF4FE881F981CB58D04080819181A8
:10B53000802B912B91838083C157DF4F28813981E4
:10B54000CF58D0402E5F3F4FC157DF4F39832883FC
:10B55000CF58D040D3018D919C9180239123892B8A
:10B5600009F4BBC0F9018081918180239123892B4B
:10B5700009F4B3C0CC56DF4FE881F981C459D040FB
:10B580008081918180239123892B09F0A6C0C090EE
:10B590004C0CD0904D0CE090500CF090510C2E9C27
:10B5A000B0012F9C700D3E9C700D11246C0D7D1D03
:10B5B0006E5F7F4F072E000C880B990B0E9465FB76
:10B5C0002B013C01C10101968E9DB0018F9D700D34
:10B5D0009E9D700D11246C0D7D1D62507109072E0A
:10B5E000000C880B990B0E9465FB4B015C0180915C
:10B5F0004E0C90914F0CC856DF4F28813981C859A5
:10B60000D040289FB001299F700D389F700D1124E4
:10B6100080914A0C90914B0C680F791F16161706F3
:10B620000CF01FC1683C710514F067EC70E0072E48
:10B63000000C880B990B0E9465FB6B017C01E7965F
:10B64000CCAEDDAEEEAEFFAEE797EF96CCAEDDAEA4
:10B65000EEAEFFAEEF9720E030E040E85FE3C301DD
:10B66000B2010E945FFB87FF03C1412C512C30E8DF
:10B67000632E3FE3732EEB964CAE5DAE6EAE7FAEA7
:10B68000EB9720E030E040E85FE3C501B4010E94A1
:10B690005FFB87FFFFC0812C912C90E8A92E9FE3D0
:10B6A000B92EE3968CAE9DAEAEAEBFAEE397AE01C3
:10B6B00049585F4FC701B6010E94324B8111FCC04F
:10B6C000CC56DF4FA881B981C459D0408D919C914F
:10B6D0001197802B912B8D939C93BFEF2B1A3B0AD4
:10B6E000CC56DF4FE881F981C459D0403296CC5610
:10B6F000DF4FF983E883C459D040C557DF4F288115
:10B700003981CB58D0402E5F3F4FC557DF4F39832B
:10B710002883CB58D04036E02316310409F03ECEC2
:10B72000C957DF4F88819981C758D0400196C957C2
:10B73000DF4F99838883C758D040079709F0E9CD38
:10B74000C356DF4FE881F981CD59D0403197C356B8
:10B75000DF4FF983E883CD59D040EF2B09F4F5C0D2
:10B76000C456DF4FF881CC59D040F7FDEEC0CD561E
:10B77000DF4F2881C359D04027FF0FCBE6C020E020
:10B7800030E047E453E4C501B4010F94FF011816FB
:10B790000CF075CE812C912C77E4A72E73E4B72E94
:10B7A0006ECE60E070E080E89FE38FCE20E030E076
:10B7B00047E453E4C701B6010F94FF0118160CF0DB
:10B7C000A0CEC12CD12C57E4E52E53E4F52E99CE12
:10B7D000AE0141595F4FC701B6010E94324B882329
:10B7E00009F49ECE80919C03882361F1B501A401E8
:10B7F00086E79DE00E94E18DEB964CAD5DAD6EADB0
:10B800007FADEB9780E79DE00E94E18DE7964CAD20
:10B810005DAD6EAD7FADE79786E69DE00E94E18D60
:10B82000E3964CAD5DAD6EAD7FADE39780E69DE0F8
:10B830000E94E18D89E290E00E94CBA58AE090E031
:10B840000E94CBA59E0121593F4FAE014D585F4F3D
:10B85000BE0169587F4FCE0185589F4F0E94ABCCE7
:10B860005FCEC12CD12C40E8E42E4FE3F42EE7CE7E
:10B8700020E030E047E453E4C301B2010F94FF013C
:10B8800018160CF0F8CE412C512C27E4622E23E43C
:10B89000722EF1CE20E030E047E453E4C501B4015C
:10B8A0000F94FF0118160CF0FCCE812C912C87E42C
:10B8B000A82E83E4B82EF5CEAE0141595F4FC701E3
:10B8C000B6010E94324B882309F4FACE80919C0382
:10B8D000882361F1B701A6018CE39DE00E94E18D10
:10B8E000EB964CAD5DAD6EAD7FADEB9786E39DE025
:10B8F0000E94E18DE7964CAD5DAD6EAD7FADE797F3
:10B900008CE29DE00E94E18DE3964CAD5DAD6EADA5
:10B910007FADE39786E29DE00E94E18D89E290E0B1
:10B920000E94CBA58AE090E00E94CBA59E01215900
:10B930003F4FAE014D585F4FBE0169587F4FCE015A
:10B9400085589F4F0E94ABCCBBCE8CE99DE00E94F6
:10B9500025C10E947FCC80E090E0A0EAB0E4809313
:10B960004E1490934F14A0935014B0935114E39637
:10B970001CAE1DAE1EAE1FAEE3979E0121593F4F78
:10B980004EE454E16AE474E186E494E10E949C5040
:10B990008091500490915104A0915204B0915304AD
:10B9A0008093461490934714A0934814B09349147D
:10B9B00080914C0490914D04A0914E04B0914F049D
:10B9C00080934A1490934B14A0934C14B0934D144D
:10B9D000E3961CAE1DAE1EAE1FAEE3979E0121592D
:10B9E0003F4F4EE454E16AE474E186E494E10E943E
:10B9F0009C50C056DF4FF881C05AD040F1110DC0A5
:10BA00001092FD131092FC130E9426691092FF13EE
:10BA10001092FE1380E00E947169CE55DF4F0FB681
:10BA2000F894DEBF0FBECDBFDF91CF911F910F9174
:10BA3000FF90EF90DF90CF90BF90AF909F908F904E
:10BA40007F906F905F904F903F902F900895EF926E
:10BA5000FF920F931F93CF93DF938C017C018FEFA5
:10BA6000E80EF11CF701808190E0FB01C481D581D3
:10BA70009E01280F391F2F3F310520F0CFEFD0E076
:10BA8000C81BD90BFB0160817181AE01800F911F32
:10BA90000F94D103F70180818C0FF7018083F801A7
:10BAA0008281C80FC283C801DF91CF911F910F918E
:10BAB000FF90EF9008950F931F93CF93DF9300D0E3
:10BAC00000D0CDB7DEB78C01FC01E150FF4F808183
:10BAD0008E3FC0F491E0980F9083A801480F511D4C
:10BAE000DB0111962C91DA012C938E5F8083F80193
:10BAF000E90FF11DDB018C918083F80182818E5F5B
:10BB000082830AC060EA71E1CE0101960E94397613
:10BB1000CE0101960E943476C80126960FB6F8949D
:10BB2000DEBF0FBECDBFDF91CF911F910F91089562
:10BB30000F931F93CF93DF9300D000D0CDB7DEB724
:10BB40008C01FC01E150FF4F80818F3F71F091E04B
:10BB5000980F9083FB019081F801E80FF11D90830D
:10BB6000F80182818F5F82830AC061E971E1CE01B1
:10BB700001960E943976CE0101960E943476C80162
:10BB800026960FB6F894DEBF0FBECDBFDF91CF91E2
:10BB90001F910F910895BF92CF92DF92EF92FF9283
:10BBA0000F931F93CF93DF9300D000D0CDB7DEB7B4
:10BBB0008C017B016A01BA010E941375B701CE01A5
:10BBC00001967C010E9441760E151F0521F0B701F8
:10BBD000C8010E94DA74C7010E94347680E2B82E50
:10BBE000F801848195818C159D0548F4B9821A82EB
:10BBF00041E050E0B701C8010E943A75F1CF2696A6
:10BC00000FB6F894DEBF0FBECDBFDF91CF911F916D
:10BC10000F91FF90EF90DF90CF90BF9008959F928B
:10BC2000AF92BF92CF92DF92EF92FF920F931F934A
:10BC3000CF93DF9300D000D0CDB7DEB75C017B019E
:10BC40008A016AE973E00E944176D70114968D91CA
:10BC50009C9115970817190730F06D917C91A801F8
:10BC6000C50199DF31C06AE973E0FE0131966F01C9
:10BC7000CF010E944176D70114968D919C91159722
:10BC80000097C1F08017910708F48C01D701ED915E
:10BC9000FC911197E00FF11F908010826D917C91C3
:10BCA000C6010E940A76F70140815181FA01E00F36
:10BCB000F11F9082AC14BD0421F0B601C5010E94B1
:10BCC000DA74C6010E94347626960FB6F894DEBF69
:10BCD0000FBECDBFDF91CF911F910F91FF90EF90DD
:10BCE000DF90CF90BF90AF909F900895EF92FF921A
:10BCF0000F931F93CF93DF93CDB7DEB72C970FB67B
:10BD0000F894DEBF0FBECDBF8C017B016AE973E002
:10BD10000E9441766BEE72E0CE0107960E9441765A
:10BD20006BEE72E0CE0101960E9441766F2D70E0BD
:10BD3000C8010E946775BE016F5F7F4FC8010E94F6
:10BD40009675B701772784E0769567958A95E1F730
:10BD5000C8010E946775BE01695F7F4FC8010E94DC
:10BD60009675B7016F707727C8010E946775CE017D
:10BD700001960E943476CE0107960E943476C8015F
:10BD80002C960FB6F894DEBF0FBECDBFDF91CF91DA
:10BD90001F910F91FF90EF900895CF938091F7132B
:10BDA0008823B9F14091EF135091F0136091F11392
:10BDB0007091F2132FEE31E18091F8139091F91305
:10BDC0000E94E993C82F811102C0C0E023C04091B6
:10BDD000F3135091F4136091F5137091F61341151C
:10BDE00051056105710591F02FEE31E18091F81355
:10BDF0009091F9130E94E993882339F31092F31379
:10BE00001092F4131092F5131092F6131092F71388
:10BE100001C0C1E08C2FCF910895CF92DF92EF92B5
:10BE2000FF92CF936B017C01C42F8091EF1390910F
:10BE3000F013A091F113B091F2138C159D05AE058E
:10BE4000BF05C9F0AADF811102C080E018C02FEE43
:10BE500031E1B701A6018091F8139091F9130E9486
:10BE60004B94882391F3C092EF13D092F013E09299
:10BE7000F113F092F21381E0C1118093F713CF9187
:10BE8000FF90EF90DF90CF9008954F925F926F9266
:10BE90007F928F929F92AF92BF92CF92DF92EF925A
:10BEA000FF920F931F93CF93DF93EC016A017B0105
:10BEB00028013901423051056105710510F480E017
:10BEC00064C089859A85AB85BC850196A11DB11D8D
:10BED00084179507A607B70790F38F89803149F437
:10BEE0008D2C9E2CAF2CBB248B899C89AD89BE895F
:10BEF0000FC0803221F78B889C88AD88BE88DB011B
:10BF0000CA0157E0B695A795979587955A95D1F7A9
:10BF1000880E991EAA1EBB1E41E0C501B4017DDF3B
:10BF2000882369F29F89903161F4DD24EE24FF2497
:10BF30009601220F331FF901E151FE4E51824082DA
:10BF400011C0E894C7F8DD24EE24FF249601220FE7
:10BF5000331F220F331FF901E151FE4E40825182FF
:10BF6000628273829A89923080F04D815E816F8106
:10BF70007885840E951EA61EB71E8092F3139092AC
:10BF8000F413A092F513B092F613DF91CF911F91A5
:10BF90000F91FF90EF90DF90CF90BF90AF909F9068
:10BFA0008F907F906F905F904F900895CF92DF9227
:10BFB000EF92FF920F931F93CF93DF93FC01818544
:10BFC0009285A385B4850196A11DB11D841795079F
:10BFD000A607B70710F480E060C08789803149F474
:10BFE000BB27A72F962F852FC388D488E588F6888E
:10BFF0000FC0803281F783899489A589B6896A0147
:10C000007B01C7E0F694E794D794C794CA95D1F71B
:10C010008C0D9D1DAE1DBF1DE9016A017B018F01C5
:10C020004091EF135091F0136091F1137091F2135E
:10C0300084179507A607B70731F040E0BC01CD0192
:10C04000ECDE882341F2F8018789803179F4B70169
:10C05000A601552766277727440F551FFA01E1519E
:10C06000FE4E80819181A0E0B0E012C0B701A60130
:10C070004F77552766277727440F551F440F551FC5
:10C08000FA01E151FE4E80819181A281B381BF709E
:10C0900088839983AA83BB8381E0DF91CF911F912D
:10C0A0000F91FF90EF90DF90CF9008954F925F92A5
:10C0B0006F927F92AF92BF92CF92DF92EF92FF92F8
:10C0C0000F931F93CF93DF9300D01F92CDB7DEB7AE
:10C0D0008C0149835A836B837C835901C12CD12CF9
:10C0E0007601412C82E0582E612C712C49815A81B5
:10C0F0006B817C819E012F5F3F4FC80157DF8823F2
:10C1000041F1D301C201F801058404C0880F991FD1
:10C11000AA1FBB1F0A94D2F7C80ED91EEA1EFB1E27
:10C1200049815A816B817C818789803139F481E032
:10C13000483F5F4F6105710538F4D8CF81E0483F33
:10C140005F4F6F4F7F4090F2F501C082D182E28253
:10C15000F3820F900F900F900F90DF91CF911F916E
:10C160000F91FF90EF90DF90CF90BF90AF907F90B6
:10C170006F905F904F900895CF93DF93EC018B8188
:10C18000882331F1898187FF20C061E0CE010E94C0
:10C190002E92FC01892BE1F08081853EC9F08B81D4
:10C1A000823040F489899A89AB89BC89848F958FC4
:10C1B000A68FB78F8D899E89AF89B88D938F828F17
:10C1C000B58BA48B89818F778983DF91CF91E5CD62
:10C1D00081E0888380E0DF91CF9108958F929F92D4
:10C1E000AF92BF92CF92DF92EF92FF920F931F9385
:10C1F000CF93DF93EC018B81811102C080E076C088
:10C2000009891A892B893C890417150726073707DE
:10C21000A8F36A017B01823029F4C886D986EA86B0
:10C22000FB860DC0C114D104E104F10451F4188659
:10C2300019861A861B861C821D821E821F8281E03F
:10C2400055C088849984AA84BB84E98DFA8D25859C
:10C2500030E0275F3F4FB501A4014150510961090A
:10C260007109022E04C076956795579547950A94F3
:10C27000D2F7D701C6010197A109B10904C0B6954B
:10C28000A795979587952A95D2F784179507A607BE
:10C29000B70720F089288A288B2849F44D895E89C0
:10C2A0006F89788D4C835D836E837F8304C0841B8C
:10C2B000950BA60BB70B4C015D018E010C5F1F4F58
:10C2C00081149104A104B10409F4A7CF4C815D81CC
:10C2D0006E817F819801898D9A8D68DE91E0891A3F
:10C2E0009108A108B1088111EBCF88CFDF91CF91E0
:10C2F0001F910F91FF90EF90DF90CF90BF90AF9084
:10C300009F908F9008952F923F924F925F926F92DD
:10C310007F928F929F92AF92BF92CF92DF92EF92D5
:10C32000FF920F931F93CF93DF9300D01F92CDB74F
:10C33000DEB78C014B011A01DC0113968C91139727
:10C340008130C1F411968C9181FF14C082FF18C016
:10C35000F801418952896389748980859185A28514
:10C36000B38584179507A607B70751F0C80136DFD4
:10C37000811106C081E0F80180838FEF9FEF2CC10F
:10C38000610185C0D80159968D919C915A97FC0105
:10C39000248121502A013B0139E076946794579417
:10C3A00047943A95D1F7722E74207A01F1E0FF227A
:10C3B000772009F478C080E092E08E199F09560139
:10C3C0008C159D0508F45C01D80159962D913C917E
:10C3D0005A9714968D919D910D90BC91A02D029726
:10C3E000A109B109F901058404C0880F991FAA1F8A
:10C3F000BB1F0A94D2F74685578560897189840FDF
:10C40000951FA61FB71F9C01AD01270D311D411DB2
:10C41000511D29013A01A11432E0B30609F089C087
:10C420008091EF139091F013A091F113B091F2135A
:10C4300084159505A605B70569F41092F7138FEFDB
:10C440009FEFDC018093EF139093F013A093F1130F
:10C45000B093F2139401B301A2018091F81390916B
:10C46000F9130E94E993882309F484CFF8018085A9
:10C470009185A285B3858A0D9B1DA11DB11D808765
:10C480009187A287B3878A0C9B1CCA18DB08D80146
:10C4900018964D915D916D917C911B97C114D104BB
:10C4A00009F070CF7AC0E114F10409F084CF14963A
:10C4B0004D915D916D917C911797411551056105E5
:10C4C000710559F455968D919D910D90BC91A02DBB
:10C4D0000097A105B10539F520C09E012F5F3F4FA0
:10C4E00065DD882309F446CF89819A81AB81BC81BF
:10C4F000F801218D328DF9012789203139F4883FE7
:10C50000FFEF9F07A105B10540F40DC0883F2FEF55
:10C510009207A2072FE0B20730F0C8010E944A92AA
:10C52000811149CF27CFF80184839583A683B783F0
:10C5300042CFE114F10411F5D80118964D915D91A7
:10C540006D917C911B9751968D919D910D90BC9111
:10C55000A02D481759076A077B0780F01EDC882347
:10C5600009F408CF81E08093F7134092EF135092C3
:10C57000F0136092F1137092F21307C041E0C3010F
:10C58000B2014BDC882309F4F5CEA501B401C70143
:10C5900081519E4E0F94D10369CF51968D919D91FB
:10C5A0000D90BC91A02D84179507A607B70740F4FE
:10C5B000F801418B528B638B748B818180688183FE
:10C5C000D80111968C9183FD02C0C10105C0C8013C
:10C5D000D3DD8111FACFCECE0F900F900F900F9038
:10C5E000DF91CF911F910F91FF90EF90DF90CF904F
:10C5F000BF90AF909F908F907F906F905F904F9083
:10C600003F902F900895CF93DF931F92CDB7DEB761
:10C61000698341E050E0BE016F5F7F4F049673DE97
:10C620000F90DF91CF9108952F923F924F925F929A
:10C630006F927F928F929F92AF92BF92CF92DF9232
:10C64000EF92FF920F931F93CF93DF9300D01F922F
:10C65000CDB7DEB79C838B834B015A01DC01139667
:10C660008C91811103C08FEF9FEFE9C0EB81FC81BA
:10C67000818180FFF8CFAB81BC8151960D911D91D6
:10C680002D913C91549718964D915D916D917C91AF
:10C690001B97C501A0E0B0E068017901C41AD50A72
:10C6A000E60AF70AC816D906EA06FB0618F4580186
:10C6B000A41AB50A75018B819C8104969A8389839B
:10C6C000612C92E0792EE114F10409F48AC0AB8167
:10C6D000BC8118964D915D916D917C911B976A017B
:10C6E000B1E0DB22EB81FC8123811A012B0189E07F
:10C6F00056944794379427948A95D1F7818D928DDB
:10C70000223061F4FC01828D938DA48DB58DBC0126
:10C71000CD01620D731D841D951D49C0DC01149669
:10C720001C9111501221C114D104F9F411111DC032
:10C73000452B462B472B59F4EB81FC818589968943
:10C74000A789B08D84839583A683B7830EC0AB8100
:10C75000BC8114964D915D916D917C9117972981C3
:10C760003A8124DC882309F47ECFEB81FC81218D82
:10C77000328D84819581A681B7810297A109B10983
:10C78000F901058404C0880F991FAA1FBB1F0A94D2
:10C79000D2F74685578560897189840F951FA61F3A
:10C7A000B71FBC01CD01610F711D811D911D93014A
:10C7B0002C193D0987012E153F0508F48901011543
:10C7C000F2E01F0779F52091EF133091F0134091BB
:10C7D000F1135091F213621773078407950719F448
:10C7E00021C0C5012CC09401AB01BC018091F8139C
:10C7F0009091F9130E944B94882309F434CF800E52
:10C80000911EEB81FC8180859185A285B385800F87
:10C81000911FA11DB11D80879187A287B387E01A60
:10C82000F10A51CF40E0F9DA882309F41CCFB601B0
:10C8300061517E4EA801C4010F94D103E0CF0F9047
:10C840000F900F900F90DF91CF911F910F91FF905C
:10C85000EF90DF90CF90BF90AF909F908F907F90A0
:10C860006F905F904F903F902F900895DF92EF92DE
:10C87000FF920F931F93CF93DF937C01EB018A010B
:10C880008DE0D82E40E250E0BE01C701CDDE8032FF
:10C89000910539F021E0892B09F420E0822F819560
:10C8A0003EC02881222399F1253E61F32E3251F3B7
:10C8B0000115110541F13B853F733F3021F54A8D4C
:10C8C0005B8D452B01F52F713FEF320F3230D8F4DD
:10C8D00030E021503109D29EC001D39E900D112429
:10C8E000D801A80FB91FFE0120E0AD01253088F462
:10C8F00031813D932F5F32962D30C1F7288126FF7D
:10C9000002C0FA0115862B8523FDBCCF08C080E04C
:10C9100006C02B3010F43481ECCF3681EACFDF91A2
:10C92000CF911F910F91FF90EF90DF9008954F925C
:10C930005F926F927F92AF92BF92CF92DF92EF920F
:10C94000FF920F931F93CF93DF931F92CDB7DEB764
:10C950008C017B015A01D22EDB0159968D919C915D
:10C960005A97F801928F818F40E050E0BA01C701D9
:10C9700035DCC12CF70180859185A285B38541897D
:10C9800052896389748984179507A607B70708F049
:10C9900062C025E0B695A795979587952A95D1F71A
:10C9A000F82FFF707F2ED70113968C91823008F4F8
:10C9B00063C041E050E0BE016F5F7F4FC70134DECE
:10C9C000019719F4898190E002C08FEF9FEF0196E3
:10C9D00009F452C0F70180859185A285B3854F96F1
:10C9E000A11DB11D80879187A287B387F0E27F9E4A
:10C9F000C0011124BC0161517E4E61157105E1F148
:10CA0000DB012C91222319F0253ED1F465C1C11020
:10CA10000EC04091EF135091F0136091F11370919B
:10CA2000F213F8014487558766877787708AFC017F
:10CA3000E151FE4E8081882361F0CC24C3949ACFCB
:10CA40004BE050E0C5010F94C403892B09F092CF4D
:10CA500015C0CC24C3948D2D8274823469F4CC200B
:10CA600009F489C0D80150967C9061E0C8010E9409
:10CA70002E92009709F005C180E031C1D7FCFCCFB0
:10CA8000F0E27F9EA00111249A0121513E4ED9016E
:10CA90001B968C91817121F08D2D827109F067C0F8
:10CAA0008091EF139091F013A091F113B091F213D4
:10CAB000F80184879587A687B787708AFA01E151C4
:10CAC000FE4E4489558960E070E0BA01552744273D
:10CAD000D80155964D935D936D937C935897828DB5
:10CAE000938DA0E0B0E0482B592B6A2B7B2BD8010B
:10CAF00055964D935D936D937C935897D9011B96F2
:10CB00008C91887159F4848D958DA68DB78DF8011F
:10CB1000818B928BA38BB48B81E00FC0803139F570
:10CB200098012F5E3F4FD80159968D919C915A974D
:10CB3000BDDA8823E1F084E0F80183838D2D8F70C6
:10CB4000D80111968C931197F801148215821682E0
:10CB5000178218961D921D921D921C921B97D4FE4F
:10CB6000AFC0C8010E941CA88111AAC085CFD801FE
:10CB700013961C9281CFF7018381823009F47CCF18
:10CB800081899289A389B489803E9F4FAF41B105C5
:10CB900008F072CFC7010E944A92882309F46CCF33
:10CBA000FCD8882309F468CFD70159962D913C9180
:10CBB0005A9714968D919D910D90BC91A02D02973E
:10CBC000A109B109F901058404C0880F991FAA1FA2
:10CBD000BB1F0A94D2F74684578460887188480E38
:10CBE000591E6A1E7B1E81E08093F7134092EF135B
:10CBF0005092F0136092F1137092F21380E092E081
:10CC0000EFEEF1E1DF019C011D9221503040E1F790
:10CC1000CC24C394D7015996ED91FC915A97848105
:10CC2000C81698F42FEE31E1B301A2014C0D511D4D
:10CC3000611D711D8091F8139091F9130E94E99381
:10CC4000882309F419CFC394E5CF80E092E0A0E0F7
:10CC5000B0E0058404C0880F991FAA1FBB1F0A9467
:10CC6000D2F7F7014189528963897489840F951F2E
:10CC7000A61FB71F818B928BA38BB48B8FEE91E194
:10CC8000712C20E2DC011D922A95E9F72BE0F501D9
:10CC9000DC0101900D922A95E1F721E238E2FC01D6
:10CCA000318B208B40E058E057874687338B228BAF
:10CCB000318F208F578B468B70D88111E1CEDCCE1F
:10CCC000D5FE08C0F8014189528963897489C80179
:10CCD00085DA05C081E003C0C110AFCE9ACE0F90B7
:10CCE000DF91CF911F910F91FF90EF90DF90CF9048
:10CCF000BF90AF907F906F905F904F9008950F938B
:10CD00001F93CF93DF93FC012381222311F080E056
:10CD100043C08B01EC01FB018789803131F1803206
:10CD2000B1F783E08B83F801428D538D648D758D4F
:10CD30004D8B5E8B6F8B788F9E012F5E3F4FC801AE
:10CD4000B5D9882321F31A8F098F81E0898318864A
:10CD500019861A861B861C821D821E821F82188AD3
:10CD60001C861D861E861F8617C082E08B831D8A47
:10CD70001E8A1F8A188EFB01808D918DA0E0B0E085
:10CD800025E0880F991FAA1FBB1F2A95D1F7898B11
:10CD90009A8BAB8BBC8BD7CFDF91CF911F910F912B
:10CDA0000895CF93DF93EC01E7D91B82DF91CF91F8
:10CDB00008952F923F924F925F926F927F928F923F
:10CDC0009F92AF92BF92CF92DF92EF92FF920F931A
:10CDD0001F93CF93DF93CDB7DEB7C254D1090FB6FF
:10CDE000F894DEBF0FBECDBF4C015B018A01322E2D
:10CDF0001C8E1F8E19821C826115710511F410E0C2
:10CE0000A3C0FC0183818111FACFFA0180818F32A6
:10CE100009F098C0F50183818250823058F0618D0D
:10CE2000728DCE0101966BDF882349F3CE01019606
:10CE30007C0101C07501C8018C010196F8012081B7
:10CE40002F32D1F36E01FCE1CF0ED11C3601CE01A1
:10CE500001962C012396CFAE23972D2C9BE0915069
:10CE6000E7E3F0E0EC0FFD1FE90FF11D80E28083A6
:10CE70009111F5CFD80127E04A2F3B2F8D918111D9
:10CE800007C08FA9803209F4BACF842F932F2CC00A
:10CE90008F32B9F38E3231F42A3009F4B0CF98E0F2
:10CEA0002AE0EACFE1E8F1E13491332321F0319631
:10CEB0003813FACFA4CF291708F4A1CF813208F490
:10CEC0009ECF8F3709F49BCF31E0390FE7E3F0E0D5
:10CED000EC0FFD1FE90FF11D9FE9980F9A3108F43F
:10CEE00080528083932FC8CF8C01FC012081019652
:10CEF0002F32D1F32223E9F021E0AE01495C5F4FEC
:10CF0000B701C60114DD882309F479CFEA14FB04C4
:10CF100011F0C70146DFC614D70441F023969FAD38
:10CF20002397822D7601C92ED82E98CF942D852D4A
:10CF3000F9CF232DAE01495C5F4FB701C401F7DC87
:10CF4000182F02C07B017ECFCE0101960E94D24FE6
:10CF5000CE014C960E94D24F812FCE5BDF4F0FB691
:10CF6000F894DEBF0FBECDBFDF91CF911F910F911F
:10CF7000FF90EF90DF90CF90BF90AF909F908F90F9
:10CF80007F906F905F904F903F902F9008952F92D9
:10CF90003F924F925F926F927F928F929F92AF9249
:10CFA000BF92CF92DF92EF92FF92CF93DF9300D0A8
:10CFB0001F92CDB7DEB76090FE137090FF13809084
:10CFC000021490900314A0900414B0900514B301BF
:10CFD000072C000C880B990B0E9465FBA50194019E
:10CFE0000E94D8FF6B017C016093DC097093DD091E
:10CFF0008093DE099093DF0920ED3CEC4CE45DE387
:10D0000060913219709133198091341990913519CA
:10D010000E94C4FB1B012C012091D8093091D90931
:10D020004091DA095091DB09C501B4010E94D8FF93
:10D030009B01AC01C201B1010E94C4FB1B012C0188
:10D0400023E333E343E75FE36091D4097091D509AB
:10D050008091D6099091D7090E94C4FB9B01AC0135
:10D06000C201B1010E94D9FF69837A838B839C83BB
:10D070006093D4097093D5098093D6099093D7090A
:10D080008092D8099092D909A092DA09B092DB096E
:10D0900020E030E040E251E4C701B6010F94FF0107
:10D0A000181624F481E08093D30989C020E030E091
:10D0B00040E251ECC701B6010E945FFB87FD02C050
:10D0C000672821F481E08093D3099DC08091D30922
:10D0D000882351F01092CF091092D0091092D109F3
:10D0E0001092D2091092D30920912A1930912B194C
:10D0F00040912C1950912D19C701B6010E94C4FB13
:10D100002B013C016093CB097093CC098093CD092E
:10D110009093CE092091CF093091D0094091D10947
:10D120005091D209C701B6010E94D9FF4B015C01A1
:10D130006093CF097093D0098093D1099093D2095D
:10D1400020912E1930912F19409130195091311999
:10D150000E94C4FB9B01AC016093C7097093C8098E
:10D160008093C9099093CA09C301B2010E94D9FFF3
:10D1700029813A814B815C810E94D8FF2B013C01BF
:10D1800020E030E04FE753E40F94FF0120E030E06F
:10D19000A9011816DCF4C701B6010F94FF01181697
:10D1A00074F4A7019601C501B4010E94D8FF6093F1
:10D1B000CF097093D0098093D1099093D209412C63
:10D1C000512C8FE7682E83E4782E20C0C301B20172
:10D1D0000E945FFB87FF1AC020E030E0A901C70171
:10D1E000B6010E945FFB87FF0EC0A7019601C50133
:10D1F000B4010E94D8FF6093CF097093D009809347
:10D20000D1099093D209412C512C3201C301B201B2
:10D210000F900F900F900F90DF91CF91FF90EF90B4
:10D22000DF90CF90BF90AF909F908F907F906F9046
:10D230005F904F903F902F900895609106147091E9
:10D24000071480910814909109140895CF92DF92E9
:10D25000EF92FF92C0900614D0900714E09008144B
:10D26000F09009148091FC139091FD130797BC0175
:10D27000990F880B990B0E9465FB9B01AC01C701BC
:10D28000B6010E945FFB87FF1FC020E030E040E452
:10D2900050E4C701B6010E94D9FF0F942201709398
:10D2A000FB096093FA090E94E2B7DC01CB01805AC6
:10D2B0009541AF4FBF4F8093F6099093F709A09324
:10D2C000F809B093F90908C01092F6091092F7090D
:10D2D0001092F8091092F909FF90EF90DF90CF902B
:10D2E0000895CF92DF92EF92FF92C0900214D090F7
:10D2F0000314E0900414F09005148091FE139091B3
:10D30000FF130797BC01990F880B990B0E9465FBCF
:10D310009B01AC01C701B6010E945FFB87FF1FC0E4
:10D3200020E030E040E450E4C701B6010E94D9FF9C
:10D330000F9422017093F5096093F4090E94E2B7FB
:10D34000DC01CB01805D9A48AF4FBF4F8093F0095D
:10D350009093F109A093F209B093F30908C01092D9
:10D36000F0091092F1091092F2091092F309FF905E
:10D37000EF90DF90CF9008952F923F924F925F925F
:10D380006F927F928F929F92AF92BF92CF92DF92D5
:10D39000EF92FF920F931F93CF93DF93EC0142E63E
:10D3A00055E281E090E0FA0125913491C217D3074C
:10D3B0000CF05DC09C0121503109220F331F220F58
:10D3C000331FD901A05ABA4DFD0165917491225ABB
:10D3D0003A4DF901A590B490FC01EE0FFF1FEE0F3E
:10D3E000FF1FE05AFA4DE590F490FD01C590D490EE
:10D3F000FA0105911491F90125903490072E000C43
:10D40000880B990B0E9465FB2B013C01CA19DB09B3
:10D41000BE01DD0F880B990B0E9465FB4B015C017F
:10D42000B7016C197D09072E000C880B990B0E941F
:10D4300065FB9B01AC01C501B4010E94C4FB6B01FB
:10D440007C01B80162197309072E000C880B990B37
:10D450000E9465FB9B01AC01C701B6010F94B500AA
:10D460009B01AC01C301B2010E94D9FF11C001961A
:10D470004C5F5F4F8034910509F095CFECE5F6E203
:10D4800065917491072E000C880B990B0E9465FB27
:10D49000DF91CF911F910F91FF90EF90DF90CF9090
:10D4A000BF90AF909F908F907F906F905F904F90C4
:10D4B0003F902F90089560E08091CF119091D0110E
:10D4C0000E9438B86093021470930314809304147C
:10D4D000909305148091CD119091CE114DDF609302
:10D4E0000614709307148093081490930914A89558
:10D4F0008FB7F8941092D1118FBF0895DF92EF92F9
:10D50000FF920F931F93CF93DF93F82ED62EE72E23
:10D510008A0161E082E50E9454A780910C02882371
:10D5200009F446C0ECE5F9E28491EF0121968823E5
:10D5300039F0082E000C990B0E94CBA5FE01F4CF08
:10D54000ED2DFE2D8491EF012196882339F0082ED0
:10D55000000C990B0E94CBA5FE01F4CFE0ECF9E1A1
:10D560008491EF012196882339F0082E000C990B45
:10D570000E94CBA5FE01F4CFF7FC0CC06F2DFF0C71
:10D58000770B8EEA9DE00E94BDA68AE090E00E94A3
:10D59000CBA50EC0EBEBF9E18491EF012196882336
:10D5A00039F0082E000C990B0E94CBA5FE01F4CF98
:10D5B0008091C609811108C010920C0281E080930D
:10D5C000C609C8010E942096DF91CF911F910F914B
:10D5D000FF90EF90DF900C94D8BA2F923F924F9229
:10D5E0005F926F927F928F929F92AF92BF92CF92F3
:10D5F000EF92FF920F931F93CF93DF9300D000D051
:10D60000CDB7DEB73C017A8369832B833C834D839E
:10D610005E8317012801C7FC05C00C2D0C2C000CE3
:10D62000110B02C001E010E0000F111F000F111FCD
:10D63000C8018450964F7C01A2019101FC016081D8
:10D640007181828193810E945FFB8823B1F0F70191
:10D650002082318242825382EE24E394F12C20E036
:10D6600030E0A901C201B1010F94FF01181614F0B6
:10D67000E12CF12CF301F182E082F30180819181B0
:10D6800082309105D9F08330910509F45CC001978F
:10D6900009F076C0F801E450F64F208131814281D3
:10D6A00053816B817C818D819E810E945FFB87FD10
:10D6B00067C082E090E0F301918380830450164FAD
:10D6C000B40180E090E00E9463FB9B01AC01F80193
:10D6D00060817181828193810E94D8FF9B01AC019E
:10D6E0006B817C818D819E810F94FF0187FD16C027
:10D6F0000E94E2B72B013C019501A8EEB3E00E9425
:10D70000C9FFDC01CB01840D951DA61DB71DE98164
:10D71000FA8180839183A283B38332C00E94E2B7EF
:10D72000E981FA810081118122813381DC01CB0101
:10D73000801B910BA20BB30BB7FD22C083E090E0DE
:10D74000F301918380834AE15AE16AE27AE18C2D08
:10D7500026960FB6F894DEBF0FBECDBFDF91CF91F6
:10D760001F910F91FF90EF90CF90BF90AF909F903F
:10D770008F907F906F905F904F903F902F90BECE94
:10D7800026960FB6F894DEBF0FBECDBFDF91CF91C6
:10D790001F910F91FF90EF90CF90BF90AF909F900F
:10D7A0008F907F906F905F904F903F902F90089553
:10D7B0004F925F926F927F928F929F92AF92BF92A1
:10D7C000CF92DF92EF92FF920F931F938091D1112E
:10D7D00081110FC01F910F91FF90EF90DF90CF90BC
:10D7E000BF90AF909F908F907F906F905F904F9081
:10D7F000089561DE0E94E2B72B013C016091FE13A7
:10D800007091FF13072E000C880B990B0E9465FB8B
:10D810002091021430910314409104145091051486
:10D82000B6E08B2E912C1CE3A12EB12CC12C7B01D8
:10D830008C016CEE79E08AEE99E0CFDEC0900214A4
:10D84000D0900314E0900414F09005148091080A1D
:10D850009091090ABC01990F880B990B0E9465FBF6
:10D860009B01AC01C701B6010F94FF011816CCF45F
:10D870006091110270911202072E000C880B990B17
:10D880000E9465FB9B01AC01C701B6010E945FFBD2
:10D8900087FF07C080E07BDB0F941D0175956795BE
:10D8A00001C060E06093D3118091F0099091F1097B
:10D8B000A091F209B091F3090097A105B105F9F023
:10D8C000A3019201281B390B4A0B5B0B57FD17C0B4
:10D8D0000E94D7B86B017C018091F4099091F50901
:10D8E000BC0180E090E00E9463FB9B01AC01C7019A
:10D8F000B6010E945FFB87FDA7C080E0F2DC80914B
:10D90000F6099091F709A091F809B091F9090097EB
:10D91000A105B10511F1A3019201281B390B4A0B96
:10D920005B0B57FD1AC089DC6B017C018091FA0901
:10D930009091FB09BC0180E090E00E9463FB9B0199
:10D94000AC01C701B6010E945FFB87FF7BC04EEDB3
:10D9500059E16DEE79E18FEFD1DD8091E60990918B
:10D96000E709A091E809B091E909A3019201281BF8
:10D97000390B4A0B5B0B57FD2DCF38E8430E33E1D3
:10D98000531E611C711C4092E6095092E709609297
:10D99000E8097092E9096091FC137091FD13072E5C
:10D9A000000C880B990B0E9465FB209106143091A6
:10D9B00007144091081450910914E3E08E2E912C25
:10D9C000FEE1AF2EB12CCC24CA947B018C0160EE19
:10D9D00079E084EE99E001DEC0900614D09007143F
:10D9E000E0900814F090091420E030E040EA50E4A0
:10D9F000C701B6010F94FF0187FD20C020E030E091
:10DA000046E153E4C701B6010E945FFB1816B4F06B
:10DA10006091FC137091FD13072E000C880B990B7D
:10DA20000E9465FB9B01AC01C701B6010E945FFB30
:10DA300087FD11C080E08093D411CCCE1092D41118
:10DA40007598C8CE03DC89CF4CEF59E16BE07AE1E1
:10DA500080E054DD54CF8FE7EECF0F931F93CF9329
:10DA6000DF93EC0188819981019719F40E94E2B754
:10DA700004C06A857B858C859D850E811F812885E4
:10DA80003985601B710B820B930B28EE33E040E06D
:10DA900050E00E947BFF8A819B81AC81BD81BC01EB
:10DAA000CD01620F731F841F951FDF91CF911F91CE
:10DAB0000F910895CF93DF93FC01208131812130B4
:10DAC000310569F4EC0182E090E0918380830E944B
:10DAD000E2B76A877B878C879D8781E001C080E001
:10DAE000DF91CF910895880F991F880F991FFC012E
:10DAF000EF51F34F4081518162817381FC01E55DFB
:10DB0000F54F4083518362837383E0919C09F091C8
:10DB10009D0982899389A489B5898093C2099093CC
:10DB2000C309A093C409B093C5098FEF9FEF9093E9
:10DB30009F0980939E090895CF93DF932FB7F894A0
:10DB4000EC01CC0FDD1FCC0FDD1FFE01EF51F34FB9
:10DB500060817181828193812FBF0E9465FBC55EC8
:10DB6000D54F288139814A815B810E94C4FBDF91B6
:10DB7000CF9108950E94D84F882319F00E9457969C
:10DB8000F9CF80919E0990919F09892BB9F708954B
:10DB90001F920F920FB60F9211240BB60F92BF92E5
:10DBA000CF92DF92EF92FF920F931F932F933F93A9
:10DBB0004F935F936F937F938F939F93AF93BF9395
:10DBC000EF93FF93CF93DF9300D01F92CDB7DEB7D3
:10DBD00080916E008B7F80936E0080916F008D7FAF
:10DBE00080936F007894C090BE09D090BF09E090F8
:10DBF000C009F090C109C114D104E104F104D1F1CC
:10DC00008091720E811104C080910A0A882391F1DB
:10DC10000E9494E6D701C601E9EBCE16EBE0DE06E2
:10DC2000E104F10420F088EB9BE0A0E0B0E0C81A2A
:10DC3000D90AEA0AFB0AC092BE09D092BF09E09253
:10DC4000C009F092C10990938900809388002091C7
:10DC500088003091890080918400909185004096E1
:10DC60002817390708F02DC1809184009091850014
:10DC7000409630C0E0909E09F0909F09E114F104B5
:10DC800071F1F7FE5DC180919C0990919D09892BEE
:10DC900009F04AC10E94D84F882309F41CC6E091BC
:10DCA000700E0DE4E09FF0011124E453FB4F8081DE
:10DCB00084FF11C60E94D84F882331F08091700EE6
:10DCC0008F5F8F708093700E10929D0910929C0947
:10DCD00088EC90E09093890080938800F2C0E090F7
:10DCE0009C09F0909D09E114F10409F446C180916A
:10DCF000720E8111F5C580910A0A8111F1C520913A
:10DD0000B9092111B7C2B12C4091C2095091C30980
:10DD10006091C4097091C509E0909C09F0909D093B
:10DD2000F70186899789A08DB18D84179507A6077D
:10DD3000B70708F496C44091B0095091B1096091B9
:10DD4000B2097091B309068D178D20A131A1AA27C0
:10DD5000419FB12D529FC001629F900D619F800D28
:10DD6000911D429FB00D811D9A1F519FB00D811DC5
:10DD70009A1F609FB00D811D9A1F509FB10D8A1F81
:10DD80009A1FB6958A1F9A1F349F800D911D359F4B
:10DD9000900D112423AD34AD820F931F9093B509DC
:10DDA0008093B40947A950AD61AD72ADA0E0B0E079
:10DDB000481759076A077B0720F45093B509409329
:10DDC000B4098091B4099091B5098134BCE99B07ED
:10DDD00008F00DC48132EEE49E0708F40BC496955A
:10DDE00087959695879524E02093B9098C01005278
:10DDF0001109011528E0120708F40EC4E12FFF27CE
:10DE0000EE0FFF1FEE0FFF1FCF0181559A4EFC0151
:10DE1000329625913491AA27039FA001029F410DBC
:10DE20005A1F06944A1F5A1F1124FC012591349150
:10DE3000241B350B2436310550F469E473E08EEA77
:10DE40009DE0A7D7C8010E94BAD324E630E08091B4
:10DE5000720E882309F4FFC3C901293B4BE0340744
:10DE600008F041C590938900809388008091B009A3
:10DE70009091B109A091B209B091B309820F931F9B
:10DE8000A11DB11D8093B0099093B109A093B2096F
:10DE9000B093B3092091880030918900809184006B
:10DEA0009091850040962817390748F480918400A6
:10DEB0009091850040969093890080938800B110DE
:10DEC000FAC4F8948091D211882321F080916E00D9
:10DED0008B7F03C080916E00846080936E00809180
:10DEE0006F00826080936F000F900F900F900F90E3
:10DEF000DF91CF91FF91EF91BF91AF919F918F9162
:10DF00007F916F915F914F913F912F911F910F9151
:10DF1000FF90EF90DF90CF90BF900F900BBE0F90CF
:10DF20000FBE0F901F9018950E94D84F882309F4B8
:10DF3000B1CE8091700E8F5F8F708093700EAACEDD
:10DF40000E94D84F882331F08091700E8F5F8F70C0
:10DF50008093700E11E0E11AF108F0929F09E092AF
:10DF60009E09EF2809F0B0CE8FEA99E19093FB1358
:10DF70008093FA130E94BA4BA7CE0E94D84F8823F1
:10DF800061F09091700E2DE4929FF0011124E45302
:10DF9000FB4F8081886080837F01F0929D09E09231
:10DFA0009C09E114F10409F462C1D70192965C91D5
:10DFB00092978091CB0411964C9158130AC0242F4C
:10DFC00030E080910B02082E000C990B28173907BE
:10DFD00031F05093CB0440930B020E94418D10927C
:10DFE000BA091092BB091092BC091092BD09F70141
:10DFF00087A990AD8134FCE99F0728F481320EE4B3
:10E00000900748F002C080E49CE996958795969524
:10E01000879524E007C0813117E2910730F096958B
:10E02000879522E02093B90908C021E02093B9091F
:10E030008032910510F480E290E08C0100521109C9
:10E04000011528E01207D8F0E12FFF27EE0FFF1F80
:10E05000EE0FFF1FCF0181559A4EFC01329645917C
:10E060005491AA27059F9001049F210D3A1F069401
:10E070002A1F3A1F1124FC01859194911CC098011C
:10E08000369527952C7F21553E4EF9018591949127
:10E09000F901329665917491A80147705527649FE4
:10E0A0009001659F300D749F300D112443E036952B
:10E0B00027954A95E1F7821B930B8436910550F41E
:10E0C00069E473E08EEA9DE064D6C8010E94BAD389
:10E0D00084E690E09093B8098093B7098091B909DC
:10E0E0008093B609E0919C09F0919D0983AD94ADB0
:10E0F0009093B5098093B40981343CE9930728F4DF
:10E1000081324EE4940748F002C080E49CE9969581
:10E1100087959695879524E007C0813167E2960739
:10E1200030F09695879522E02093B90908C021E048
:10E130002093B9098032910510F480E290E08C01BF
:10E1400000521109011588E01807D8F0E12FFF27C8
:10E15000EE0FFF1FEE0FFF1FCF0181559A4EFC01FE
:10E16000329645915491AA27059F9001049F210D55
:10E170003A1F06942A1F3A1F1124FC01859194919D
:10E180001CC09801369527952C7F21553E4EF901EC
:10E1900085919491F901329665917491A801477027
:10E1A0005527649F9001659F300D749F300D112499
:10E1B00063E0369527956A95E1F7821B930B8436C9
:10E1C000910550F469E473E08EEA9DE0E2D5C80160
:10E1D0000E94BAD384E690E0AC0160E070E0409326
:10E1E000B0095093B1096093B2097093B309909349
:10E1F000890080938800E0919C09F0919D098289B3
:10E200009389A489B589B695A79597958795B09573
:10E21000A095909581959F4FAF4FBF4F8093AC09CC
:10E220009093AD09A093AE09B093AF098093A8096C
:10E230009093A909A093AA09B093AB098093A4096C
:10E240009093A509A093A609B093A7098093A0096C
:10E250009093A109A093A209B093A3091092C209B7
:10E260001092C3091092C4091092C50940CD80EDE7
:10E2700097E030CDE0919C09F0919D094091A00973
:10E280005091A1096091A2097091A30982819381A3
:10E29000A481B581840F951FA61FB71F8093A00985
:10E2A0009093A109A093A209B093A3091816190687
:10E2B0001A061B060CF48F9AE0919C09F0919D09B7
:10E2C0004091A4095091A5096091A6097091A709F0
:10E2D00086819781A085B185840F951FA61FB71FE2
:10E2E0008093A4099093A509A093A609B093A709C8
:10E2F000181619061A061B0644F49FB7F894809165
:10E3000008018460809308019FBFE0919C09F0910F
:10E310009D094091A8095091A9096091AA0970919D
:10E32000AB0982859385A485B585840F951FA61FAB
:10E33000B71F8093A8099093A909A093AA09B09345
:10E34000AB09181619061A061B0644F49FB7F89471
:10E35000809108018062809308019FBFE0919C0931
:10E36000F0919D094091AC095091AD096091AE09C1
:10E370007091AF0986859785A089B189840F951F13
:10E38000A61FB71F8093AC099093AD09A093AE0967
:10E39000B093AF09181619061A061B060CF48C9ACE
:10E3A0008091A0099091A109A091A209B091A3091F
:10E3B000181619061A061B0684F5E0919C09F091BF
:10E3C0009D094289538964897589841B950BA60B25
:10E3D000B70B8093A0099093A109A093A209B093D1
:10E3E000A309809107024091E10C5091E20C6091E9
:10E3F000E30C7091E40C082E000C990BAA0BBB0BDC
:10E40000840F951FA61FB71F8093E10C9093E20C19
:10E41000A093E30CB093E40C8F988091A4099091A1
:10E42000A509A091A609B091A709181619061A0600
:10E430001B06BCF5E0919C09F0919D094289538926
:10E4400064897589841B950BA60BB70B8093A4096F
:10E450009093A509A093A609B093A70980910802FB
:10E460004091E50C5091E60C6091E70C7091E80C3E
:10E47000082E000C990BAA0BBB0B840F951FA61F2F
:10E48000B71F8093E50C9093E60CA093E70CB09334
:10E49000E80C9FB7F894809108018B7F8093080166
:10E4A0009FBF8091A8099091A909A091AA09B09154
:10E4B000AB09181619061A061B06BCF5E0919C0953
:10E4C000F0919D094289538964897589841B950B54
:10E4D000A60BB70B8093A8099093A909A093AA094A
:10E4E000B093AB09809109024091E90C5091EA0C7C
:10E4F0006091EB0C7091EC0C082E000C990BAA0BA0
:10E50000BB0B840F951FA61FB71F8093E90C909338
:10E51000EA0CA093EB0CB093EC0C9FB7F8948091AD
:10E5200008018F7D809308019FBF8091AC09909175
:10E53000AD09A091AE09B091AF09181619061A06D7
:10E540001B0684F5E0919C09F0919D09428953894D
:10E5500064897589841B950BA60BB70B8093AC0956
:10E560009093AD09A093AE09B093AF0980910A02D0
:10E570004091ED0C5091EE0C6091EF0C7091F00C0D
:10E58000082E000C990BAA0BBB0B840F951FA61F1E
:10E59000B71F8093ED0C9093EE0CA093EF0CB0930B
:10E5A000F00C8C988091C2099091C309A091C40984
:10E5B000B091C5090196A11DB11D8093C209909328
:10E5C000C309A093C409B093C5092150E0919C09E7
:10E5D000F0919D094289538964897589841795074B
:10E5E000A607B70708F48DCBBB24B3948DCB80E48A
:10E5F0009CE9F5CB8131F7E29F0720F0969587954E
:10E6000022E0F2CB21E02093B9098032910508F095
:10E61000EDCB80E290E0EACBA801569547954C7F80
:10E6200041555E4EFA0125913491FA013296659179
:10E630007491A80147705527649FC001659F900D94
:10E64000749F900D1124A3E096958795AA95E1F704
:10E65000281B390BEFCB80910A0A8111FDCBC90130
:10E6600001CC4091C2095091C3096091C4097091D5
:10E67000C509F701828D938DA48DB58D84179507FB
:10E68000A607B70708F0E4C04091BA095091BB094A
:10E690006091BC097091BD09068D178D20A131A133
:10E6A000AA27419FB12D529F6001629FD00C619FAC
:10E6B000C00CD11C429FB00DC11CDA1E519FB00D81
:10E6C000C11CDA1E609FB00DC11CDA1E509FB10D37
:10E6D000CA1EDA1EB695CA1EDA1E349FC00CD11CA3
:10E6E000359FD00C11248091B4099091B509FF9603
:10E6F000C816D90680F48C199D0940815181628128
:10E7000073816C01E12CF12CC416D506E606F706E0
:10E7100020F4CA0102C0808191818134BCE99B0749
:10E7200028F48132EEE49E0748F002C080E49CE9C0
:10E73000969587959695879524E007C08131F7E2F5
:10E740009F0730F09695879522E02093B90908C07D
:10E7500021E02093B9098032910510F480E290E025
:10E760008C0100521109011528E01207E8F0E12F91
:10E77000FF27EE0FFF1FEE0FFF1FCF0181559A4EAF
:10E78000FC01329625913491AA27039FA001029F94
:10E79000410D5A1F06944A1F5A1F1124FC0125914E
:10E7A0003491241B350B1EC0C801969587958C7F2C
:10E7B00081559E4EFC0125913491FC013296659164
:10E7C0007491A80147705527649FC001659F900D03
:10E7D000749F900D112443E0969587954A95E1F733
:10E7E000281B390B2436310550F469E473E08EEAB6
:10E7F0009DE0CFD2C8010E94BAD324E630E08091D8
:10E80000720E811104C080910A0A882339F0C9016F
:10E81000293B4BE0340708F081C001C0C901909347
:10E820008900809388008091BA099091BB09A091DA
:10E83000BC09B091BD09820F931FA11DB11D80932A
:10E84000BA099093BB09A093BC09B093BD0922CB30
:10E850002091B7093091B8098091720E811104C0DE
:10E8600080910A0A8823F1F0293B6BE03607D0F04B
:10E87000C90168EB7BE00F94A102883E13E0910789
:10E8800008F067C08854944FA901481B590B60E0F9
:10E8900070E04093BE095093BF096093C009709324
:10E8A000C1099C0130938900209388008091B609AA
:10E8B0008093B909EFCA10929D0910929C090E9499
:10E8C000D84F882309F4FDCA8091700E8F5F8F7036
:10E8D0008093700EF6CA10929F0910929E09F4C997
:10E8E0000E9494E60CCA68EB7BE00F94A102883E7C
:10E8F000F3E09F0780F48854944FA901481B590BFB
:10E9000060E070E04093BE095093BF096093C00976
:10E910007093C109A7CA88EB9BE0EFCF68EB7BE05F
:10E920000F94A102883E03E0900780F48854944F2E
:10E93000A901481B590B60E070E04093BE09509359
:10E94000BF096093C0097093C10969CF88EB9BE050
:10E95000EFCF88EB9BE098CF0895CF92DF92EF92B4
:10E96000FF920F931F93CF93DF936C017A018B017A
:10E97000C0E0D0E0CE15DF0589F0D8016D918D01A2
:10E98000D601ED91FC910190F081E02DC601199521
:10E99000892B11F47E0102C02196ECCFC701DF91D3
:10E9A000CF911F910F91FF90EF90DF90CF9008953E
:10E9B0000F94B8030F931F93CF93DF938C01EB0158
:10E9C000FC01808191810097B1F0688179816115A6
:10E9D000710579F0428153812C813D8142175307A3
:10E9E00040F00F940C048C819D81F8019583848301
:10E9F00013C00E94C9F588819981F80191838083B1
:10EA00008A819B81938382838C819D81958384837A
:10EA1000198218821B821A821D821C82DF91CF917B
:10EA20001F910F9108950F931F93CF93DF93EC01E4
:10EA300088819981009729F02A813B812617370721
:10EA400088F48B016F5F7F4F0F94D002009761F0C5
:10EA5000998388831B830A832C813D81232B11F4A6
:10EA6000FC01108281E001C080E0DF91CF911F9115
:10EA70000F910895EF92FF920F931F93CF93DF931F
:10EA8000FC01248135816115710511F480E018C005
:10EA900041155105A1F07B01EC018A01020F131F02
:10EAA000B801C1DF882391F3288139818C819D8150
:10EAB000B701820F931F0F940C041D830C8381E018
:10EAC000DF91CF911F910F91FF90EF900895EF92FA
:10EAD000FF920F931F93CF93DF93CDB7DEB72797A6
:10EAE0000FB6F894DEBF0FBECDBF7C01CB014AE06C
:10EAF0008E010F5F1F4FB8010E94DFFAF8010190ED
:10EB00000020E9F73197AF01401B510BB801C70155
:10EB1000B1DF27960FB6F894DEBF0FBECDBFDF91F1
:10EB2000CF911F910F91FF90EF900895FB014481C9
:10EB30005581608171819ECFCF93DF93EC018881F5
:10EB40009981009711F00E94C9F5198218821D82DF
:10EB50001C821B821A82DF91CF910895CF93DF939D
:10EB6000EC016115710559F0FB0101900020E9F7F6
:10EB70003197AF01461B570B7DDF811102C0CE01DB
:10EB8000DBDFCE01DF91CF910895EF92FF920F93DB
:10EB90001F93CF93DF93EC018B016115710549F051
:10EBA000CB010E948BFA7C01BC01CE013CDF8111BC
:10EBB00003C0CE01C1DF07C0FD82EC82B8018881AD
:10EBC00099810E9484FACE01DF91CF911F910F911C
:10EBD000FF90EF900895EF92FF920F931F93CF93C2
:10EBE000DF93EC017B018A01BA011DDF811103C0B3
:10EBF000CE01A2DF07C01D830C83B70188819981F4
:10EC00000F940C04CE01DF91CF911F910F91FF90D3
:10EC1000EF900895CF93DF93EC016115710551F0EA
:10EC2000FB0101900020E9F73197AF01461B570B1C
:10EC3000D2DF01C081DFCE01DF91CF910895CF9364
:10EC4000DF93EC01FB018617970751F0608171811A
:10EC50006115710521F044815581BDDF01C06CDF74
:10EC6000CE01DF91CF910895FC01808191810C94B8
:10EC7000C9F5FC011182108213821282158214825E
:10EC800084CFFC01118210821382128215821482B9
:10EC90006115710549F0FB0101900020E9F73197FA
:10ECA000AF01461B570B97CF0895CF93DF9300D04A
:10ECB0001F92CDB7DEB7611571058105910579F019
:10ECC0009B01AC0169833A834B835C830E94ADF660
:10ECD00029813A814B815C810E949DFF03C060E0E5
:10ECE00070E0CB010F900F900F900F90DF91CF91BC
:10ECF00008954F925F926F927F92EF92FF920F93DF
:10ED00001F93CF93DF93CDB7DEB7A1970FB6F894DB
:10ED1000DEBF0FBECDBF7C01FA01CB0119A22230AC
:10ED200008F42AE08E010F5D1F4F422E512C612CFA
:10ED3000712CBF01A30192010E947BFFF901CA015E
:10ED4000015011096A3014F4605D01C0695CD8019A
:10ED50006C93232B242B252B61F7B801C7010E944C
:10ED600097B5A1960FB6F894DEBF0FBECDBFDF9169
:10ED7000CF911F910F91FF90EF907F906F905F90D8
:10ED80004F900895DC01ED91FC910190F081E02D10
:10ED900019940C9497B50F931F93CF93C82F882382
:10EDA00019F0E1E8FEE10FC0ECECF2E284918F0192
:10EDB0000F5F1F4F8823A9F3082E000C990B0E94A8
:10EDC000CBA5F801F3CF84918F010F5F1F4F8823EC
:10EDD00039F0082E000C990B0E94CBA5F801F3CF57
:10EDE0008AE090E00E94CBA5C11137C0ECECF2E2C2
:10EDF00084918F010F5F1F4F882339F0082E000C7C
:10EE0000990B0E94CBA5F801F3CFEEE6FEE18491C9
:10EE10008F010F5F1F4F882339F0082E000C990BCC
:10EE20000E94CBA5F801F3CF8091560C882329F0DE
:10EE30008AE090E00E94CBA545C0E3E6FEE1849124
:10EE40008F010F5F1F4F882309F43CC0082E000C70
:10EE5000990B0E94CBA5F801F2CF40915B0C509129
:10EE60005C0C60915D0C70915E0C8AE59EE10E94E5
:10EE7000E18D8AE090E00E94CBA58091560C811133
:10EE800031C0CC2319F0EFE4FEE10FC0ECECF2E26C
:10EE900084918F010F5F1F4F8823A9F3082E000C68
:10EEA000990B0E94CBA5F801F3CF84918F010F5FDE
:10EEB0001F4F8823B9F0082E000C990B0E94CBA598
:10EEC000F801F3CFECECF2E284918F010F5F1F4F5A
:10EED000882309F4C2CF082E000C990B0E94CBA501
:10EEE000F801F2CFC1112DC0ECECF2E284918F0158
:10EEF0000F5F1F4F882339F0082E000C990B0E94DA
:10EF0000CBA5F801F3CFEEE3FEE184918F010F5F13
:10EF10001F4F882339F0082E000C990B0E94CBA5B7
:10EF2000F801F3CFECECF2E284918F010F5F1F4FF9
:10EF3000882339F0082E000C990B0E94CBA5F8010C
:10EF4000F3CF4091010D5091020D6091030D70912E
:10EF5000040D86E39EE10E94E18D4091050D5091E4
:10EF6000060D6091070D7091080D83E39EE10E94EC
:10EF7000E18D4091090D50910A0D60910B0D70913A
:10EF80000C0D80E39EE10E94E18D40910D0D5091AA
:10EF90000E0D60910F0D7091100D8DE29EE10E949B
:10EFA000E18D8AE090E00E94CBA5C1112DC0ECEC70
:10EFB000F2E284918F010F5F1F4F882339F0082EF2
:10EFC000000C990B0E94CBA5F801F3CFEFE0FEE116
:10EFD00084918F010F5F1F4F882339F0082E000C9A
:10EFE000990B0E94CBA5F801F3CFECECF2E28491EF
:10EFF0008F010F5F1F4F882339F0082E000C990BEB
:10F000000E94CBA5F801F3CF4091D6035091D703CE
:10F010006091D8037091D90386E09EE10E94E18D52
:10F020004091DA035091DB036091DC037091DD03C2
:10F0300083E09EE10E94E18D4091DE035091DF0369
:10F040006091E0037091E10380E09EE10E94E18D18
:10F050004091E2035091E3036091E4037091E50372
:10F060008DEF9DE10E94E18D8AE090E00E94CBA5AA
:10F07000C1112DC0ECECF2E284918F010F5F1F4FA4
:10F08000882339F0082E000C990B0E94CBA5F801BB
:10F09000F3CFEBEDFDE184918F010F5F1F4F8823CC
:10F0A00039F0082E000C990B0E94CBA5F801F3CF84
:10F0B000ECECF2E284918F010F5F1F4F882339F04F
:10F0C000082E000C990B0E94CBA5F801F3CF4091BC
:10F0D000BE035091BF036091C0037091C10382EDE4
:10F0E0009DE10E94958D4091C2035091C3036091B0
:10F0F000C4037091C5038FEC9DE10E94958D4091F2
:10F10000C6035091C7036091C8037091C9038CEC8A
:10F110009DE10E94958D4091CA035091CB0360916F
:10F12000CC037091CD0389EC9DE10E94958D8AE01E
:10F1300090E00E94CBA5C1112DC0ECECF2E28491CD
:10F140008F010F5F1F4F882339F0082E000C990B99
:10F150000E94CBA5F801F3CFEFE7FDE184918F0189
:10F160000F5F1F4F882339F0082E000C990B0E9467
:10F17000CBA5F801F3CFECECF2E284918F010F5FA5
:10F180001F4F882339F0082E000C990B0E94CBA545
:10F19000F801F3CF4091BA035091BB036091BC03D7
:10F1A0007091BD0386E79DE10E94E18D4091B60319
:10F1B0005091B7036091B8037091B90383E79DE163
:10F1C0000E94E18D4091B2035091B3036091B4036A
:10F1D0007091B50380E79DE10E94E18D8AE090E0A7
:10F1E0000E94CBA5C1112DC0ECECF2E284918F01FD
:10F1F0000F5F1F4F882339F0082E000C990B0E94D7
:10F20000CBA5F801F3CFECEFFCE184918F010F5F08
:10F210001F4F882339F0082E000C990B0E94CBA5B4
:10F22000F801F3CFECECF2E284918F010F5F1F4FF6
:10F23000882339F0082E000C990B0E94CBA5F80109
:10F24000F3CF4091D2035091D3036091D4037091D6
:10F25000D50383EF9CE10E94E18D4091CE03509154
:10F26000CF036091D0037091D10380EF9CE10E94A5
:10F27000E18D4091600C5091610C6091620C709135
:10F28000630C8DEE9CE10E94958D4091A2035091FC
:10F29000A3036091A4037091A5038AEE9CE10E94F0
:10F2A000E18D4091A6035091A7036091A80370914E
:10F2B000A90387EE9CE10E94E18D4091AA03509141
:10F2C000AB036091AC037091AD0384EE9CE10E94AE
:10F2D000E18D4091AE035091AF036091B003709106
:10F2E000B10381EE9CE10E94E18D8AE090E00E94F2
:10F2F000CBA5C1112DC0ECECF2E284918F010F5F20
:10F300001F4F882339F0082E000C990B0E94CBA5C3
:10F31000F801F3CFE3EDFCE184918F010F5F1F4F04
:10F32000882339F0082E000C990B0E94CBA5F80118
:10F33000F3CFECECF2E284918F010F5F1F4F882333
:10F3400039F0082E000C990B0E94CBA5F801F3CFE1
:10F3500040910B0A50910C0A60910D0A70910E0AAF
:10F360008AEC9CE10E94E18D40910F0A5091100AB5
:10F370006091110A7091120A87EC9CE10E94E18D64
:10F380004091130A5091140A6091150A7091160A5F
:10F3900084EC9CE10E94E18D8AE090E00E94CBA584
:10F3A000C1112DC0ECECF2E284918F010F5F1F4F71
:10F3B000882339F0082E000C990B0E94CBA5F80188
:10F3C000F3CFE0EBFCE184918F010F5F1F4F8823A7
:10F3D00039F0082E000C990B0E94CBA5F801F3CF51
:10F3E000ECECF2E284918F010F5F1F4F882339F01C
:10F3F000082E000C990B0E94CBA5F801F3CF609169
:10F40000181470E087EA9CE10E94028E4091191462
:10F4100050911A1460911B1470911C1484EA9CE1A1
:10F420000E94E18D8AE090E00E94CBA5C1112DC021
:10F43000ECECF2E284918F010F5F1F4F882339F0CB
:10F44000082E000C990B0E94CBA5F801F3CFE5E93B
:10F45000FCE184918F010F5F1F4F882339F0082E44
:10F46000000C990B0E94CBA5F801F3CFECECF2E273
:10F4700084918F010F5F1F4F882339F0082E000CF5
:10F48000990B0E94CBA5F801F3CF40912A19509116
:10F490002B1960912C1970912D198CE89CE10E9418
:10F4A000E18D2CEA35EC47E25EE360912E19709114
:10F4B0002F1980913019909131190F94B500AB013B
:10F4C000BC0189E89CE10E94C08D2CEA35EC47E242
:10F4D0005EE36091321970913319809134199091E3
:10F4E00035190E94C4FBAB01BC0186E89CE10E9477
:10F4F000C08D8AE090E00E94CBA5C1112DC0ECEC3C
:10F50000F2E284918F010F5F1F4F882339F0082E9C
:10F51000000C990B0E94CBA5F801F3CFE0E7FCE1CA
:10F5200084918F010F5F1F4F882339F0082E000C44
:10F53000990B0E94CBA5F801F3CFECECF2E2849199
:10F540008F010F5F1F4F882339F0082E000C990B95
:10F550000E94CBA5F801F3CF409136145091371497
:10F56000609138147091391487E69CE10E94E18D16
:10F570008AE090E0CF911F910F910C94CBA5CF938F
:10F58000DF9321E03DE0C6EDD3E0AEEBB3E080E0F9
:10F5900090E0FC01E95AF34E4591559165917491C3
:10F5A000F90141935193619371939F01FC01E95BD0
:10F5B000F34E45915591659174914993599369938F
:10F5C0007993FC01E95CF34E4591559165917491F5
:10F5D0004D935D936D937D93049680319105C9F6AB
:10F5E00080E090E0A8E4B4E48093BA039093BB0376
:10F5F000A093BC03B093BD038093B6039093B7036D
:10F60000A093B803B093B9038093B2039093B3036C
:10F61000A093B403B093B5031092D2031092D30316
:10F620001092D4031092D5031092CE031092CF0300
:10F630001092D0031092D10380E29EE4A0E0B0E0EB
:10F640008093600C9093610CA093620CB093630C58
:10F6500080E090E0A0E0B1E48093A2039093A30344
:10F66000A093A403B093A5038093A6039093A7034C
:10F67000A093A803B093A9038DEC9CECACECBEE383
:10F680008093AA039093AB03A093AC03B093AD0314
:10F6900080E090E0A0E8BFE38093AE039093AF03D7
:10F6A000A093B003B093B10383EC90E090938F0EDE
:10F6B00080938E0E8DEC90E09093930E8093920E3B
:10F6C0008BEE90E09093970E8093960E82E390E0FD
:10F6D0009093910E8093900E8CE390E09093950E12
:10F6E0008093940E8AE590E09093990E8093980E03
:10F6F0008CE0EBE0FAE0DF011D928A95E9F71092C9
:10F70000520C1092530C1092540C1092550C0E94F3
:10F710006BD810923614109237141092381410923D
:10F72000391487ED93EAA5E0B2E480932A19909307
:10F730002B19A0932C19B0932D1985E090EAA6E718
:10F74000BEE380932E1990932F19A0933019B09394
:10F7500031198CEC96E6A0E9B4E4809332199093C9
:10F760003319A0933419B09335191092560C80E0D8
:10F7700090E0A0EEBFE380935B0C90935C0CA093B1
:10F780005D0CB0935E0C1092720E1092710E0E947E
:10F790000AB0ECECF2E28491EF012196882339F073
:10F7A000082E000C990B0E94CBA5FE01F4CFE4E1DA
:10F7B000FCE18491EF012196882339F0082E000C9A
:10F7C000990B0E94CBA5FE01F4CFDF91CF91089554
:10F7D0002F923F924F925F926F927F928F929F9261
:10F7E000AF92BF92CF92DF92EF92FF920F931F934F
:10F7F000CF93DF93CDB7DEB7C256D1090FB6F894D9
:10F80000DEBF0FBECDBF2DB73EB7A1963FAF2EAF27
:10F81000A19767961FAE1EAE679784E690E0659647
:10F820009FAF8EAF65979E012B5A3F4F44E050E04B
:10F83000BE016B5B7F4FCE018D5A9F4F0E94D0AFB0
:10F840009E012B5A3F4F42E050E0BE016F5A7F4F5E
:10F85000CE018D5A9F4F0E94D0AF43E050E0BE01D1
:10F860006B5B7F4F8DE892E00F941304892B09F4B2
:10F8700042C026968FAD2697863539F08FE32696BF
:10F880008FAF269727961FAE2797ECECF2E2849174
:10F890008F010F5F1F4F882339F0082E000C990B42
:10F8A0000E94CBA5F801F3CFEBEFFBE184918F0130
:10F8B0000F5F1F4F882339F0082E000C990B0E9410
:10F8C000CBA5F801F3CFBE016B5B7F4F82EF9BE1CD
:10F8D0000E94268EE4EEFBE184918F010F5F1F4FA3
:10F8E000882339F0082E000C990B0E94CBA5F80153
:10F8F000F3CF45DE94C46DB67EB625961CAE1DAE24
:10F900001EAE1FAE259767961FAE1EAE67979E016F
:10F910002B5A3F4F41E050E0BE01635A7F4FCE016A
:10F920008D5A9F4F0E94D0AF80E1EDE5F2E0DE01FD
:10F93000919601900D928A95E1F780E1EDE6F2E073
:10F94000DE01519601900D928A95E1F780E1EDE795
:10F95000F2E08E010F5F1F4FD80101900D928A9542
:10F96000E1F76E96CFAC6E97D12C33E0C30ED11C6D
:10F97000CC0CDD1CCC0CDD1C8DB79EB78C199D0901
:10F980000FB6F8949EBF0FBE8DBFEDB7FEB7319690
:10F990004F012DB73EB72C193D090FB6F8943EBF65
:10F9A0000FBE2DBF8DB79EB701965C01EDB7FEB7B8
:10F9B000EC19FD090FB6F894FEBF0FBEEDBF2DB7D1
:10F9C0003EB72F5F3F4F79019E012B5A3F4FA60153
:10F9D000B401CE018D5A9F4F0E94D0AF9E012B5A89
:10F9E0003F4FA601B501CE018D5A9F4F0E94D0AF67
:10F9F0009E012B5A3F4FA601B701CE018D5A9F4F52
:10FA00000E94D0AF6E962FAD6E9730E02E5F3F4FC5
:10FA10008EEB93E0A3969FAF8EAFA397A6EDB3E0D6
:10FA200061E07DE080E090E040E050E024173507A1
:10FA300014F0640105C0F1E2CF2ED12CCC0EDD1EF6
:10FA4000C80ED91EF6012080318042805380FB0110
:10FA50002192319241925192BF012417350714F03F
:10FA6000650105C0E1E1CE2ED12CCC0EDD1EC80E05
:10FA7000D91EF60120803180428053802D923D9224
:10FA80004D925D922417350714F0670101C068019B
:10FA9000C80ED91EF6012080318042805380A39683
:10FAA000EEADFFADA3972192319241925192A39670
:10FAB000FFAFEEAFA3974F5F5F4F04964430510501
:10FAC00009F0B4CF9E012B5A3F4F44E050E06AEB5F
:10FAD00073E0CE018D5A9F4F0E94D0AF9E012B5AEA
:10FAE0003F4F44E050E066EB73E0CE018D5A9F4FEC
:10FAF0000E94D0AF9E012B5A3F4F44E050E062EB92
:10FB000073E0CE018D5A9F4F0E94D0AF9E012B5AB9
:10FB10003F4F44E050E062ED73E0CE018D5A9F4FBD
:10FB20000E94D0AF9E012B5A3F4F44E050E06EEC54
:10FB300073E0CE018D5A9F4F0E94D0AF9E012B5A89
:10FB40003F4F44E050E060E67CE0CE018D5A9F4F8D
:10FB50000E94D0AF9E012B5A3F4F40E150E062EA35
:10FB600073E0CE018D5A9F4F0E94D0AF9E012B5A59
:10FB70003F4F4CE050E06BE07AE0CE018D5A9F4F52
:10FB80000E94D0AF9E012B5A3F4F44E050E062E507
:10FB90007CE0CE018D5A9F4F0E94D0AF9E012B5A20
:10FBA0003F4F41E050E0BE01645A7F4FCE018D5A75
:10FBB0009F4F0E94D0AF9E012B5A3F4F44E050E030
:10FBC000BE016F5B7F4FCE018D5A9F4F0E94D0AF19
:10FBD0009E012B5A3F4F41E050E0BE01655A7F4FD6
:10FBE000CE018D5A9F4F0E94D0AF9E012B5A3F4F9E
:10FBF00041E050E0BE01665A7F4FCE018D5A9F4FC3
:10FC00000E94D0AF6C968FAD6C976B960FAD6B97D3
:10FC1000809F80011124E12CF12C9E012B5A3F4F33
:10FC200044E050E0E016F10661F0BE016F5B7F4FEB
:10FC3000CE018D5A9F4F0E94D0AFFFEFEF1AFF0AFF
:10FC4000ECCF66E374E1CE018D5A9F4F0E94D0AF96
:10FC50001AE011509E012B5A3F4F112359F044E0F6
:10FC600050E0BE016F5B7F4FCE018D5A9F4F0E94C7
:10FC7000D0AFEFCF41E050E0BE01675A7F4FCE01D9
:10FC80008D5A9F4F0E94D0AF9E012B5A3F4F41E0AB
:10FC900050E0BE01685A7F4FCE018D5A9F4F0E949F
:10FCA000D0AF6A968FAD6A97863069F569968FAD49
:10FCB0006997863041F580E00E941DD89E012B5A3D
:10FCC0003F4F44E050E06EE47CE0CE018D5A9F4F00
:10FCD0000E94D0AF9E012B5A3F4F44E050E06AE4AF
:10FCE0007CE0CE018D5A9F4F0E94D0AF9E012B5ACF
:10FCF0003F4F40E950E06AEB7BE0CE018D5A9F4FC9
:10FD00000E94D0AF39C09E012B5A3F4F44E050E0D3
:10FD1000BE016B5C7F4FCE018D5A9F4F0E94D0AFCA
:10FD20009E012B5A3F4F44E050E0BE016F5C7F4F75
:10FD3000CE018D5A9F4F0E94D0AF6A968FAD6A97C1
:10FD400069960FAD6997809F80011124E12CF12CF9
:10FD5000E016F10689F09E012B5A3F4F44E050E037
:10FD6000BE016F5B7F4FCE018D5A9F4F0E94D0AF77
:10FD70002FEFE21AF20AECCF9E012B5A3F4F41E0DF
:10FD800050E0BE01625A7F4FCE018D5A9F4F0E94B4
:10FD9000D0AF9E012B5A3F4F41E050E0BE01695A5F
:10FDA0007F4FCE018D5A9F4F0E94D0AF1CE0115063
:10FDB0009E012B5A3F4F44E050E0BE01112341F019
:10FDC0006F5B7F4FCE018D5A9F4F0E94D0AFEFCF18
:10FDD000635C7F4FCE018D5A9F4F0E94D0AF9E0132
:10FDE0002B5A3F4F44E050E0BE01675C7F4FCE018D
:10FDF0008D5A9F4F0E94D0AF9E012B5A3F4F44E037
:10FE000050E0BE016B5C7F4FCE018D5A9F4F0E9428
:10FE1000D0AF9E012B5A3F4F44E050E0BE016F5BD4
:10FE20007F4FCE018D5A9F4F0E94D0AF11113EC01F
:10FE30002596CCACDDACEEACFFAC259720E030E8ED
:10FE40004BE355E4C701B6010E945FFB882371F1C3
:10FE5000C0922A19D0922B19E0922C19F0922D19E8
:10FE60009E012B5A3F4F44E050E06EE279E1CE0113
:10FE70008D5A9F4F0E94D0AF9E012B5A3F4F44E0B6
:10FE800050E062E379E1CE018D5A9F4F0E94D0AFDE
:10FE90009E012B5A3F4F44E050E0BE016F5B7F4F05
:10FEA000CE018D5A9F4F0E94D0AF11C004E0015087
:10FEB00071F09E012B5A3F4F44E050E0BE016F5B52
:10FEC0007F4FCE018D5A9F4F0E94D0AFF0CF1F5F62
:10FED000153009F09ECF9E012B5A3F4F42E050E073
:10FEE000BE01615B7F4FCE018D5A9F4F0E94D0AF04
:10FEF00014E011509E012B5A3F4F112359F044E05A
:10FF000050E0BE016F5B7F4FCE018D5A9F4F0E9424
:10FF1000D0AFEFCF42E050E0BE01635B7F4FCE0138
:10FF20008D5A9F4F0E94D0AF9E012B5A3F4F41E008
:10FF300050E0BE01625A7F4FCE018D5A9F4F0E9402
:10FF4000D0AF19E011509E012B5A3F4F112359F0A9
:10FF500044E050E0BE016F5B7F4FCE018D5A9F4F52
:10FF60000E94D0AFEFCF41E050E066E57CE0CE01EB
:10FF70008D5A9F4F0E94D0AF9E012B5A3F4F44E0B5
:10FF800050E0BE016F5B7F4FCE018D5A9F4F0E94A4
:10FF9000D0AF11110EC025968CAD9DADAEADBFADED
:10FFA000259780935B0C90935C0CA0935D0CB093B1
:10FFB0005E0C1F5F153001F71CE011509E012B5A9B
:10FFC0003F4F42E050E0BE01112341F0655B7F4F9F
:10FFD000CE018D5A9F4F0E94D0AFEFCF675B7F4F0E
:10FFE000CE018D5A9F4F0E94D0AF9E012B5A3F4F9A
:10FFF00042E050E0BE01675B7F4FCE018D5A9F4FBC
:020000021000EC
:100000000E94D0AF9E012B5A3F4F44E050E0BE010A
:100010006F5B7F4FCE018D5A9F4F0E94D0AF9E01E4
:100020002B5A3F4F44E050E0BE016F5B7F4FCE0143
:100030008D5A9F4F0E94D0AF00E010E0B801625788
:10004000714F9E012B5A3F4F42E050E0CE018D5A36
:100050009F4F0E94D0AFB8016057714F9E012B5A3D
:100060003F4F42E050E0CE018D5A9F4F0E94D0AFEB
:100070000C5F1F4F0C30110509F714E0115071F09F
:100080009E012B5A3F4F44E050E0BE016F5C7F4F12
:10009000CE018D5A9F4F0E94D0AFF0CF1CE111507E
:1000A00071F09E012B5A3F4F44E050E0BE016F5B60
:1000B0007F4FCE018D5A9F4F0E94D0AFF0CF14E0FA
:1000C000115071F09E012B5A3F4F44E050E0BE01A9
:1000D0006F5B7F4FCE018D5A9F4F0E94D0AFF0CF04
:1000E00067962EAD3FAD679763968EAD9FAD6397D4
:1000F0002817390709F03BC00E940AB0ECECF2E285
:1001000084918F010F5F1F4F882339F0082E000C58
:10011000990B0E94CBA5F801F3CF6DE872E08EEA4F
:100120009DE00E94C97665966EAD7FAD6597645679
:10013000710987EC9BE10E94028E67964EAD5FAD20
:10014000679760E070E08AEB9BE10E94958DE7EB9A
:10015000FBE184918F010F5F1F4F882309F45AC080
:10016000082E000C990B0E94CBA5F801F2CFECE50C
:10017000F9E284918F010F5F1F4F882339F0082E19
:10018000000C990B0E94CBA5F801F3CFE7E9FBE146
:1001900084918F010F5F1F4F882339F0082E000CC8
:1001A000990B0E94CBA5F801F3CF63964EAD5FADDE
:1001B000639760E070E02AE08EEA9DE00E94797625
:1001C000E2E9FBE184918F010F5F1F4F882339F033
:1001D000082E000C990B0E94CBA5F801F3CF67966F
:1001E0004EAD5FAD679760E070E02AE08EEA9DE07B
:1001F0000E947976E2E8FBE184918F010F5F1F4F47
:10020000882339F0082E000C990B0E94CBA5F80129
:10021000F3CFB5D90FB6F8947EBE0FBE6DBE80E0A9
:100220000E94CB769091B90B81E08927A196EEAD23
:10023000FFADA1970FB6F894FEBF0FBEEDBFCE592C
:10024000DF4F0FB6F894DEBF0FBECDBFDF91CF9169
:100250001F910F91FF90EF90DF90CF90BF90AF90E4
:100260009F908F907F906F905F904F903F902F90D6
:1002700008952F923F924F925F926F927F928F924A
:100280009F92AF92BF92CF92DF92EF92FF920F9325
:100290001F93CF93DF93CDB7DEB7C456D1090FB606
:1002A000F894DEBF0FBECDBF60969FAF8EAF609754
:1002B0004DA75DAB6DAF23967FAF2397322EDC0148
:1002C000CD90DD90ED90FC9080915F0E9091600E4E
:1002D000A091610EB091620EC81AD90AEA0AFB0A0F
:1002E0006096EEADFFAD6097448155816681778160
:1002F0008091630E9091640EA091650EB091660E90
:100300008A019B01081B190B2A0B3B0B09AB1AAB8B
:100310002BAB3CAB40855185628573858091670E20
:100320009091680EA091690EB0916A0E8A019B01AE
:10033000081B190B2A0B3B0B09AF1AAF2BAF3CAFB5
:10034000448455846684778480916B0E90916C0E02
:10035000A0916D0EB0916E0E53014201881A990A58
:10036000AA0ABB0A09F4A6C080915F0C811141C0A2
:100370006091150270911602072E000C880B990BE4
:100380000E9465FB9B01AC01609102147091031403
:1003900080910414909105140E945FFB87FF29C08F
:1003A00040926B0E50926C0E60926D0E70926E0EBB
:1003B000ECECF2E284918F010F5F1F4F882339F03C
:1003C000082E000C990B0E94CBA5F801F3CFE8EBA7
:1003D000FEE184918F010F5F1F4F882339F0082EB3
:1003E000000C990B0E94CBA5F801F3CF812C912C26
:1003F0005401C501B4010E9465FB14E0319EF00177
:100400001124EC59F34F20813181428153810E94A4
:10041000C4FB0F941D012B013C0197FF08C0709491
:10042000609450944094411C511C611C711C60915B
:100430000D0D70910E0D80910F0D9091100D0F9478
:100440001D019B01AC01A8ECB0E00E94B9FF64154E
:100450007505860597058CF56096EEADFFAD609746
:1004600084859585A685B78580936B0E90936C0ED9
:10047000A0936D0EB0936E0EECECF2E284918F01BE
:100480000F5F1F4F882339F0082E000C990B0E9434
:10049000CBA5F801F3CFE9E9FEE184918F010F5F6D
:1004A0001F4F882339F0082E000C990B0E94CBA512
:1004B000F801F3CF812C912C5401D701C601882774
:1004C000B7FD83959927AA27BB27182F29A93AA9F1
:1004D0004BA95CA957FD126089AD9AADABADBCAD1F
:1004E000B7FD1460B7FC1860C501B4010E9465FB3C
:1004F000A4E03A9EF0011124EC59F34F20813181A0
:10050000428153810E94C4FB4B015C0120E030E03A
:10051000A9010F94FF0118164CF420E030E040E0F0
:100520005FE3C501B4010E94D9FF08C0A501940191
:1005300060E070E080E09FE30E94D8FF0F941D010F
:1005400022966CAF7DAF8EAF9FAF229780916F0EDA
:100550008F5F8F70A1968FAFA1978091700EA1963B
:100560000FADA197801303C00E945796F6CFE0917C
:100570006F0E2E2F30E03CA72BA73DE4E39FF00148
:100580001124E453FB4F108212A3D701C601F7FEDA
:1005900007C088279927DC018C199D09AE09BF097E
:1005A00082839383A483B5838DE40BA51CA5809FD0
:1005B000F001819FF00D1124E453FB4F89A99AA902
:1005C000ABA9BCA9B7FF07C0B095A0959095819540
:1005D0009F4FAF4FBF4F86839783A087B1878DE42E
:1005E0000BA51CA5809FF001819FF00D1124E45301
:1005F000FB4F89AD9AADABADBCADB7FF07C0B095B1
:10060000A095909581959F4FAF4FBF4F828793875D
:10061000A487B5878DE40BA51CA5809FF001819F61
:10062000F00D1124E453FB4F22962CAD3DAD4EADA1
:100630005FAD229726873787408B518B428153814C
:10064000648175810681178120853185041715071E
:100650002607370714F48A019B018DE4ABA5BCA5DE
:100660008A9FF0018B9FF00D1124E453FB4F82858C
:100670009385A485B58580179107A207B30774F405
:1006800022968CAD9DADAEADBFAD22978017910780
:10069000A207B30774F4D901C80111C022960CADAA
:1006A0001DAD2EAD3FAD2297081719072A073B074E
:1006B00034F022968CAD9DADAEADBFAD22972DE44A
:1006C0000BA51CA5209FF001219FF00D1124E453E0
:1006D000FB4F828B938BA48BB58B0697A105B1053D
:1006E00010F40C94278DDF01A95BBF4F809100149B
:1006F000909101148D939C933182452B462B472B6F
:1007000009F08E988DE40BA51CA5809FF001819FB8
:10071000F00D1124E453FB4F86819781A085B185AC
:10072000892B8A2B8B2B41F09FB7F894809108017D
:100730008D7F809308019FBF8DE40BA51CA5809F32
:10074000F001819FF00D1124E453FB4F82859385C6
:10075000A485B585892B8A2B8B2B41F09FB7F89404
:10076000809108018F7E809308019FBF22962CAD57
:100770003DAD4EAD5FAD2297232B242B252BB1F041
:1007800080917D0C882319F0815080937D0C31106D
:1007900004C08B9880E280937D0C0091D20320905E
:1007A000D3033090D4031091D50308C00091CE0339
:1007B0002090CF033090D0031091D103202F322D01
:1007C000432D512F6DA57DA98DAD23969FAD239708
:1007D0000E945FFB87FD02C00C941F8DC701B6010C
:1007E0000E9465FB20911B0A30911C0A40911D0A52
:1007F00050911E0A0E94C4FB2B013C01698B7A8B2D
:100800008B8B9C8B69A97AA98BA99CA90E9465FBFB
:1008100020911F0A3091200A4091210A5091220A0A
:100820000E94C4FB6DA77EA78FA798AB6D8B7E8BB4
:100830008F8B988F69AD7AAD8BAD9CAD0E9465FBB7
:100840002091230A3091240A4091250A5091260ACA
:100850000E94C4FB6B017C01698F7A8F8B8F9C8F08
:100860002091270A3091280A4091290A50912A0A9A
:10087000C501B4010E94C4FB6D8F7E8F8F8F98A33A
:100880002DE44BA55CA5249FF001259FF00D1124BC
:10089000E453FB4F228133814481558129AB3AAB2C
:1008A0004BAB5CAB2630310541055105E4F4868045
:1008B0009780A084B18436E083169104A104B1042A
:1008C00094F482849384A484B58446E084169104CD
:1008D000A104B10444F4DC01CB01BF7787A790AB3E
:1008E000A1ABB2AB34C0A3019201C301B2010E941B
:1008F000C4FB2B013C012DA53EA54FA558A9CA015B
:10090000B9010E94C4FB9B01AC01C301B2010E946A
:10091000D9FF4B015C01A7019601C701B6010E94F6
:10092000C4FB9B01AC01C501B4010E94D9FF0F9427
:1009300044022DE4ABA5BCA52A9FF0012B9FF00D2E
:100940001124E453FB4F67A770AB81AB92AB8DE4EE
:100950002BA53CA5829FF001839FF00D1124E45349
:10096000FB4F87A590A9A1A9B2A9A0968CAF9DAF76
:10097000AEAFBFAFA0979C01AD0160E070E080E832
:100980009FE30F94B5002E966CAF7DAF8EAF9FAFF7
:100990002E979B01AC01602F722D832D912F0E9409
:1009A000C4FB6B017C0180916F0E9091700E891BCE
:1009B0008F7027968FAF2797A701960160E074E2AA
:1009C00084E799E40F94B5000F940A024B015C018F
:1009D00027968FAD279782508630C0F58091600CA6
:1009E0009091610CA091620CB091630C88169906ED
:1009F000AA06BB0658F588199909AA09BB09BC01C2
:100A0000CD01660F771F881F991F2796AFAD2797D7
:100A10000A2F10E020E030E0A90198010E947BFF3E
:100A2000CA01B9010E9463FB0F940A02680D791D87
:100A30008A1D9B1D0E9463FB9B01AC0160E074E278
:100A400084E799E40F94B5006B017C01A70196013E
:100A5000A0966CAD7DAD8EAD9FADA0970E94C4FBFE
:100A600064966CAF7DAF8EAF9FAF64978DE4EBA5BE
:100A7000FCA58E9F80018F9F100D112404531B4FE6
:100A800064962CAD3DAD4EAD5FAD6497D8019396A5
:100A90002D933D934D935C93969752962D913D9156
:100AA0004D915C91559729AF3AAF4BAF5CAFCA01FE
:100AB000B9010E9463FB6DA77EA78FA798ABA70122
:100AC00096010E94C4FB0F949F000F9422016A9626
:100AD0006CAF7DAF8EAF9FAF6A97F80167AB70AF19
:100AE00081AF92AF8E010F5E1F4F24961FAF0EAFE6
:100AF00024970051110966961FAF0EAF669706ED59
:100B000013E06C961FAF0EAF6C978E010F5D1F4FF9
:100B10001AA709A766960EAD1FAD669726961FAF5A
:100B20000EAF2697212C312C10E81DAB0FE30DAF33
:100B30002496AEADBFAD24976D917D918D919D9121
:100B40002496BFAFAEAF2497A70196010E94C4FBC5
:100B50002696EEADFFAD26976193719381939193A5
:100B60002696FFAFEEAF26974B015C01E894B7F8ED
:100B70006C96AEADBFAD6C974D905D906D907D90D5
:100B80006C96BFAFAEAF6C97A3019201C501B401E3
:100B90000F94FF011816A4F4A5019401C301B2013A
:100BA0000F94B5005B018C019B01AC01B1018DA9D3
:100BB0009DAD0F94FF0118161CF415010DAB1DAF70
:100BC00024960EAD1FAD249729A53AA50217130749
:100BD00009F0AECF20E030E040E85FE3B1018DA93D
:100BE0009DAD0E945FFB87FF4BC07E0131E1E30EAC
:100BF000F11C66960EAD1FAD669791014DA95DADD6
:100C0000D8016D917D918D919C910E94C4FBF8015A
:100C100061937193819391938F01EE15FF0569F7AD
:100C20008DE42BA53CA5829F8001839F100D11248C
:100C300004531B4F91014DA95DAD64966CAD7DAD24
:100C40008EAD9FAD64970E94C4FBD80193966D93BF
:100C50007D938D939C9396976A966CAD7DAD8EAD8A
:100C60009FAD6A970E9463FB91014DA95DAD0E9403
:100C7000C4FB0F942201F80167AB70AF81AF92AF54
:100C80002E962CAD3DAD4EAD5FAD2E976DA57EA5DC
:100C90008FA598A90E94C4FB6DAB7EAB8FAB98AFBC
:100CA00009A91AA92BA93CA9012B022B032B59F541
:100CB0008DE40BA51CA5809FF001819FF00D1124F0
:100CC000E453FB4F86819781A085B185892B8A2BC0
:100CD0008B2BC9F482859385A485B585892B8A2BB6
:100CE0008B2B89F42091B6033091B7034091B80360
:100CF0005091B9036DA97EA98FA998AD0E94C4FB3C
:100D00000F949F0035C222962CAD3DAD4EAD5FAD28
:100D10002297232B242B252B49F06091BA03709145
:100D2000BB038091BC039091BD0308C06091B203E6
:100D30007091B3038091B4039091B5032DA93EA99E
:100D40004FA958AD0E94C4FB0F949F000F9422013D
:100D50006B017C0180917E0C90917F0CA091800CA6
:100D6000B091810C09AD1AAD2BAD3CAD8017910748
:100D7000A207B30708F4E9C029A93AA94BA95CA9BD
:100D8000232B242B252B61F12091690C30916A0CC7
:100D900040916B0C50916C0C2C153D054E055F0578
:100DA000F8F469AD7AAD8BAD9CAD0E946CFF4B0140
:100DB0005C01A701960169A97AA98BA99CA90E9447
:100DC0006CFF86169706A806B90650F4C501B40153
:100DD00029A93AA94BA95CA90E947BFF69017A0164
:100DE0008DE40BA51CA5809FF001819FF00D1124BF
:100DF000E453FB4F86809780A084B18481149104D2
:100E0000A104B10441F120916D0C30916E0C409120
:100E10006F0C5091700C2C153D054E055F05D8F4F4
:100E200069AD7AAD8BAD9CAD0E946CFF2B013C018E
:100E3000A7019601C501B4010E946CFF4616570632
:100E40006806790640F4C301B201A50194010E942D
:100E50007BFF69017A018DE40BA51CA5809FF00141
:100E6000819FF00D1124E453FB4F82849384A4846A
:100E7000B58481149104A104B10441F12091710C55
:100E80003091720C4091730C5091740C2C153D05EF
:100E90004E055F05D8F469AD7AAD8BAD9CAD0E946F
:100EA0006CFF2B013C01A7019601C501B4010E9412
:100EB0006CFF461657066806790640F4C301B20176
:100EC000A50194010E947BFF69017A018DE40BA5C5
:100ED0001CA5809FF001819FF00D1124E453FB4F6E
:100EE00086849784A088B18881149104A104B104F8
:100EF00009F442C12091750C3091760C4091770C29
:100F00005091780C2C153D054E055F0508F034C155
:100F100069AD7AAD8BAD9CAD0E946CFF2B013C019D
:100F2000A7019601C501B4010E946CFF4616570641
:100F30006806790608F020C1C301B201A501940139
:100F40000E947BFF69017A0117C129A93AA94BA91F
:100F50005CA9232B242B252BB9F16091690C70918E
:100F60006A0C80916B0C90916C0C6C157D058E0554
:100F70009F0550F50E9463FB2DA53EA54FA558A9DE
:100F80000E94C4FB4B015C0169A97AA98BA99CA9A9
:100F90000E9465FB2B013C01C701B6010E9463FB67
:100FA000A30192010E94C4FBA50194010F94FF01CB
:100FB000181654F4A3019201C501B4010F94B500B1
:100FC0000F9422016B017C018DE40BA51CA5809F71
:100FD000F001819FF00D1124E453FB4F46805780B0
:100FE000608471844114510461047104A9F1609119
:100FF0006D0C70916E0C80916F0C9091700C6C1553
:101000007D058E059F0540F50E9463FB2DA53EA53D
:101010004FA558A90E94C4FB4B015C01C301B2015A
:101020000E9465FB2B013C01C701B6010E9463FBD6
:10103000A30192010E94C4FBA50194010F94FF013A
:10104000181654F4A3019201C501B4010F94B50020
:101050000F9422016B017C018DE40BA51CA5809FE0
:10106000F001819FF00D1124E453FB4F428453841F
:10107000648475844114510461047104A9F1609180
:10108000710C7091720C8091730C9091740C6C15B2
:101090007D058E059F0540F50E9463FB2DA53EA5AD
:1010A0004FA558A90E94C4FB4B015C01C301B201CA
:1010B0000E9465FB2B013C01C701B6010E9463FB46
:1010C000A30192010E94C4FBA50194010F94FF01AA
:1010D000181654F4A3019201C501B4010F94B50090
:1010E0000F9422016B017C018DE40BA51CA5809F50
:1010F000F001819FF00D1124E453FB4F8684978407
:10110000A088B18881149104A104B104A9F160916F
:10111000750C7091760C8091770C9091780C6C1511
:101120007D058E059F0540F50E9463FB2DA53EA51C
:101130004FA558A90E94C4FB2B013C01C501B40175
:101140000E9465FB4B015C01C701B6010E9463FB75
:10115000A50194010E94C4FBA30192010F94FF0119
:10116000181654F4A5019401C301B2010F94B500FF
:101170000F9422016B017C018DE42BA53CA5829F7D
:101180008001839F100D112404531B4FF801ED5B68
:10119000FF4FC082D182E282F382C701B6010E9472
:1011A00063FB6B017C012DA93EA94FA958AD0F949B
:1011B000B5006A966CAF7DAF8EAF9FAF6A97D801CE
:1011C000D3966D937D938D939C93D69720E030E0DA
:1011D00040E85BE4C701B6010E94C4FB20E034E2B2
:1011E00044EF59E40F94B5000F941D01F801668F88
:1011F000778F80A391A3F3A1FDABD8019496BC9106
:10120000BDAFF801F5A12396FFAF2397D8019696BD
:10121000BC912596BFAF259702EA13E06C961FAFED
:101220000EAF6C972E0111E1410E511C42EA242EA3
:1012300043E0342E66966EAC7FAC66970DA90EAF78
:101240001DAD19ABF9AFBDA710E0D3018D909D90F6
:10125000AD90BD903D01E894B7F8F101C190D190F7
:10126000E190F1901F01A7019601C501B4010F940F
:10127000FF01181674F5112339F12DA93DAD239600
:101280004FAD239725965FAD2597C701B6010E9404
:10129000C4FB6B017C012EAD39A949AD5DA5C5012B
:1012A000B4010E94C4FBA70196010F94FF01181618
:1012B0007CF4A5019401C701B6010F94B5006EAF8F
:1012C00079AB89AF9DA704C0CEAED9AAE9AEFDA681
:1012D00011E06414750409F0B8CF27960FAD279775
:1012E000002309F455C1C0904B0ED0904C0EE090F5
:1012F0004D0EF0904E0E2DEB37E346E855E3B60168
:10130000C7010E945FFB87FD43C19601A7016DA93C
:101310007DAD23968FAD239725969FAD25970E948F
:101320005FFB87FD05C00C2D2D2C3E2C1F2D08C00A
:101330000DA92DAC23963FAC239725961FAD25977D
:101340009601A701602F722D832D912F0F94B50068
:10135000A5966CAF7DAF8EAF9FAFA5972FE43EE013
:1013600062963FAF2EAF629780E090E0A0E8BFE3C7
:101370002A968CAF9DAFAEAFBFAF2A972B961FAE0C
:101380002B976296AEADBFAD62976D917D918D91B9
:101390009D916296BFAFAEAF6297A5962CAD3DAD65
:1013A0004EAD5FADA5970E94C4FB6B017C016696B4
:1013B000EEADFFAD669781909190A190B190669649
:1013C000FFAFEEAF66972B96FFAD2B97FF23B1F0E3
:1013D0002A962CAD3DAD4EAD5FAD2A970E94C4FB61
:1013E0006B017C012A962CAD3DAD4EAD5FAD2A97C9
:1013F000C501B4010E94C4FB4B015C01A50194012D
:10140000C701B6010F94FF0120E030E0A9011816D2
:101410002CF5C501B4010F94FF0118164CF020E023
:1014200030E0A901C701B6010E945FFB87FF05C03C
:10143000A5019401C701B60124C02401350177FA42
:10144000709477F87094A3019201C701B6010F94CC
:10145000FF0118165CF52601370128C0C501B4014B
:101460000E945FFB87FD09C020E030E0A901C701B1
:10147000B6010F94FF0118164CF4A7019601C5019F
:10148000B4010E94D8FF2B013C0110C02601370196
:1014900077FA709477F87094A5019401C301B201B2
:1014A0000F94FF01181614F0240135016C96AEADAF
:1014B000BFAD6C97CD90DD90ED90FD906C96BFAF79
:1014C000AEAF6C97A7019601C301B2010F94FF0163
:1014D0001816ECF4A3019201C701B6010F94B500F0
:1014E0009B01AC012A966CAD7DAD8EAD9FAD2A9768
:1014F0000E94C4FB2A966CAF7DAF8EAF9FAF2A9738
:101500002B96BFAD2B97BF5F2B96BFAF2B976296E5
:10151000EEADFFAD6297EF55FE4009F032CF2B964E
:101520003FAD2B97332381F02A962CAD3DAD4EADC8
:101530005FAD2A97602F722D832D912F0E94C4FBDF
:10154000062F272E382E192F24EA30E74DE75FE3C8
:10155000602F722D832D912F0E94C4FB6B017C01A3
:101560009B01AC016091790C70917A0C80917B0C9D
:1015700090917C0C0F94FF011816DCF4A7019601E2
:101580006EAD79A989AD9DA50F94FF0118168CF455
:101590008DE40BA51CA5809FF001819FF00D112407
:1015A000E453FB4F8081846080830EAD29A839AC61
:1015B0001DA58DE42BA53CA5829FF001839FF00D16
:1015C0001124E453FB4F802F922DA32DB12F83A71D
:1015D00094A7A5A7B6A76A966CAD7DAD8EAD9FAD5D
:1015E0006A9790589B01AC010E94D9FFA0962CAD40
:1015F0003DAD4EAD5FADA0970E94C4FB9B01AC0119
:101600006BE077ED83E29BE30E94D8FF0F944402E6
:101610006B017C019B01AC01602F722D832D912FFA
:101620000E945FFB87FD04C00C2D2D2C3E2C1F2D2E
:101630008DE44BA55CA5849FF001859FF00D1124DE
:10164000E453FB4F802F922DA32DB12F87A390A79A
:10165000A1A7B2A7B0809601A7016DA97DAD239681
:101660008FAD239725969FAD25970E945FFB181697
:1016700014F481E001C083E03DE4C32EABA5BCA51A
:10168000CA9E9001CB9E300D1124F901E453FB4F0B
:101690007F01B82AB08280E1FE013196AFE4BEE05E
:1016A00001900D928A95E1F78DA99DAD2396AFAD7E
:1016B00023972596BFAD259780934B0E90934C0EA4
:1016C000A0934D0EB0934E0E8EAD99A9A9ADBDA5B8
:1016D0008093790C90937A0CA0937B0CB0937C0C44
:1016E0002DA93DAD23964FAD239725965FAD259748
:1016F00060E070E080E89FE30F94B5004B015C016F
:101700009B01AC016EAD79A989AD9DA50E94C4FB7A
:101710006DA37EA38FA398A7A5019401602F722DBE
:10172000832D912F0E94C4FB69A37AA38BA39CA352
:10173000AE014B5D5F4FBE016F5D7F4FC7010E94E1
:1017400047E4A1960FADA19700936F0E80E16096DC
:10175000EEADFFAD6097AFE5BEE001900D928A95CA
:10176000E1F780916F0E9091700E891B8F7084301D
:1017700048F41091700EF12C00E080E090E02DE430
:10178000E22EA5C04090700E82E0840D8F708BA772
:10179000F0906F0E8FEF8F0D8F70F82EC89EC001E6
:1017A00011249C0124533B4F69018FEF8F0D8F70E3
:1017B000F82E882E880F99083DE4389D8001399DC8
:1017C000100D112404531B4FD8016C9062FCD1CF33
:1017D0000115110509F476C0C114D10409F472C0D1
:1017E0009B967C909B979C96AC909C979D96BC906A
:1017F0009D979E96EC909E97272D3A2D4B2D5E2D12
:1018000097966D917D918D919C919A970E945FFB27
:10181000882309F457C061FC40C0F60127A030A41A
:1018200041A452A4A2019101672D7A2D8B2D9E2DEA
:101830000E945FFB18168CF5A2019101C201B10153
:101840000E94C4FB1B012C01F80183A994A9A5A93E
:10185000B6A9BC01CD0190589B01AC010E94D9FFF3
:10186000D8019F962D913D914D915C91D2970E9408
:10187000C4FB9B01AC01C201B1010E94D8FF0F94CF
:1018800044021B016C019B01AC01672D7A2D8B2D4D
:101890009E2D0E945FFB87FF04C0272C3A2CCB2C87
:1018A000DE2CBDE4B89DF001B99DF00D1124E45388
:1018B000FB4FC101D60187A390A7A1A7B2A7862D90
:1018C0008160808368010BA5F0126FCF52CF209109
:1018D0006F0E121791F0E19E90011124A90144535B
:1018E0005B4F6A016F2D702F0E94D1E31F5F1F7045
:1018F0008F2D902FFC2C0D2DEACF6F2D702F0E9475
:10190000D1E3F090700E00E010E08DE4E82EAF2CF3
:101910000F2C000CBB0880916F0E90E0A816B90642
:1019200009F456C0EA9CC001EB9C900D1124DC0127
:10193000A453BB4F6D010115110509F443C0F80113
:10194000808180FD03C08C9180FF3CC0D8019396BC
:101950002D913D914D915C91969760E070E080E80B
:101960009FE30F94B5002B013C01EA9CF001EB9C36
:10197000F00D1124E453FB4F9B01AC0167A170A54E
:1019800081A592A50E94C4FB69A37AA38BA39CA303
:10199000A3019201F80167A170A581A592A50E94FB
:1019A000C4FB6DA37EA38FA398A7AE014F5D5F4FCD
:1019B000BE016B5D7F4FC8010E9447E4D8018C9146
:1019C0008E7F8C9381E08F0D8F70F82E86019FCFD4
:1019D00001151105E1F1F80123A134A145A156A19A
:1019E00060E070E080E89FE30F94B5006B017C013C
:1019F0002DEC3CEC4CE45DE30E94C4FB69A37AA3AC
:101A00008BA39CA3A7019601D80197966D917D9118
:101A10008D919C919A970E94C4FB6DA37EA38FA386
:101A200098A7AE014F5D5F4FBE016B5D7F4FC80150
:101A30000E9447E4F80180818E7F808308C00DA555
:101A40002DA83DAC23961FAD23970C94EE83CC5963
:101A5000DF4F0FB6F894DEBF0FBECDBFDF91CF9141
:101A60001F910F91FF90EF90DF90CF90BF90AF90BC
:101A70009F908F907F906F905F904F903F902F90AE
:101A800008958091CB049FB780FF09C0F89480919E
:101A900008018160809308019FBF8FEF08C0F89410
:101AA000809108018E7F809308019FBF81E0809321
:101AB00007028091CB049FB781FF09C0F894809101
:101AC00008018860809308019FBF8FEF08C0F894D9
:101AD00080910801877F809308019FBF81E08093F8
:101AE00008028091CB049FB782FF09C0F8948091CF
:101AF00008018F77809308019FBF8FEF08C0F8948B
:101B0000809108018068809308019FBF81E08093E5
:101B100009028091CB0483FF03C08D988FEF02C030
:101B20008D9A81E080930A0208950F931F93CF93BB
:101B3000DF9300D01F92CDB7DEB7FC0124918C015A
:101B40000F5F1F4F222379F0822F220F990B4983B9
:101B50005A836B837C830E94CBA5C80149815A813B
:101B60006B817C81EACF2AE08EEA9DE00F900F9096
:101B70000F900F90DF91CF911F910F910C94797678
:101B8000CF92DF92EF92FF92CF93DF936A017B01B6
:101B9000FC012491EC012196222339F0822F220F9F
:101BA000990B0E94CBA5CE01F3CF42E050E0C701D4
:101BB000B601DF91CF91FF90EF90DF90CF900C9422
:101BC000A7C7CF92DF92EF92FF92CF93DF936A0184
:101BD0007B01FC012491EC012196222339F0822F14
:101BE000220F990B0E94CBA5CE01F3CF42E050E02B
:101BF000C701B601DF91CF91FF90EF90DF90CF90BA
:101C00000C94A7C70F931F93CF93DF931F921F923C
